:020000040800F2
:100000004C2801203B05000885040008290302084C
:10001000890400088B0400088D040008000000001B
:100020000000000000000000000000008F04000835
:1000300091040008000000009304000895040008E3
:1000400097040008990400089B0400089D04000818
:100050009F040008A1040008A3040008A5040008E8
:10006000A7040008A9040008AB040008AD040008B8
:10007000AF040008B1040008B3040008B504000888
:10008000B7040008B9040008BB040008BD04000858
:10009000BF040008C1040008C3040008C504000828
:1000A000C7040008C9040008CB040008CD040008F8
:1000B000CF040008D1040008D3040008D5040008C8
:1000C000D7040008D9040008DB040008DD04000898
:1000D000DF040008E1040008E3040008E504000868
:1000E000E7040008E9040008EB040008ED04000838
:1000F000EF040008F1040008F3040008F504000808
:10010000F7040008F9040008FB040008FD040008D7
:10011000FF040008010500080305000805050008A4
:1001200007050008090500080B0500080D05000873
:100130000F05000811050008130500081505000843
:1001400017050008190500081B0500081D05000813
:100150001F050008210500082305000825050008E3
:1001600027050008290500082B0500082D050008B3
:100170002F05000831050008330500083505000883
:080180003705000839050008ED
:10020000DECEA5ED02003078463430370000000025
:1002100000000000000044523234305F3139303881
:100220000000000000004170706C69636174696FC8
:100230006E00000000000000000000000000000050
:100240000000000000000503BF00DAF7DECEA5EDD8
:100250000200307846343037000000000000000013
:10026000000053504C6174436F6E74726F6C6C6518
:1002700072004170706C69636174696F6E00000098
:10028000000000000000000000000000000000006E
:0802900000000000FE00DAF797
:100298000100020818000000C9010208030000005C
:1002A8000508020806000000150D020809000000F4
:1002B8009912020802000000A913020810000000A9
:1002C80065150208FF000000ED1C02080C00000084
:1002D800D9220208000000001525020805000000C8
:1002E800454B0208120000006D4E02080A0000008B
:1002F800B55202080A000000695B020814000000F9
:10030800F55F0208080000000D67020807000000FA
:10031800B56D0208100000009D710208130000006E
:100328003D83020813000000A9AF02081600000070
:100338006D080308170000003D460308160000007A
:100348006547030817000000395A03081500000024
:100358002F49072291438D462E492F480A1A06D065
:100368000722914381F30988022282F314882B48DB
:100378002B492C4A00F039F82B482C492C4A00F01C
:1003880034F82C482C492D4A00F02FF82C482D49D8
:100398002D4A00F02AF82D482D492E4A00F025F85C
:1003A8002D482E492E4A00F020F82E482E490022CA
:1003B80000F026F82D482E49091A082903DB0022E7
:1003C8000260043001601F481F49884205D0026856
:1003D800043003B4904703BCF7E700208646EC4698
:1003E80000200021234A9047FEE7884207D0521A8E
:1003F80005D0037801300B700131013AF9D170470B
:10040800884202D002700130FAE770471A487047F4
:100418004C2801204C3001204C28012030BD030815
:1004280088010020040200200000020800000208E1
:10043800088E030830BD03088801002088010020C9
:100448009405000894050008940500089405000820
:100458009405000894050008088E0308088E030810
:1004680030BD030804020020002501204C2501208E
:100478004C2501204D330208FFFFFFFFFEE7FEE792
:10048800FEE7FEE7FEE7FEE7FEE7FEE7FEE7FEE73C
:10049800FEE7FEE7FEE7FEE7FEE7FEE7FEE7FEE72C
:1004A800FEE7FEE7FEE7FEE7FEE7FEE7FEE7FEE71C
:1004B800FEE7FEE7FEE7FEE7FEE7FEE7FEE7FEE70C
:1004C800FEE7FEE7FEE7FEE7FEE7FEE7FEE7FEE7FC
:1004D800FEE7FEE7FEE7FEE7FEE7FEE7FEE7FEE7EC
:1004E800FEE7FEE7FEE7FEE7FEE7FEE7FEE7FEE7DC
:1004F800FEE7FEE7FEE7FEE7FEE7FEE7FEE7FEE7CC
:10050800FEE7FEE7FEE7FEE7FEE7FEE7FEE7FEE7BB
:10051800FEE7FEE7FEE7FEE7FEE7FEE7FEE7FEE7AB
:10052800FEE7FEE7FEE7FEE7FEE7FEE7FEE7FEE79B
:10053800FEE71348854600F022F84EF68850CEF2C2
:100548000000016851F47001016000BF00BF00BFE6
:10055800F1EE100A50F04070E1EE100A4FF0000082
:1005680080F314884EF63C71CEF20001086850F012
:1005780040700860034804490160FFF7E9BE70470E
:0C0588000000022008ED00E00000000868
:020000040801F1
:1000000000000000000000000000000000000000F0
:1000100000000000000000000000000000000000E0
:100020000000000000000000000000000000013B94
:100030000F018600003D8601003D680220830044D8
:10004000F430F4301E00000A830123014413F5311B
:1000500083012FF5330000F4030066000000F40371
:100060000100000000094A004AFF51008F35008F4F
:10007000360098000000009637430942088F21009F
:100080008F34FF680020F406F4022034009BF4074C
:100090000000640088830129800086420942084AE2
:1000A000FF7100442370004422AE009624AE0196F6
:1000B00028AE02962CAE03963045210C018200C179
:1000C0000C4421F535F406F402453460002000DBD1
:1000D000F5358100DB0C018200DB0C45211281002B
:1000E000EBF40700006400C7800066690020453516
:1000F00045365551009437AF0045365F0080009F6C
:100100001E00006483012301451312810100441382
:100110001E0000648301230145131282010EF53194
:1001200080010070084A0F52096E012080012F6083
:1001300001200138F5390009F53901092113340787
:10014000FFFFFFFFFFFFFFFFFFFFFFFFFFFFFFFFBF
:10015000FFFFFFFFFFFFFFFFFFFFFFFFFFFFFFFFAF
:10016000FFFFFFFFFFFFFFFFFFFFFFFFFFFFFFFF9F
:10017000FFFFFFFFFFFFFFFFFFFFFFFFFFFFFFFF8F
:020000040802F0
:1000000030B583B04FF0010004F016FF4FF000044C
:1000100000944FF0F805019520464FF003014FF092
:1000200002024FF0010302F0F1FC40F20420C2F2A0
:10003000010040F20421C2F200014FF480324FF07F
:10004000020315F059FE4FF00100294614F0B4FDEB
:100050004FF00300214640F2CD02C0F6020203F049
:10006000D3FC4FF0010040F2DD01C0F6020140F286
:10007000BD02C0F6020203F0C7FC4FF008004FF0CB
:100080000901024610F01CFB4FF009030093019494
:100090004FF004004EF68531C3F6D16141F6B862E7
:1000A000C3F685624FF0020313F01EFC48F6286089
:1000B000C0F6030007F0FEFA03B030BD08B519B969
:1000C0004FF0030015F082FC08BD00BF08B5012900
:1000D00003D14FF0010015F079FC08BD08B54FF0D1
:1000E0000A0000F0C9FE08BD48F64863C0F60303E5
:1000F0001A684EF60C50CEF200000260FEE700BF18
:1001000008B5FFF7F1FF00BF51E8002FBFF35F8F85
:1001100041E80003012B3FF4F7AF1046704700BFE2
:1001200013461A462DE9F00F0B460C460D460E46B7
:100130000F46884689468A468B46092AC0F00780C2
:10014000A0E8F80FA2F10902092ABFF4F9AF4FF0B5
:10015000080303FB02F2144B1A44974600F020B840
:1001600000BF00BF046000F01BB800BF80E8300093
:1001700000F016B880E8700000F012B880E8F000D7
:1001800000F00EB880E8F00100F00AB880E8F00353
:1001900000F006B880E8F00700F002B880E8F00F41
:1001A000BDE8F00F704713465C010208EFF31180C1
:1001B0004FF0800181F3118870474FF0000000BFBD
:1001C00080F31188704700BF30B440F20003C0F6DE
:1001D000000340F28812C0F60002D01A4FEAA001D4
:1001E000B1F5C47F04D81346264A9A4201D324E0CD
:1001F000FEE7254D254C601B20F003054FF0000362
:1002000040F20002C2F2000240F20001C0F600011A
:1002100005F10400C5F380045D589D5003F104030B
:10022000834226D109E05C589C5003F104035C58DA
:10023000D45003F104038342F5D14EF60853CEF2B5
:10024000000340F20002C2F200021A604FF0B50152
:10025000CBF26B1142F24C50C2F2010001604EF63B
:100260001453CEF200031A6842F01001196030BC3A
:100270007047002CD7D05C589C5003F10403834294
:10028000D1D1DAE700000008040000088B01000863
:1002900010B4034600283ED002F1100440F20000E2
:1002A000C2F2000040F82430002A0ADA12F10C0FE2
:1002B00035DB02F10C024EF61850CEF2000011545C
:1002C0002DE04EF20014CEF200040F299CBF09016C
:1002D000C9B24EF20043CEF20003D1541146002AB7
:1002E000B8BF02F11F014FEA611004EB80014FF02B
:1002F0001F03C8F200031340002B05DA03F1FF329D
:1003000062F01F0303F1010358B24FF0010202FA39
:1003100000F30B6003E0002AC8DB024CD5E710BCF9
:10032000704700BF80E100E01EF0040F0CBFEFF348
:100330000880EFF3098020E9F00F00F001B800BF5A
:1003400010B5026842F20053C2F201031A6041681C
:10035000596082689A60C168D96002691A6141690E
:10036000596182699A61C169D961026A1A62416AF6
:100370005962826A9A62C16AD962026B1A63416BDE
:100380005963826B9A63C16BD96300F140001864B2
:100390004EF62850CEF2000002685A6418F0F4FCC1
:1003A000002800F0FB8148F64C60C0F6030018F00E
:1003B000F1FC4EF62C54CEF200042368002B05DA33
:1003C00048F65C60C0F6030018F0E4FC4EF62C51D1
:1003D000CEF20001086810F0020F05D048F66C60FC
:1003E000C0F6030018F0D6FC4EF62852CEF20002FA
:1003F0005478002C72D048F68460C0F6030018F0E0
:10040000C9FC4EF62853CEF20003597811F0010FC3
:1004100005D048F69460C0F6030018F0BBFC4EF619
:100420002850CEF20000427802F00204E3B22BB171
:1004300048F6B460C0F6030018F0ACFC4EF6285144
:10044000CEF20001487800F00402D4B22CB148F694
:10045000D860C0F6030018F09DFC4EF62853CEF28B
:100460000003597801F00800C2B22AB148F6FC60D6
:10047000C0F6030018F08EFC4EF62854CEF20004AD
:10048000637803F01001C8B228B148F61C70C0F6BA
:10049000030018F07FFC4EF62852CEF2000254788A
:1004A00004F02003D9B229B148F63C70C0F603002D
:1004B00018F070FC4EF62850CEF20000427802F0A0
:1004C0008004E3B253B14EF63851CEF20001096810
:1004D00048F65C70C0F6030018F05CFC4EF628503D
:1004E000CEF20000428894B2002C5ED048F67C70B8
:1004F000C0F6030018F04EFC4EF62853CEF200036F
:10050000598811F0010F05D048F68C70C0F6030031
:1005100018F040FC4EF62850CEF20000428802F05F
:100520000204A3B22BB148F6B870C0F6030018F06D
:1005300031FC4EF62851CEF20001488800F004024A
:1005400094B22CB148F6DC70C0F6030018F022FC1F
:100550004EF62853CEF20003598801F0080082B20B
:100560002AB149F21C00C0F6030018F013FC4EF645
:100570002854CEF20004638803F4807188B228B155
:1005800049F24C00C0F6030018F004FC4EF6285265
:10059000CEF20002548804F4007399B229B149F2F2
:1005A0006800C0F6030018F0F5FB4EF62850CEF2B6
:1005B00000000278002A63D049F28000C0F60300F0
:1005C00018F0E8FB4EF62854CEF20004237813F01E
:1005D000010F05D049F29000C0F6030018F0DAFBD5
:1005E0004EF62851CEF20001087800F00202D4B293
:1005F0002CB149F2B000C0F6030018F0CBFB4EF668
:100600002853CEF20003197801F00800C2B22AB1D3
:1006100049F2C800C0F6030018F0BCFB4EF628549F
:10062000CEF20004237803F01001C8B228B149F2D9
:10063000EC00C0F6030018F0ADFB4EF62852CEF2E7
:100640000002147804F02003D9B229B149F2101045
:10065000C0F6030018F09EFB4EF62850CEF20000C4
:10066000027802F08004E3B253B14EF63451CEF278
:100670000001096849F23010C0F6030018F08AFB47
:1006800042F20054C2F20104216A49F25C10C0F641
:10069000030018F07FFB616A49F27010C0F6030096
:1006A00018F078FBA16A49F28410C0F6030018F034
:1006B00071FBE16A49F29810C0F6030018F06AFB7A
:1006C000216849F2AC10C0F6030018F063FB6168C2
:1006D00049F2C010C0F6030018F05CFBA16849F2B3
:1006E000D410C0F6030018F055FBE16849F2E81099
:1006F000C0F6030018F04EFB216949F2FC10C0F669
:10070000030018F047FB616949F21020C0F60300AE
:1007100018F040FBA16949F22420C0F6030018F04C
:1007200039FBE16949F23820C0F6030018F032FBCA
:10073000216B49F24C20C0F6030018F02BFB216C12
:1007400049F26020C0F6030018F024FB616B49F207
:100750007420C0F6030018F01DFBA16B49F298202D
:10076000C0F6030018F016FB42F24850C2F2010036
:10077000026849F2BC20C0F603001146126818F066
:1007800009FB41F69803C2F201031A6849F2D4202A
:10079000C0F603001146126818F0FCFAFFF7B0FC2F
:1007A00010BD00BF00B506F0CBF9002808BF5DF80A
:1007B00004FBEFF30981EFF3118221E9F40F5DF8F7
:1007C00004EB1EF0100F08BF21ED108A41F804ED74
:1007D0000B4C2268002A18BF516006F023FA2268E9
:1007E000516851F804EB1EF0100F08BFB1EC108AED
:1007F000B1E8F40F82F3118881F309887047000093
:100800004825012008B540F2A570C0F602004FF05F
:10081000FF016FF00102FFF73BFD08BDF8B5074689
:100820000C461E460799089D14F0030F00D0FEE702
:1008300022B1A4EB8500A0F1480401E004F14800D6
:10084000012D01D8A16205E02A4601F071FEA7EB57
:100850008507A7624FF0000363604FF01130E0623C
:100860004FF0223121634FF0333262634FF0443353
:10087000A3604FF05530E0604FF0663121614FF0DA
:10088000773262614FF08833A3614FF09930E061B5
:100890004FF0AA3121624FF0BB3262624FF0CC338D
:1008A000A363E663069820644FF0807161646FF083
:1008B0000202226005F11200F8BD00BF62B64EF6DA
:1008C0000453CEF200031A6842F08050186000BF53
:1008D00043F64003C4F202031A6861F35D721A60C2
:1008E000704700BF4FEA001049F2EC23C0F6030343
:1008F0001A5849F62C41C0F6030151F822007047FE
:100900002DE9F04F8BB083468A46914698469DF973
:1009100050709DF954609DF958509DF95C100091FC
:100920009DF960200192FFF7DDFF036849F2EC2199
:10093000C0F6030101EB0B1BDBF80420012A02D0F7
:10094000022A34D119E01C46C3F340310991C3F3A4
:1009500000310891C3F303210791C3F3811106917C
:10096000C3F3C2010591C3F380010491C3F34001B5
:10097000039103F00101029119E043F30F44C3F323
:1009800040710991C3F300710891C3F303610791AA
:10099000C3F381510691C3F3C2410591C3F3804172
:1009A0000491C3F340410391C3F300410291BAF1B2
:1009B000000FA4BF0AF0010ACDF808A0B9F1000F9A
:1009C000A4BF09F00109CDF80C90B8F1000FA4BF45
:1009D00008F00108CDF81080002FA4BF07F007072A
:1009E0000597002EA4BF06F003060696002DA4BFAF
:1009F00005F00F05079500990029A4BF01F001013A
:100A0000089101990029A4BF01F001010991012A6F
:100A100002D0022A35D11AE0029A62F30004039947
:100A200061F34104049A62F38204059961F3C504F9
:100A3000069A62F38714079961F30B24089A62F30C
:100A40000C34099961F34D3464F30F0319E0029AF1
:100A500062F30004039961F34104049A62F382048F
:100A6000059961F3C504069A62F38714079961F347
:100A70000B24089A62F30C34099961F34D3464F342
:100A80001F4303600BB0BDE8F08F00BF38B50446CC
:100A90000D46FFF727FF49F2EC23C0F6030303EBF3
:100AA00004146168012902D0022903D101E08560A4
:100AB00038BD456138BD00BF10B540F20403C4F233
:100AC00002031C6849F2CC31C0F603010A6824EA2B
:100AD000020449F2D842C0F60302106804431C60C5
:100AE00040F20443C4F202031868186040F604049C
:100AF000C4F202042368236040F60444C4F20204F2
:100B00002068206041F20403C4F202031C680969F2
:100B100024EA0104126944EA0200186041F2044325
:100B2000C4F202031C681C6041F60401C4F2020115
:100B30000A680A6041F60440C4F2020003680360D8
:100B400042F20404C4F202042168216040F20C0164
:100B5000C4F202010C6849F27C32C0F6030210684C
:100B600024EA000449F28443C0F6030318680443EE
:100B70000C6040F20C41C4F202010C68506824EA97
:100B80000004586804430C6040F60C01C4F20201F2
:100B90000C68906824EA0004986804430C6040F6EE
:100BA0000C41C4F202010C68D06824EA0004D86841
:100BB00004430C6041F20C01C4F20201086812699E
:100BC00020EA02001B6940EA03040C6041F20C4178
:100BD000C4F202010868086041F60C03C4F2020383
:100BE0001A681A6041F60C44C4F2020421682160BC
:100BF00042F20C00C4F202000368036049F21032B2
:100C0000C0F60302146840F21401C4F202010C6041
:100C10004FF0000040F21443C4F20203186040F6A3
:100C20001404C4F20204206040F61441C4F202012C
:100C30000860136941F21402C4F20202136041F227
:100C40001444C4F20204206041F61401C4F202010B
:100C5000086041F61443C4F20203186042F2140221
:100C6000C4F20202106040F20001C4F202010C68FA
:100C700049F2A032C0F60302106824EA000449F2E7
:100C80003433C0F60303186804430C6040F200419B
:100C9000C4F202010C68506824EA00045868044356
:100CA0000C6040F60001C4F202010868086040F6DA
:100CB0000041C4F202010C68D06824EA0004D8683C
:100CC0002043086041F20001C4F202010868126981
:100CD00020EA02001B691843086041F20041C4F297
:100CE00002010A680A6041F60003C4F202031868B0
:100CF000186041F60041C4F202010A680A6042F23B
:100D00000003C4F20203186818604FF0010003F0FA
:100D1000E1FF10BD08B543F63002C4F202021368C9
:100D20006FEA53206FEA4021116043F62003C4F2BA
:100D300001031A6842F001001860FFF7BDFE08BD0C
:100D40002DE9F0019DF814709DF81860079D49F297
:100D50005834C0F6030454F820004FEA4104FF2F32
:100D600012D0D0F80C8049F2504CC0F6030C1CF89D
:100D7000077007FA04FC4FF0030707FA04F728EAA4
:100D800007074CEA0707C760FF2B10D0D0F804C054
:100D900049F20C37C0F60307FF5C07FA01F74FF082
:100DA000010303FA01F32CEA03033B434360FF2EE4
:100DB0000FD0876849F2C433C0F603039E5D06FA7C
:100DC00004F64FF0030303FA04F327EA0303334363
:100DD0008360B5F1FF3F16D04FEAD10303F108035A
:100DE00050F8236001F007014FEA810105F00F057B
:100DF00005FA01F54FF00F0707FA01F126EA0101A4
:100E0000294340F82310FF2A10D0016849F2C83363
:100E1000C0F603039B5C03FA04F34FF0030202FAEB
:100E200004F421EA040143EA01040460BDE8F0018E
:100E3000704700BF49F22043C0F6030353F8201067
:100E40000A6849F2F033C0F6030353F820100A4051
:100E500049F2FC43C0F6030353F82000824214BF5A
:100E600000200120704700BF49F25833C0F6030349
:100E700053F820000069704749F2F033C0F60303CD
:100E800053F820307BB139B149F2A841C0F60301D3
:100E900051F820201360704749F25442C0F6030213
:100EA00052F820000360704700EB800049F2305395
:100EB000C0F6030353F8202002F1FF300D2800F2A2
:100EC0008680DFE800F0071019222B343D464F588A
:100ED000616A737C43F64400C4F20200036861F364
:100EE00000030360704743F64003C4F202031A682C
:100EF00061F300021A60704743F64003C4F2020334
:100F0000186861F341001860704743F64000C4F26E
:100F10000200026861F382020260704743F64000FB
:100F2000C4F20200036861F3C3030360704743F631
:100F30004003C4F202031A6861F304121A60704796
:100F400043F64003C4F20203186861F345101860C9
:100F5000704743F64400C4F20200026861F34102A4
:100F60000260704743F64400C4F20200036861F374
:100F700010430360704743F64403C4F202031A6847
:100F800061F351421A60704743F64403C4F202030E
:100F9000186861F392401860704743F64000C4F24D
:100FA0000200026861F386120260704743F6400057
:100FB000C4F20200036861F3C7130360704743F68D
:100FC0004003C4F202031A6861F308221A607047F2
:100FD00000EB800049F23053C0F6030353F82020A1
:100FE00049F67041C0F6030151F82200704700BF76
:100FF0002DE9F84F04468A46914698469DF9287097
:101000009DF92C609DF93050FFF7E2FF04EB84025C
:1010100049F23053C0F6030303EB82035A68022AF5
:1010200094BF8369C369016A02F1FF3CBCF1030FFD
:101030002ED8DFE80CF0021802186FF30103BAF1A2
:10104000000FC8BF6AF38203B9F1000FC8BF69F38C
:10105000C303B8F1000FC8BF68F30613002F17DDF4
:1010600067F3C71314E06FF30923BAF1000FC8BF89
:101070006AF38A23B9F1000FC8BF69F3CB23B8F133
:10108000000FC8BF68F30E33002FC8BF67F3CF331C
:1010900002F1FF37032F44D8DFE807F002142638A7
:1010A000312C04D1002E06DD66F3820103E0002E10
:1010B000C8BF66F30001002DC8BF65F341016FF39F
:1010C000C30130E0332C04D1002E06DD66F3861117
:1010D00003E0002EC8BF66F30411002DC8BF65F3FE
:1010E00045116FF3C7111EE0352C04D1002E06DD2B
:1010F00066F38A2103E0002EC8BF66F30821002DA5
:10110000C8BF65F349216FF3CB210EE0002EC8BFA5
:1011100066F30C31002DC8BF65F34D316FF3CF314D
:1011200003E0022A01D8836100E0C361016204EB9D
:10113000840449F23050C0F6030050F82430012BEB
:1011400002D0082B16D10BE049F22C53C0F6030352
:101150001A6840F24401C4F201010A60BDE8F88F48
:1011600049F22C52C0F60302116840F24440C4F226
:1011700001000160BDE8F88F38B504460D46FFF761
:1011800027FF04EB840149F23053C0F6030303EB5D
:101190008104626802F1FF3103290AD8DFE801F017
:1011A00002040608456338BD856338BDC56338BD94
:1011B000056438BD40F21C23C2F201031B689BB1D9
:1011C000A8B91A686FF300021A604FF00000586265
:1011D00040F22021C2F2010108801A6842F00100A9
:1011E00018604FF0010070474FF0000070474FF05B
:1011F0000000704710B483B040F21C23C2F2010318
:101200001B6803B310BB40F22022C2F20102586AED
:10121000148840EA0440019000BF00BF00BF00BF37
:1012200000BF586A148840EA04400090019C00986E
:101230008442ECD1DDED017AB8EEE70A81ED000AD7
:101240004FF0010004E04FF0000001E04FF000001B
:1012500003B010BC704700BF40F21C23C2F2010370
:101260001B689BB1A8B91A686FF300021A60596233
:101270004FEA114140F22020C2F2010001801A68B9
:1012800042F0010119604FF0010070474FF000007B
:1012900070474FF00000704743F67403C4F2020336
:1012A000186847F20402C4F20002136840F22222D6
:1012B000C2F201024FF00001117013F0010F04D0CF
:1012C00010464FF0040202703EE04FEA106212F046
:1012D000600F07D040F22221C2F201014FF020033B
:1012E0000B7031E002F00401C9B239B140F22220A2
:1012F000C2F201004FF04002027025E0C3F3400348
:1013000043EAD06010F0010F07D040F22221C2F270
:1013100001014FF080030B7016E002F01001CBB218
:101320003BB140F22220C2F201004FF001020270F4
:101330000AE002F00202D0B230B140F22221C2F241
:1013400001014FF002030B7043F67401C4F2020175
:101350000B6843F08070086047F20001C4F200019E
:101360000A6842F008030B6042F24850C2F20100E2
:10137000016840F22422C2F201021160704700BFEE
:1013800040F22223C2F201031878704708B547F6ED
:101390001021C1F6FF714FF00C0215F015FF4FF050
:1013A0000C0008BD0000000010B542F20803CEF2A8
:1013B00004031A6842F01000186041F26140C0F660
:1013C00002004FF00F014FF03602FEF761FF43F6C7
:1013D0004001C4F202010C6844F010030B6041F2BA
:1013E0000004C4F2000449F69412C0F60302106827
:1013F000206049F63441C0F60301886914F0A2FC6C
:1014000015A3D3E9002314F0E1FE4FF000024FF0E2
:101410000003C3F6F07314F093FD14F0FFFC41F2E7
:101420002C03C4F20003188041F22800C4F200002B
:101430004FF00002028049F69011C0F603010868DF
:1014400041F20C03C4F200031860228842F001014B
:10145000218010BDAFF300802D431CEBE2362A3F04
:10146000684620F007018D4601B541F21003C4F231
:1014700000034FF000021A6005F072FEBDE8014063
:101480008546704770B50446B0F5CC7F2FD940F241
:101490003233984216D940F26560844215D940F63D
:1014A000CB418C4214D941F69712944213D943F29E
:1014B0002F36B44212D946F25F639C4298BF06258C
:1014C0000ED90FE04FF001050AE04FF0020507E0EA
:1014D0004FF0030504E04FF0040501E04FF005056F
:1014E000072D06D1FEF70CFE4FF0070501E04FF087
:1014F0000005FEF75BFE064604EB84044FEAC400D9
:1015000049F69811C0F6030151F83520B0FBF2F30B
:101510009CB2012C05D9B4F5805F04D3FEF7F0FD31
:1015200001E04FF0020443F20000C4F2000045F273
:101530005551016049F69812C0F6030202EBC50549
:101540002B7943F20401C4F200010B6043F208025C
:10155000C4F2000214604AF6AA2303603046FEF784
:101560002FFE70BD08B543F20003C4F200034CF631
:10157000CC421A604FF0C800FFF784FF08BD00BFDF
:1015800043F20003C4F200034AF6AA221A6070472D
:1015900010B5044643F21003C4F20003186810F0BB
:1015A000010F74D04FF0320007F084F843F21001BD
:1015B000C4F200010A6812F0010F68D04FF0320047
:1015C00007F078F843F21003C4F20003186810F033
:1015D000010F5CD04FF0320007F06CF843F21001BD
:1015E000C4F200010A6812F0010F50D04FF032002F
:1015F00007F060F843F21003C4F20003186810F01B
:10160000010F44D04FF0320007F054F843F21001BC
:10161000C4F200010A6812F0010F38D04FF0320016
:1016200007F048F843F21003C4F20003186810F002
:10163000010F2CD04FF0320007F03CF843F21001BC
:10164000C4F200010A6812F0010F20D04FF03200FE
:1016500007F030F843F21003C4F20003186810F0EA
:10166000010F14D04FF0320007F024F843F21001BC
:10167000C4F200010A6812F0010F08D04FF03200E6
:1016800007F018F843F21003C4F200031B68204669
:10169000FFF7F8FE10BD00BF02469CF8043043B1CE
:1016A000DCF8000040B141F2A421C2F2010141F88E
:1016B0002200DCF8000050B941F2A423C2F2010379
:1016C00053F8220049F64042002808BF10467047F0
:1016D0004FF0010303FA00F010F0180F0CBF0020C8
:1016E0000120704770B50D4649F60023C0F603038C
:1016F00053F82040002C45D000EB800040F2282613
:10170000C2F2010606EBC00630464FF0000104F0BD
:10171000ADFC122D07D142F20431C4F201010A6876
:1017200042F480030B60606B65F304006063E36C5C
:101730004FF0050006F0BEFFA16841F08042A260B4
:10174000236813F0020FFBD0E46C122D16D142F285
:101750000430C4F2010001686FF39651016042F257
:101760000002CEF2040213684FEA03504FEA105110
:1017700040F2194291420CBFA4006400304604F0CC
:1017800083FD01E04FF0FF34204670BD38B52DEDEC
:10179000028B044608EE101A49F6D815C0F6030568
:1017A00005EB8005F7EE007AB4EEE78AF1EE10FA69
:1017B00009DC084614F01CFF00289FED260A18BF1C
:1017C000B0EE408A01E0B7EE008A2B78012B1CD1E5
:1017D0006878FFF7FDFBD0ED0B1A6D78B8EE612A43
:1017E00062EE082A12EE900A14F052FB4FF000024B
:1017F0004FF00003C3F6E07314F0A4FB14F00EFBEB
:1018000001462846FFF7B8FC18E0022B16D16D7888
:10181000DFED110A28EE201A11EE100A14F038FB41
:101820004FF000024FF00003C3F6E07314F08AFBA0
:1018300014F0F4FA01462846FFF728F940F2A020F8
:10184000C2F2010000EB840484ED008ABDEC028B3F
:1018500038BD00BF0000000000F07F4510B54FF01C
:1018600000044FF000002146FFF790FF4FF0010009
:101870002146FFF78BFF4FF002002146FFF786FF5E
:101880004FF003002146FFF781FF4FF0040021468F
:10189000FFF77CFF4FF005002146FFF777FF4FF081
:1018A00006002146FFF772FF4FF007002146FFF7C1
:1018B0006DFF4FF008002146FFF768FF4FF0090069
:1018C0002146FFF763FF40F20C01C4F202010C68ED
:1018D00049F69422C0F60302136824EA030449F689
:1018E0004023C0F60303186804430C6040F20C4127
:1018F000C4F202010C68506824EA000458680443EA
:101900000C6040F60C01C4F202010868926820EAFB
:1019100002009B6840EA03040C6040F60C41C4F2EC
:1019200002010868086041F20C03C4F202031A685D
:101930001A6041F20C44C4F202042168216041F6AD
:101940000C00C4F202000368036041F60C44C4F2C8
:1019500002042268226042F20C01C4F2020108680B
:10196000086040F20001C4F202010C6849F614223A
:10197000C0F60302136824EA030449F66C23C0F698
:101980000303186804430C6040F20041C4F20201F2
:101990000C68506824EA000458682043086040F648
:1019A0000001C4F202010868926820EA02009B6804
:1019B0001843086040F60041C4F202010A680A6058
:1019C00041F20003C4F202031868186041F20041BA
:1019D000C4F202010A680A6041F60003C4F202037D
:1019E0001868186041F60041C4F202010A680A60F2
:1019F00042F20003C4F202031868186010BD00BF71
:101A000008B505280ED849F60C23C0F60303195C67
:101A1000FF290AD049F6BC22C0F60302105CFFF78A
:101A200061FE08BD4FF0FF3008BD4FF0FF3008BD2C
:101A300010B50446FFF7E4FF07EE900AB8EE677AA8
:101A400049F60C23C0F60303185D11280BD147F6A5
:101A50002A21C1F6FF710A8801EE102AF8EEC11A98
:101A6000C1EE870A03E09FED030AC7EE000A10EEFD
:101A7000900A10BD00F07F4540F2A023C2F201039E
:101A800003EB80000068704738B50D46044600B38C
:101A90000E2801D9FEF734FB49F63443C0F60303A0
:101AA00053F8240055B1B0FBF5F14FEA114202F1B1
:101AB0000103B0FBF3F0B0FBF5F502E04FF00005D9
:101AC0002A4649F67041C0F6030151F824309A6263
:101AD000DD6238BD10B582B000918DF804200A286F
:101AE00040F0E2804FF00000FFF7F2FD48B1EC4615
:101AF0004FF00000FFF7D0FD01464FF00000FFF768
:101B0000C3FF4FF00100FFF7E3FD48B1EC464FF093
:101B10000100FFF7C1FD01464FF00100FFF7B4FFE0
:101B20004FF00200FFF7D4FD48B1EC464FF0020041
:101B3000FFF7B2FD01464FF00200FFF7A5FF4FF09F
:101B40000300FFF7C5FD48B1EC464FF00300FFF777
:101B5000A3FD01464FF00300FFF796FF4FF004008E
:101B6000FFF7B6FD48B1EC464FF00400FFF794FDD7
:101B700001464FF00400FFF787FF4FF00500FFF725
:101B8000A7FD48B1EC464FF00500FFF785FD014683
:101B90004FF00500FFF778FF4FF00600FFF798FDC4
:101BA00048B1EC464FF00600FFF776FD01464FF0D6
:101BB0000600FFF769FF4FF00700FFF789FD48B106
:101BC000EC464FF00700FFF767FD01464FF00700B6
:101BD000FFF75AFF4FF00800FFF77AFD48B1EC46D7
:101BE0004FF00800FFF758FD01464FF00800FFF7DF
:101BF0004BFF4FF00900FFF76BFD48B1EC464FF08B
:101C00000900FFF749FD01464FF00900FFF73CFFCF
:101C10004FF00A00FFF75CFD48B1EC464FF00A00B8
:101C2000FFF73AFD01464FF00A00FFF72DFF4FF096
:101C30000B00FFF74DFD48B1EC464FF00B00FFF7EE
:101C40002BFD01464FF00B00FFF71EFF4FF00C007D
:101C5000FFF73EFD48B1EC464FF00C00FFF71CFDCE
:101C600001464FF00C00FFF70FFF4FF00D00FFF79C
:101C70002FFD48B1EC464FF00D00FFF70DFD01467A
:101C80004FF00D00FFF700FF4FF00E00FFF720FDB3
:101C900048B3EC464FF00E00FFF7FEFC01464FF054
:101CA0000E00FFF7F1FE1EE049F6D813C0F603035D
:101CB00013F82010012916D149F6D812C0F60302F4
:101CC00002EB8000447804EB840349F23051C0F603
:101CD000030151F82340EC462046FFF7DDFC0146A6
:101CE0002046FFF7D1FE02B010BD00BF70B586B030
:101CF00040F22825C2F2010549F63C24C0F603044F
:101D00002846214604F09AF905F12800214604F0FE
:101D100095F905F15000214604F090F943F644038B
:101D2000C4F202031A6842F480701860196841F422
:101D300000761E6049F66825C0F603052C6842F25D
:101D40000433C4F201031C6049F66422C0F60302A6
:101D5000106842F20401C4F20101086042F2041664
:101D6000C4F20106306049F6B825C0F603052C68B8
:101D700042F20C03C4F201031C6042F20C12C4F2E2
:101D80000102146049F63820C0F60300016842F2EF
:101D90001006C4F20106316042F21015C4F20105CA
:101DA000296049F6D014C0F60304236842F22C02DD
:101DB000C4F20102136042F22C10C4F2010003606D
:101DC00049F6D411C0F603010E6842F20805C4F2C8
:101DD00001052E6042F20814C4F2010426604FF09F
:101DE00023004FF00101FFF75FF84FF022004FF0A2
:101DF0000101FFF759F84FF021004FF00101FFF703
:101E000053F84FF020004FF00101FFF74DF84FF06D
:101E100019004FF00101FFF747F84FF018004FF09D
:101E20000101FFF741F84FF017004FF00101FFF7F4
:101E30003BF84FF016004FF00101FFF735F84FF077
:101E4000000400944FF00106019602944FF0230025
:101E5000214632464FF00603FFF7CAF849F23055E3
:101E6000C0F6030595F8C802D5F8CC120094019489
:101E7000D5F8C43202934FF003022346FEF760FF09
:101E80000094019602944FF02200214632464FF012
:101E90000603FFF7ADF895F8B402D5F8B812009430
:101EA0000194D5F8B02202924FF003022346FEF7C8
:101EB00047FF0094019602944FF0210021463246DC
:101EC0004FF00603FFF794F895F8A002D5F8A41296
:101ED00000940194D5F89C3202934FF003022346FC
:101EE000FEF72EFF0094019602944FF02000214649
:101EF00032464FF00603FFF77BF895F88C02D5F8D1
:101F0000901200940194D5F8882202924FF00302B7
:101F10002346FEF715FF0094019602944FF0190036
:101F2000214632464FF00603FFF762F895F80002AB
:101F3000D5F8041200940194D5F8FC3102934FF0C7
:101F400003022346FEF7FCFE0094019602944FF034
:101F50001800214632464FF00603FFF749F895F87E
:101F6000EC01D5F8F01100940194D5F8E821029223
:101F70004FF003022346FEF7E3FE0094019602941D
:101F80004FF01700214632464FF00603FFF730F8B6
:101F900095F8D801D5F8DC1100940194D5F8D43126
:101FA00002934FF003022346FEF7CAFE0094019607
:101FB00002944FF01600214632464FF00603FFF719
:101FC00017F895F8C401D5F8C81100940194D5F814
:101FD000C05102954FF003022346FEF7B1FE4FF0C9
:101FE0000A0021462246FFF775FD4FF00005204606
:101FF0002946FFF7CBFB30462946FFF7C7FB4FF0DA
:1020000002002946FFF7C2FB4FF003002946FFF705
:10201000BDFB4FF004002946FFF7B8FB4FF0050069
:102020002946FFF7B3FB4FF006002946FFF7AEFB4A
:102030004FF007002946FFF7A9FB4FF0080029469B
:10204000FFF7A4FB4FF009002946FFF79FFB30463E
:10205000FFF73EFB50B149F67040C0F603004168FF
:1020600049F69024C0F6030422680A604FF002008B
:10207000FFF72EFB50B149F67043C0F603039D688D
:1020800049F69020C0F60300016829604FF0030074
:10209000FFF71EFB50B149F67044C0F60304E36835
:1020A00049F69022C0F6030215681D604FF0040047
:1020B000FFF70EFB50B149F67040C0F6030001690E
:1020C00049F69024C0F6030423680B604FF0050026
:1020D000FFF7FEFA50B149F67042C0F603025569A7
:1020E00049F69020C0F60300016829604FF0060011
:1020F000FFF7EEFA50B149F67044C0F60304A36945
:1021000049F69022C0F6030215681D604FF00700E3
:10211000FFF7DEFA50B149F67040C0F60300C1691E
:1021200049F69024C0F6030423680B604FF00800C2
:10213000FFF7CEFA50B149F67042C0F60302156AB5
:1021400049F69020C0F60300016829604FF00900AD
:10215000FFF7BEFA50B149F67044C0F60304636A53
:1021600049F69022C0F6030215681D604FF00A0080
:10217000FFF7AEFA50B149F67040C0F60300816A2D
:1021800049F69024C0F6030423680B604FF00B005F
:10219000FFF79EFA50B149F67042C0F60302D56AC5
:1021A00049F69020C0F60300016829604FF00C004A
:1021B000FFF78EFA50B149F67044C0F60304236B62
:1021C00049F69022C0F6030215681D604FF00D001D
:1021D000FFF77EFA50B149F67040C0F60300416B3C
:1021E00049F69024C0F6030423680B604FF00E00FC
:1021F000FFF76EFA50B149F67042C0F60302956BD4
:1022000049F69020C0F60300016829604FF00100F4
:102210000146FEF75DFB4FF001004FF00001FEF7B5
:1022200035FC4FF00004009401940294039404944C
:102230004FF00100014602462346FEF761FB49F2DA
:10224000EC25C0F60305287EE96900940194029408
:102250004FF002022346FEF773FD20464FF00101C6
:10226000FEF736FB20462146FEF710FC0094019451
:1022700002940394049420464FF001012246234621
:10228000FEF73EFB287AE9680094019402944FF02F
:1022900002022346FEF754FDFFF7E0FA06B070BDD8
:1022A00010B504464FF000004FF01101FFF71AFA85
:1022B00047F62A23C1F6FF73198807EE901AB8EE85
:1022C000670A06EE900AB8EE667AC0EE070AC4ED19
:1022D000000A4FF0010010BD30B472B649F6D823A1
:1022E000C0F603031A684EF63470CEF200000260A6
:1022F00049F6C421C0F603010A684EF68853CEF2AF
:1023000000031A6049F6E020C0F60300016842F2BB
:102310000802CEF20402116049F6C823C0F6030396
:10232000186842F20C01CEF20401086043F6000383
:10233000C4F202031A6842F48030186019460B6830
:1023400013F4003FFBD043F64000C4F202000268E1
:1023500042F08051016047F20003C4F200031868A4
:102360006FF38E30186049F6D422C0F6030211686C
:1023700043F60803C4F20203196049F6DC20C0F6F4
:102380000300026843F60041C4F202010A6049F604
:10239000D023C0F60303186843F60402C4F2020215
:1023A000106043F60001C4F202010B6843F0807034
:1023B00008600A46116811F0007FFBD043F608035D
:1023C000C4F2020318684FF0020262F301001860C1
:1023D00019460B6803F00C000828FAD143F64401B3
:1023E000C4F202010A6842F480430B6043F63000F5
:1023F000C4F20200016841F48012026047F2000357
:10240000C4F20003196841F480721A6047F20403B1
:10241000C4F20003196841F400721A60036843F4BF
:102420008021016043F61440C4F20200016848F6BE
:102430004462C0F60302136849F6CC20C0F60300DC
:1024400002686FEA020259400A4206D048F6446028
:10245000C0F603004178CC2904D12A4B2A4999427D
:1024600021D344E043F60841C4F2020142F63B2086
:10247000C0F61900086046F67F60C4F65D4008604B
:10248000134043F61442C4F202021360136843F08F
:102490000201116043F60C40C4F20200026812F41B
:1024A000803FFBD1D9E7194C194D281B20F00305BB
:1024B0004FF0000340F20002C1F200024BF6AC51B3
:1024C000C0F6030105F10404C5F380005D589D507A
:1024D00003F10403A3420CD109E05858985003F1CA
:1024E00004035858985003F10403A342F5D130BCBB
:1024F00070470028F1D05858985003F10403A342C4
:10250000EBD1F4E738FA0308ACBD0308B0BD03080B
:102510003BFA030843F63003C4F202031A6842F49C
:1025200000101860196841F480021A60704700BFFB
:102530002DE9F0011546002A66D041F6A803C2F243
:10254000010353E8002F02F1010243E80024012CAB
:10255000F7D049F6E422C0F60302146846F20846B2
:10256000C4F20206346049F6F027C0F603073A6861
:1025700046F22843C4F202031A604FF6FF7846F28F
:10258000304CC4F2020C46F23447C4F2020746F261
:102590002C46C4F202061C46454534BF2B46434632
:1025A000CCF8001038603360226842F001022260EB
:1025B000ED1A4FEA8303C918C018226812F0010F00
:1025C000FBD1002DE8D141F6A803C2F2010353E884
:1025D000002FA2F1010243E80024012CF7D053E8B8
:1025E000002FB2F1004F0DD14FF0000243E800245C
:1025F000012CF4D04EF60450CEF20000016841F0F8
:1026000080510160BFF32F8FBDE8F001704700BF1C
:1026100070B41646002A37D046F21045C4F20205BF
:102620002C6814F0010FFBD149F6EC22C0F603022E
:10263000146846F20842C4F20202146046F21842DC
:10264000C4F20202116046F21C41C4F202010860A9
:1026500046F21440C4F20200066049F6E822C0F6D1
:102660000302116846F21040C4F2020001600268E1
:1026700042F0010101603BB146F21040C4F2020099
:10268000036813F0010FFBD170BC704743F6104391
:10269000C4F20203186800280DDA43F60441C4F2BC
:1026A000020140F22312C4F267520A6048F6AB13EB
:1026B000CCF6EF530B6043F61040C4F20200016801
:1026C00001F00042002A14BF02200020704700BF22
:1026D00043F61043C4F202031868002807DB43F6F0
:1026E0001041C4F202010A6842F000430B607047D7
:1026F00000F17840B0F5801F2CBF0020012070470A
:102700002DE9F04F83B006460D46FFF7F1FF002894
:1027100056D02846FFF7ECFF002854D0AE4255D8DB
:10272000FDF744FD0190FFF7B1FF0446002841D1B9
:1027300006F178434FEA933049F6F422C0F60302DB
:1027400012F8008041F28830FEF722FF4FF00209B4
:1027500043F6104BC4F2020B43F60C47C4F20207D7
:1027600049F6343AC0F6030AFEF70AFF494668F311
:10277000C60169F3092141F48033CBF80030386891
:1027800010F4803FFBD15AF82820B61808F1010850
:102790005FFA88F8B542E7D24FF06400FEF7F8FE22
:1027A00049F66431C0F60301086843F61043C4F2E9
:1027B00002031860FFF78CFF0198FDF701FD07E0A9
:1027C0004FF0020404E04FF0020401E04FF0020475
:1027D000204603B0BDE8F08F2DE9F04106460C46D7
:1027E00015460846FFF784FF002861D005F1FF3049
:1027F0002018FFF77DFF00285DD041F6A803C2F244
:10280000010353E8002F02F1010243E800210129EE
:10281000F7D0FFF73BFF074630BB49F66831C0F6FB
:1028200003010A6843F61040C4F2020002608DB151
:1028300006F1FF3843F60C46C4F20206336813F47F
:10284000803FFBD118F8011F04F8011BFEF798FE2A
:10285000013DF3D149F66C34C0F60304226843F617
:102860001040C4F202000260FFF732FF41F6A803F5
:10287000C2F2010353E8002FA2F1010243E8002451
:10288000012CF7D053E8002FB2F1004F0DD14FF0DB
:10289000000243E80024012CF4D04EF60450CEF29E
:1028A0000000016841F080510160BFF32F8F04E008
:1028B0004FF0020701E04FF002073846BDE8F08113
:1028C00041F2E823C2F20103186849F67032C0F6FB
:1028D0000302116801604FF00003036049F674328F
:1028E000C0F603021168416049F61C43C0F60303B9
:1028F0001A68C2614FF00701016249F67833C0F6E9
:1029000003031A680260704741F2E023C2F2010338
:102910001868704770B48568C668446806FB05404F
:102920004118196041F2E020C2F2010000688142C2
:102930000CD2521890420CD341F2E420C2F20100B2
:102940000268891819604FF0010004E04FF00000A0
:1029500001E04FF0000070BC704700BF2DE9F0416E
:102960000546FEF70DFE4FF01E044FF0000841F241
:10297000E826C2F201064FF00107052D26D8DFE850
:1029800005F0030A0F14191E3268936983F00200E0
:10299000C0F340011BE03068416901F0010116E01D
:1029A00032685369C3F3400111E030684169C1F3F3
:1029B000C0110CE032685369C3F3801107E033683B
:1029C000986980F0010101F0010100E0414689B9F8
:1029D00033685A6912F4807F10D1586910F4806FFF
:1029E00010D1384605F066FE013CC6D14FF000001C
:1029F000BDE8F0814FF00100BDE8F0814FF000002C
:102A0000BDE8F0814FF00000BDE8F0812DE9F04114
:102A100084B014461D46072900F2AD80072A00F253
:102A2000AD8001EB810249F67C33C0F6030303EB72
:102A30008202137C002B40F0A48004EB840249F650
:102A40007C33C0F6030303EB8202137C012B40F0BE
:102A50009B8049F67C33C0F6030301EB810653F8F3
:102A6000262004EB840653F826309A4240F08F80EB
:102A700041F2EC27C2F201073870022A15D0032A6E
:102A800025D0012A34D143F64000C4F20200066882
:102A900046F40012026041F2E823C2F2010345F25B
:102AA0000047C4F200071F6022E043F64000C4F272
:102AB0000200066846F48002026041F2E823C2F296
:102AC000010345F60007C4F200071F6010E043F65B
:102AD0004000C4F20200066846F40002026041F2BF
:102AE000E823C2F2010345F60047C4F200071F6065
:102AF00049F67C38C0F6030801EB810108EB81023E
:102B0000107991684FF0000700974FF00106019689
:102B1000D36802934FF003023B46FEF711F904EB32
:102B2000840408EB84042079A16800970196E26888
:102B300002924FF003023346FEF702F9FFF7C0FEA0
:102B400045B341F2E420C2F201000A99016041F26A
:102B5000E022C2F201020B9B136041F2F020C2F2AC
:102B6000010049F62041C0F603012A463B4607F022
:102B70006FFA304610E04FF000000DE04FF000001B
:102B80000AE04FF0000007E04FF0000004E04FF0D3
:102B9000000001E04FF0010004B0BDE8F08100BF8B
:102BA00038B5044641F2E823C2F201031D68A86962
:102BB00010F0020F63D0FFF783FEA96911F0020F36
:102BC0005DD03BE041F2E825C2F201052B684FF0F1
:102BD000A0021A614FF00200FFF7C0FE2868816969
:102BE00011F0010F08D0456915F4806F00F03882AC
:102BF000036843F4007202604FF0050003F02CFEFE
:102C00004FF0000516E041F2E820C2F20100016831
:102C10004FEA14230B614FF00300FFF79FFE38B11A
:102C200041F2E822C2F201021068E4B2046101E05C
:102C30004FF00005281C18BF012038BD4FF00000E0
:102C400038BD4FF0000038BD4FF0000038BD4FF0E8
:102C5000000038BD4FF0000038BD4FF0000038BD17
:102C60004FF0000038BD4FF0000038BD4FF00000BD
:102C700038BD4FF0000038BD4FF0000038BD41F2C4
:102C8000E822C2F2010213684FF00000586119688F
:102C900060F3492119601A6842F4807018604FF09F
:102CA0000100FFF75BFE0028CBD041F2E825C2F21D
:102CB00001052B684FF0A00119614FF00200FFF7EA
:102CC0004DFE2868826912F0010F08D0436913F4A1
:102CD000806F00F0C881016841F4007202604FF01B
:102CE000050003F0B9FD41F2E820C2F201000368DB
:102CF0004FF0000159611A6861F349221A6018689F
:102D000040F4807119604FF00100FFF727FE0028A2
:102D10009AD041F2E825C2F201052B684FF0A002DB
:102D20001A614FF00200FFF719FE2868816911F05F
:102D3000010F08D0436913F4806F00F09781026897
:102D400042F4007101604FF0050003F085FD41F28F
:102D5000E820C2F2010003684FF0000159611A68CF
:102D600061F349221A60186840F4807119604FF0CD
:102D70000100FFF7F3FD00283FF469AF41F2E825B9
:102D8000C2F201052B684FF0A0021A614FF0020059
:102D9000FFF7E4FD2868816911F0010F08D043694D
:102DA00013F4806F00F06581026842F400710160E5
:102DB0004FF0050003F050FD41F2E820C2F201009F
:102DC00003684FF0000159611A6861F349221A60E3
:102DD000186840F4807119604FF00100FFF7BEFDE4
:102DE00000283FF437AF41F2E825C2F201052B6815
:102DF0004FF0A0021A614FF00200FFF7AFFD286804
:102E0000816911F0010F08D0436913F4806F00F05D
:102E10003381026842F4007101604FF0050003F055
:102E20001BFD41F2E820C2F2010003684FF00001EF
:102E300059611A6861F349221A60186840F4807178
:102E400019604FF00100FFF789FD00283FF405AF3E
:102E500041F2E825C2F201052B684FF0A0021A6189
:102E60004FF00200FFF77AFD2868816911F0010F29
:102E700008D0436913F4806F00F00181026842F4C6
:102E8000007101604FF0050003F0E6FC41F2E8201C
:102E9000C2F2010003684FF0000159611A6861F342
:102EA00049221A60186840F4807119604FF00100DF
:102EB000FFF754FD00283FF4D3AE41F2E825C2F2FB
:102EC00001052B684FF0A0021A614FF00200FFF7D6
:102ED00045FD2868816911F0010F08D0436913F49A
:102EE000806F00F0CF80026842F4007101604FF003
:102EF000050003F0B1FC41F2E820C2F201000368D2
:102F00004FF0000159611A6861F349221A6018688C
:102F100040F4807119604FF00100FFF71FFD002899
:102F20003FF4A1AE41F2E825C2F201052B684FF053
:102F3000A0021A614FF00200FFF710FD28688169B6
:102F400011F0010F08D0436913F4806F00F09D80E9
:102F5000026842F4007101604FF0050003F07CFC50
:102F600041F2E820C2F2010003684FF0000159610C
:102F70001A6861F349221A60186840F48071196078
:102F80004FF00100FFF7EAFC00283FF46FAE41F27A
:102F9000E825C2F201052B684FF0A0021A614FF03C
:102FA0000200FFF7DBFC2868816911F0010F07D0F0
:102FB000436913F4806F6BD0026842F400710160C2
:102FC0004FF0050003F048FC41F2E820C2F2010096
:102FD00003684FF0000159611A6861F349221A60D1
:102FE000186840F4807119604FF00100FFF7B6FCDB
:102FF00000283FF43EAE41F2E825C2F201052B68FD
:103000004FF0A0021A614FF00200FFF7A7FC2868FA
:10301000816911F0010F07D0436913F4806F3AD032
:10302000026842F4007101604FF0050003F014FCE7
:1030300041F2E820C2F2010003684FF0000159613B
:103040001A6861F349221A60186840F480711960A7
:103050004FF00100FFF782FC00287FF4B3AD0BE6D0
:103060004FF0010519E04FF00A0516E04FF0090591
:1030700013E04FF0080510E04FF007050DE04FF0AA
:1030800006050AE04FF0050507E04FF0040504E0EF
:103090004FF0030501E04FF0020541F2EC20C2F2CF
:1030A0000100017801F1FF33DAB2012A3FF6B8AD31
:1030B000A9E500BFF8B50D461446002A6FD080B2CE
:1030C000FFF76EFD002865D04FF00300FFF746FCC8
:1030D00000285FD041F2E823C2F2010318680268B9
:1030E00042F4807101604FF00100FFF737FC0028C7
:1030F00050D041F2E823C2F20103186814F1FF3105
:1031000018BF0121026861F38A2202604FF0A10317
:1031100003614FF00200FFF721FC00283AD041F292
:10312000E820C2F2010001688A6912F0010F31D073
:103130004B6913F4806F2DD14FF0040641F2E8275C
:10314000C2F201073046FFF709FC18B304F1FF345F
:10315000012C27D1FDF72AF839680A696FEA0203C2
:1031600005F8013B0A686FF38A220A60FDF728F828
:10317000E8E72B681B6902E04FF004060E4D30466D
:10318000FFF7ECFB0028F4D10B4B1868016841F401
:1031900000720260D4F1010038BF0020F8BD4FF08A
:1031A0000100F8BD386801696FEA010205F8012BDA
:1031B000002CC7D1E0E700BFE812012030B583B092
:1031C00015461C461A4601ABFFF7A4FB48B101980F
:1031D00029462246FFF76EFF00280CBF182000206A
:1031E00001E04FF01F0003B030BD00BF2DE9F84FE4
:1031F00093460D4600295DD004464FF0030841F286
:10320000E829C2F2010901E0002E40D01FFA8BF03C
:10321000FFF7C6FC00283DD00BF0070715F0010FA3
:103220004CD14046FFF79AFB002836D0072F1AD81A
:10323000DDB13CB1D9F8000014F8011B6FEA0103BD
:10324000036104E0D9F800604FF0FF02326107F13A
:103250000107BA4605F1FF3635464046FFF77EFBCB
:10326000002845D119E02E4600E02E46D9F800008E
:10327000026842F4007101600BF1080B2BF0070BA0
:103280004FF00500FFF76AFB0028BDD107E04FF0C3
:10329000010004E04FF0000001E04FF0000041F2B7
:1032A000E823C2F2010319680A6842F400730B6054
:1032B000BDE8F88F4FF00100BDE8F88F4046FFF7FA
:1032C0004DFB0028E9D0072FCDD82CB9D9F8003014
:1032D0004FF0FF021A6106E0D9F8000014F8011B54
:1032E0006FEA0103036107F1010705F1FF3598E774
:1032F000072FB8D82CB9D9F800504FF0FF022A6137
:1033000006E0D9F8000014F8011B6FEA010303611D
:1033100007F1010706F1FF3583E700BF30B583B041
:1033200015461C461A4601ABFFF7F4FA48B1284689
:103330002146019AFFF75AFF00280CBF18200020F1
:1033400001E04FF01F0003B030BD00BF08B542F2EE
:103350004C50C2F2010042F64C02C2F20102131AB2
:103360004FF0FF314FEAA302FCF7DAFE42F64C00C1
:10337000C2F2010043F24C01C2F201010A1A4FEA03
:10338000A2024FF0FF31A2F12002FCF7C9FE02F0C9
:103390004FFA41F20030C2F2010044F20001C4F2DF
:1033A00002014FF480524FF0030312F0A5FCFDF729
:1033B00085FA4FF0000008BDBFF36F8F704700BF64
:1033C00049F6B443C0F60303185C00EB400149F62C
:1033D000D052C0F6030252F821305B68704700BF3C
:1033E00038B549F6B443C0F603031B5C03EBC304D2
:1033F00041F21832C2F2010202EB840282F821107B
:1034000014693CB141F21835C2F201051346D26984
:103410009B69A04738BD00BFF8B506460F4649F680
:10342000B443C0F603031D5C05EBC50041F218343C
:10343000C2F2010404EB8004D4F810C0BCF1000F08
:1034400007D0E2698A4204D030464FF00001A369F8
:10345000E047E76163695BB105EBC50041F21832F3
:10346000C2F2010202EB8002304639469269984767
:1034700094F8201079B127696FB105EBC50541F2C9
:103480001833C2F2010303EB8505304694F821108E
:10349000E269AB69B847F8BD49F6B443C0F6030327
:1034A000185C00EB400149F6D052C0F6030252F816
:1034B0002130D86840F08001D9607047F8B50446E3
:1034C00000EB400249F6D053C0F6030353F82260E4
:1034D00035686FEA0500306005F0010215F0020F53
:1034E0001CBF42F00202D2B215F0040F18BF42F026
:1034F000080215F0080F18BF42F0040215F4807F8F
:1035000005D0316911F4804F18BF42F0100215F058
:10351000200F00D1E2B104EBC40741F21833C2F22C
:10352000010303EB870087688FB1716804EBC40067
:1035300041F21833C2F2010303EB800349F66050F5
:10354000C0F60300005DC9B29B69B84700E073682C
:10355000F26812F0800F1CD015F0800F19D0F168BE
:103560006FF3C711F16004EBC40041F21833C2F2EB
:10357000010353F8203063B141F21832C2F2010264
:1035800002EB800249F66050C0F60300005D9169CD
:10359000984715F0400F17D004EBC40141F21833DF
:1035A000C2F2010303EB810253686BB1084641F29A
:1035B0001831C2F2010101EB800249F66050C0F6F9
:1035C0000300005D91699847F8BD00BF684620F090
:1035D00007018D4601B54FF00600FFF76FFFBDE80C
:1035E00001408546704700BF684620F007018D46C0
:1035F00001B54FF00500FFF761FFBDE801408546CA
:10360000704700BF684620F007018D4601B54FF0B6
:103610000400FFF753FFBDE801408546704700BF37
:10362000684620F007018D4601B54FF00300FFF713
:1036300045FFBDE801408546704700BF684620F061
:1036400007018D4601B54FF00200FFF737FFBDE8D7
:1036500001408546704700BF684620F007018D464F
:1036600001B54FF00100FFF729FFBDE80140854695
:10367000704700BF10B582B08DF8071049F6B4430B
:10368000C0F60303185C00EB400249F6D051C0F6C7
:10369000030151F82240236813F0800FFBD002A9E8
:1036A00011F8012D626000EBC00041F21834C2F243
:1036B000010404EB8004608C4FF0010205F012F865
:1036C000608404F1200402B010BD00BF70B582B068
:1036D0008DF8071049F6B443C0F60303185C00EBFD
:1036E000400149F6D052C0F6030252F82140256845
:1036F00015F0800F1DBF9DF807506560012600265C
:1037000000EBC00341F21830C2F2010000EB830568
:10371000688C0DF107014FF0010204F0E3FF6884AB
:1037200005F12005E16841F08002E260304602B018
:1037300070BD00BF2DE9F84F81468B4690461E466E
:103740009DF828A049F6B443C0F603031D5C05EBC1
:10375000450249F6D050C0F6030050F822409DF8CB
:103760002C70012F14BF00270127082E06D0072E2A
:1037700002D1B8F1000F01D1FCF7C2FC0AF1FF3110
:10378000CBB2012B01D9FCF7BBFC49F6B452C0F611
:10379000030252F82500B0FBFBF1A1604FF00002DC
:1037A00067F38612BAF1010F04D0002F0CBF022379
:1037B000002301E04FF0000363F30D3267F38E3214
:1037C00022614FF06C00B8F1020F14BF00230123F7
:1037D00063F3492018F1000818BF4FF0010868F39F
:1037E0008A20082E18BF4FF0000868F30C3040F410
:1037F0000051E1604846FFF7E3FDBDE8F88F00BFE8
:10380000F0B585B00D461E4649F6B443C0F6030335
:10381000195C01EB410449F6D057C0F6030757F88D
:10382000247049F6B053C0F60303185C00EB400166
:1038300049F66854C0F6030404EBC1040AB1FCF76E
:103840005FFC75B9207B21699DF82C2000924FF018
:1038500001030193626902924FF003023346FDF7C0
:103860006FFA207861689DF8283000934FF00102CC
:103870000192A36802934FF003023346FDF760FA0A
:1038800049F6B840C0F603000168012D14BF0025B9
:10389000012565F3C301796105B0F0BD2DE9F84359
:1038A000054649F6B443C0F60303185C00EBC002BA
:1038B00041F21834C2F2010404EB820449F6D051FB
:1038C000C0F6030100EB40064FEA860301EB030854
:1038D00051F80390FCF76AFC064694F82000B8B152
:1038E0004FF00007C9F80C703846394698F90420A3
:1038F000FCF7CEFC28463946FFF772FDE3681BB1A2
:103900002846E169A26998474FF0000284F8202018
:103910003046FCF755FCBDE8F88300BF2DE9F04FB9
:1039200085B005468B469246994649F6B443C0F6A3
:1039300003031E5C41F21838C2F2010806EBC60709
:103940004FEA870708EB070406EB460049F6D0511B
:10395000C0F6030101EB8006FCF728FC039043F658
:103960004003C4F202031A6849F62460C0F603005B
:10397000016822EA010249F6AC40C0F60300016882
:103980000A431A6043F64403C4F202031A681A6039
:1039900049F64C51C0F6030105EB8503C818C95C14
:1039A0004278837890F803E0CDF800E00079019048
:1039B0002846FFF725FF9DF8382000929DF83C101F
:1039C00001912846594652464B46FFF7B3FE109BDD
:1039D00048F807301298A060119A62601399E1606C
:1039E000149BA361B0684FF00F0196F90420FCF717
:1039F0004FFC4FF0010084F820000398FCF7E0FB37
:103A000005B0BDE8F08F00BF49F6B443C0F603032C
:103A1000185C00EBC00341F21830C2F2010000EB69
:103A2000830319615A61704749F6B053C0F6030326
:103A3000185C00EB400149F6BC42C0F6030202EB01
:103A400001107047FA2884BF0530C0B2032812D88D
:103A500049F6B443C0F60303185C00EBC00141F221
:103A60001832C2F2010202EB81034FF6FF70588454
:103A70004FF0010070474FF000007047FA2884BFF4
:103A80000530C0B203280ED849F6B443C0F603038C
:103A9000185C00EBC00141F21832C2F2010202EBE5
:103AA0008103588C70474FF000007047082806D9F2
:103AB000102807D920288CBF4020202070474FF0C5
:103AC000080070474FF01000704700BF022809D06F
:103AD000032804D0012814BF0020012070474FF0B4
:103AE000030070474FF00200704700BF40F600131C
:103AF000C5F20003186840F60802C5F2000211681A
:103B0000C1F34103022B12BF6FF30200032363F3DF
:103B1000020040F400406FF3995040F60012C5F2E5
:103B20000002106040F60401C5F200010B6843F486
:103B300080700860704700BF49F63C63C0F603031D
:103B40001A6840F61030C5F200000260704700BFEE
:103B500010B441F61863C2F201031A5CE0B14FF0F1
:103B6000000341F6B431C2F201014FF04C0404FBF2
:103B70000212D16821F0030202F1040262F312037F
:103B80004FF0010161F3DC4349F64462C0F60302E1
:103B900002EB401081690B6010BC704770B440F2BA
:103BA0002003C5F200031868C0F34342022A01D083
:103BB000062A29D100F00F0149F6D465C0F60305A5
:103BC00055F82160C0F30A1505F1030398081BD0CE
:103BD00041F20001C5F2000100F1FF3404F00104DC
:103BE0000A68334672604FF0010282420ED10AE049
:103BF0000C6803F1040343F8044F0C685C6002F1A5
:103C000002028242F4D1356070BC7047002CEFD0C4
:103C10000C6803F104035C6002F101028242E7D107
:103C2000F1E700BF70B449F6C463C0F6030353F86C
:103C300020603268002A3CD049F64461C0F6030196
:103C400001EB401102F103024FEA9202CB691B68BB
:103C50009A420CD940F63402C5F2000211684FF0C6
:103C6000010303FA00F008431060184623E006F150
:103C70000403C2B102F1FF3000F00105086953F8F6
:103C8000044B0460501E18D10DE00C691A4652F81E
:103C9000045B256000F1FF300C695B68236002F172
:103CA00004030138F1D14FF0000131604FF0010001
:103CB00001E04FF0000070BC7047002DE5D00A69AC
:103CC00053F8044B14600138DFD1ECE708B54FF02E
:103CD000010303FA00F041F21642C2F20102138816
:103CE000184210D023EA000341F21640C2F201004C
:103CF0000380CA6B52B1086A4FF0000103F03EFF27
:103D00004FF0000008BD4FF0000008BD4FF001006B
:103D100008BD00BF70B540F21403C5F200031C6873
:103D200049F62C60C0F6030001680C4200F0BB812C
:103D300041F66432C2F201021378012B40F2B381E2
:103D400040F21800C5F20000016849F64062C0F672
:103D500003021368194200F0A68140F61800C5F26C
:103D60000000016811F0010F56D040F60815C5F2A9
:103D700000052A6840F60830C5F2000003682A6092
:103D8000036041F61861C2F20101087841F6B431CE
:103D9000C2F201014FF04C0505FB001503F00100D4
:103DA000E96A0143E962C3F3C000296B0143296357
:103DB00003F00803D8B258BBD2B212F0010F0ED0F4
:103DC0001DE0EA6A22B105F1100000F063FF2BE06C
:103DD0002B6B002BF7D1686B0028F4D124E012F094
:103DE000900FEED040F63403C5F20003186820F0BF
:103DF000010119604FF00000FFF714FFE1E76E6B5F
:103E00004FF000002946FFF761FF30436863D8E7B1
:103E10004FF00001E963CFE740F61802C5F2000257
:103E2000136813F4803FA0D140F61801C5F20001D9
:103E30000A6802F0020398B2002856D040F628150E
:103E4000C5F200052A6840F62830C5F20000036874
:103E50002A60036041F61861C2F20101487841F618
:103E6000B431C2F201014FF04C0505FB001503F01F
:103E70000100E96A0143E962C3F3C000296B014311
:103E8000296303F00803D8B258BBD2B212F0010F75
:103E90000ED01DE0EA6A22B105F1100000F0FAFE32
:103EA0002FE02B6B002BF7D1686B0028F4D128E0B2
:103EB00012F0900FEED040F63403C5F200031868FC
:103EC00020F0020119604FF00100FFF7ABFEE1E7BF
:103ED0006E6B4FF001002946FFF7F8FE3043686330
:103EE000D8E74FF00001E963CFE740F61801C5F2CB
:103EF00000010A684FEA124303F0020081B2002970
:103F00009CD140F61801C5F200010A6802F00403D2
:103F100098B2002856D040F64815C5F200052A6828
:103F200040F64830C5F2000003682A60036041F69D
:103F30001861C2F20101887841F6B431C2F2010180
:103F40004FF04C0505FB001503F00100E96A014341
:103F5000E962C3F3C000296B0143296303F008033E
:103F6000D8B258BBD2B212F0010F0ED01DE0EA6AEF
:103F700022B105F1100000F08DFE2FE02B6B002B1D
:103F8000F7D1686B0028F4D128E012F0900FEED042
:103F900040F63403C5F20003186820F004011960EC
:103FA0004FF00200FFF73EFEE1E76E6B4FF00200BC
:103FB0002946FFF78BFE30436863D8E74FF00001D6
:103FC000E963CFE740F61801C5F200010A684FEA3D
:103FD000124303F0040081B200299CD140F618017D
:103FE000C5F200010A6802F0080398B258B940F619
:103FF0001801C5F200010A684FEA124303F00800F5
:1040000081B200294FD040F66815C5F200052A6834
:1040100040F66830C5F2000003682A60036041F68C
:104020001861C2F20101C87841F6B431C2F201014F
:104030004FF04C0505FB001503F00100E96A014350
:10404000E962C3F3C000296B0143296303F008034D
:10405000D8B210B14FF00001E963D2B212F0010FF3
:1040600008D06E6B4FF003002946FFF72FFE304358
:1040700068630EE012F0900F0BD040F63403C5F2E7
:104080000003186820F0080119604FF00300FFF7E3
:10409000C9FDEA6A1AB92B6B0BB9686B18B105F147
:1040A000100000F0F7FD14F0100F01D0FFF776FDBF
:1040B00014F4805F0DD041F6A931C2F201014FF036
:1040C00001020A7041F66833C2F20103186802F077
:1040D0002DFA14F4005F01D0FFF708FD14F4006F0F
:1040E00014D041F6A830C2F201004FF00101017076
:1040F00041F61563C2F201034FF000021A7041F657
:104100006830C2F20100006802F010FA002C14DAE4
:1041100041F6A831C2F201014FF000030B7041F6E5
:104120001560C2F201004FF00102027041F66831E1
:10413000C2F20101086802F0F9F940F21403C5F275
:1041400000031C6070BD00BF684620F007018D466B
:1041500089B500AFFFF7DEFDBD46BDE88940854665
:10416000704700BF2DE9F04141F6B436C2F20106B6
:104170004FF04C0303FB0066304650F8205F49F6D1
:104180004468C0F603084FEA451708EB07044FF0F0
:1041900000014FF01C0213F03BF835624FF00100B4
:1041A000B06258F807204FF00003136061690B609C
:1041B000A0684FF0FF02026061680B60A0690360B5
:1041C000E1680A6049F6D462C0F6030252F825009D
:1041D000036049F6C461C0F6030151F8252013605D
:1041E000BDE8F08100B583B04FF00003019340F2C9
:1041F0001001C5F200010A68B0F1FF3F08BF1020AE
:1042000060F3891242F0200040F21003C5F200036F
:104210001860194640F63F52C0F20302019800F1BF
:10422000010001900B6813F0200F02D0019890421A
:10423000F4D94FF0030004F03DFA03B000BD00BF15
:104240002DE9F8434FF04C0303FB00F041F6B43185
:10425000C2F201014418256A4FF0010606FA05F67C
:1042600049F64462C0F6030202EB451740580028A5
:1042700067D0A368FBB1D7F80080D8F8001011F41C
:10428000004F18D1D8F80020914663F30A09007A4C
:10429000FFF71CFC60F3934949F4004965F3995911
:1042A00049F08050C0F3404363F39A60C8F80000BF
:1042B0002846FFF797FFE168F1B17A68106810F4BB
:1042C000004F19D12846FFF743FCD7F80480D8F8EF
:1042D0000070E36863F30A072168087AFFF7F6FBCA
:1042E00060F3934747F4004242F01047C7F3404061
:1042F00060F39A67C8F8007049F6D463C0F6030308
:1043000053F825104FF000020A60A06858B140F63B
:104310001C03C5F20003196846EA010290B219684D
:1043200060F30F011960E3685BB140F61C00C5F251
:104330000000026846EA1246B6B2016866F31F4101
:104340000160BDE8F88300BF70B582B04FF0000295
:10435000019240F21003C5F20003196841F0010018
:10436000186001921A6812F0010F19D0019940F6F5
:104370003F53C0F20303994212D840F21000C5F235
:10438000000040F63F52C0F20302019901F1010121
:104390000191036813F0010F02D001999142F4D901
:1043A0004FF0030004F086F94FF00000019040F256
:1043B0001002C5F200021368002B1DDB019940F6C4
:1043C0003F50C0F20300814216D84FF0030640F27E
:1043D0001005C5F2000540F63F54C0F20304304614
:1043E00004F068F9019A02F1010201922B68002B96
:1043F00002DB0199A142F2D902B070BD00B583B0D1
:104400004FF00003019340F21000C5F20000026873
:1044100042F01001016040F63F52C0F20302019BDE
:1044200003F101030193016811F0100F02D0019B09
:104430009342F4D94FF0030004F03CF903B000BDFF
:1044400050B149F63461C0F603010A6840F218031E
:10445000C5F200031A60704749F63863C0F60303DB
:104460001A6840F21800C5F200000260704700BFF1
:1044700038B54FF0000440F60063C5F200031C603D
:1044800040F60002C5F20002106840F0030164F338
:10449000820164F30A11116040F22405C5F200059F
:1044A0002B684FF0400262F30F032B60204662F34B
:1044B0001F40214662F31F4162F30F0140F22805BD
:1044C000C5F2000529604FF0800363F30F0040F24E
:1044D0000412C5F2000210604FF0C00161F30F003A
:1044E00040F20815C5F2000528604FF4807363F3AD
:1044F0000F0040F20C12C5F2000210604FF0FF30C6
:10450000FFF770FEFFF77AFF40F61000C5F20000DB
:10451000046040F61401C5F200010C604FF0FF3555
:1045200040F61803C5F200031D6040F61C02C5F2F8
:10453000000214602046FFF715FE4FF00100FFF760
:1045400011FE4FF00200FFF70DFE4FF00300FFF7E2
:1045500009FE4FF00400FFF705FE4FF00500FFF7DE
:1045600001FE4FF00600FFF7FDFD4FF00700FFF7DB
:10457000F9FD40F21800C5F20000046040F2140199
:10458000C5F200010D604FF00100FFF759FF38BD83
:1045900041F21643C2F2010319884FF0010202FAF8
:1045A00000F0084000280CBF02200320704700BF25
:1045B00040F60013C5F200031B68C3F3076202F064
:1045C0008000C1B209B143F0804343F4001040F6CB
:1045D0000012C5F200021060704700BF2DE9F843D9
:1045E0000546164649F64468C0F6030808EB40182D
:1045F00049F6C463C0F6030353F820704FF0010975
:1046000009FA00F90C46A9B9386840B941F21643D5
:10461000C2F20103188819EA000F5AD10AE041F2E8
:104620001641C2F201010A8819EA020F02D0284697
:10463000FFF7D8FD06F1030107F1040388081CD039
:1046400000F1FF3202F0010CA4F1040151F8042F33
:1046500043F8042B01383ED10FE001F10402496810
:104660001C4644F8041B00F1FF3002F104015268BB
:104670005A6004F104030138EFD13E6041F2164361
:10468000C2F20103198849EA0109A3F8009065B94B
:1046900040F61010C5F2000002684FF0010161F30E
:1046A000D44266F30602026009E0D8F814000268FA
:1046B0004FF0010363F3DC4266F312020260D8F8A4
:1046C0000030186840F004421A6016B12846FFF71F
:1046D000A9FABDE8F883BCF1000FBED051F8042F51
:1046E00043F8042B0138B8D1C7E700BF70B50446C2
:1046F00049F6D463C0F6030353F82060334653F8F9
:10470000045BAA4238BF1546084619462A4612F0ED
:104710005BFD4FF0000030602046FFF719FA49F6C4
:104720004461C0F6030101EB441463681A6842F067
:1047300004401860284670BDF8B5054641F6B4330C
:10474000C2F201031868002871D041F6B431C2F2F8
:104750000101CA6C002A71D041F6B434C2F20104DE
:10476000D4F89860002E6DD041F6B437C2F201073C
:10477000D7F8E430002B69D041F6B430C2F2010022
:10478000D0F83011002965D041F6B432C2F20102EE
:10479000D2F87C41002C61D041F6B436C2F2010659
:1047A000D6F8C871002F5DD041F6B433C2F20103D0
:1047B000D3F81402002859D041F6B431C2F20101F5
:1047C000D1F86022002A55D0464E4FF00807FBF77B
:1047D00097FC2C7A002C53D041F21442C2F2010211
:1047E0001088014610F0020F55D04FF0010404F17B
:1047F000010441FA04F212F0010FF8D14FF0010167
:1048000001FA04F1084341F21443C2F20103188093
:1048100044B96889FFF74AF9B060A889FFF746F9FB
:10482000F06042E06A89B260A989F1603DE041F63A
:10483000B436C2F201064FF000071EE02A4E4FF0D8
:1048400001071AE0294E4FF0020716E0284E4FF0FC
:10485000030712E0274E4FF004070EE0264E4FF0FC
:1048600005070AE0254E4FF0060706E0244E4FF0FC
:10487000070702E01B4E4FF00807072FA9D9A6E74C
:1048800041F21443C2F20103188840F0010119807B
:104890004FF00004BDE740F0020441F21443C2F2BD
:1048A00001031C804FF00104BCE741F61860C2F21E
:1048B00001000755374647F8205B38464FF00001A6
:1048C0004FF01C0212F0A4FC34626B68B36306F173
:1048D00010004FF006012A683B4600F0BBF9204665
:1048E000F8BD00BF141E0120001C01204C1C01203B
:1048F000981C0120E41C0120301D01207C1D01209A
:10490000C81D0120022907D140F60003C5F20003AB
:104910001A6860F30A121A60704700BF10B54FF0B2
:10492000000440F63403C5F200031C6040F60400A6
:10493000C5F20000026842F0010101602046FFF765
:1049400011FC4FF00100FFF70DFC4FF00200FFF7E4
:1049500009FC4FF00300FFF705FC4FF00400FFF7E0
:1049600001FC4FF00500FFF7FDFB4FF00600FFF7DD
:10497000F9FB4FF00700FFF7F5FB4FF0FF30FFF7B3
:1049800031FC41F21643C2F201031C8040F61800CC
:10499000C5F200004FF0FF32026049F63061C0F608
:1049A0000301086840F61C03C5F20003186049F6CD
:1049B000E862C0F60302116840F61400C5F2000078
:1049C000016049F6E463C0F603031A6840F610017B
:1049D000C5F200010A6020464FF00201FFF792FF86
:1049E000FFF7AAF82046FFF72BFC4FF00100FFF776
:1049F00027FC4FF00200FFF723FC4FF00300FFF706
:104A00001FFC4FF00400FFF71BFC4FF00500FFF701
:104A100017FC4FF00600FFF713FC4FF00700FFF7FD
:104A20000FFC10BD08B5FFF779FF08BD704700BF48
:104A3000F0B585B0054641F28830FCF7A9FD002DA0
:104A400062D043F63401C4F202010C6844F08006DF
:104A50000E604FF0000400944FF0030601964FF0F3
:104A60000A07029720464FF00B0132462346FCF717
:104A700067F900940196029720464FF00C013246E8
:104A80002346FCF75DF940F20C06C5F200063368D8
:104A900043F040023260FFF757FC40F23800C5F2A5
:104AA00000004FF40411016044F6206003F002FEA0
:104AB000FCF766FD336843F0400064F3082064F3BC
:104AC00049204FF0050262F38D2064F35D7040F0E1
:104AD0008041316044F6206003F0ECFDFCF750FDAE
:104AE000FFF7C6FC40F20803C5F2000340F2811054
:104AF000186044F24910C0F602004FF00F014FF069
:104B00004302FBF7C5FB13E04FF000004FF00F012D
:104B10004FF04302FBF7BCFB4FF0000340F23802BA
:104B2000C5F20002136040F21800C5F200000360F5
:104B30002846FFF77BFF4FF06400FCF729FD05B026
:104B4000F0BD00BF2DE9F04182B049F6EC67C0F638
:104B5000030744F62546C0F6020640F28815C2F265
:104B600000054FF00408CDF8008038464FF0800172
:104B700032462B4601F026FE41F21844C2F20104EF
:104B80002060CDF8008038464FF08101324605EBB9
:104B9000080301F017FE6060CDF8008038464FF042
:104BA0008201324605F1080301F00CFEA060CDF849
:104BB000008038464FF08301324605F10C0301F0C6
:104BC00001FEE060CDF8008038464FF084013246A7
:104BD00005F1100301F0F6FD2061CDF800803846A4
:104BE0004FF08501324605F1140301F0EBFD6061E1
:104BF000CDF8008038464FF08601324605F11803A3
:104C000001F0E0FDA061CDF8008038464FF087014B
:104C1000324605F11C0301F0D5FDE06102B0BDE8AC
:104C2000F08100BF08B505464FF000060BE0FBF72A
:104C3000BDFA2C68616829606660FBF7C1FA2268DA
:104C40000AB1A06890472B68B3F1FF3FEFD101F0A4
:104C50003BFCF8E70260B3F1FF3F18BF8360FF2918
:104C60000ED142F24853C2F201031A6822B192F8FF
:104C700029304FEA530101E04FF0070101737047FB
:104C800001F07F010173704710B14FF00002026024
:104C9000704700BF38B50446FBF788FA0546A4B153
:104CA000636893B9227B40F28810C2F2000050F88A
:104CB0002210616040F82240227B41F21843C2F288
:104CC000010353F8220001F031FC2846FBF778FA83
:104CD00038BD00BF10B5044641F23860C2F2010091
:104CE0004FF000014FF0240212F092FAD4B141F2D9
:104CF0006040C2F201004FF000014FF0480212F094
:104D000087FA41F21050C2F201004FF000014FF05B
:104D1000240212F07DFA41F20853C2F201034FF06F
:104D200002021A7010BD00BF38B549F61073C0F604
:104D3000030353F8205041F2AC41C2F2010151F893
:104D4000204049F65072C0F60302105CFCF78CF864
:104D50002840A04214BF0020012038BD49F65073FE
:104D6000C0F603031A5C41F21051C2F2010151F87E
:104D7000222049F61073C0F6030353F820000242C4
:104D80000CBF00200120704770B441F6A803C2F2A6
:104D9000010353E8002F02F1010243E80021012939
:104DA000F7D049F65072C0F60302155C41F2386143
:104DB000C2F2010151F8254049F61076C0F603060B
:104DC00056F8202024EA020041F8250053E8005F4D
:104DD000A5F1010543E80056012EF7D053E8005F26
:104DE000B5F1004F0DD14FF0000543E80056012EFC
:104DF000F4D04EF60450CEF20000016841F080512C
:104E00000160BFF32F8F14420CBF0020012070BC43
:104E1000704700BF49F66073C0F60303185C704723
:104E200010B50446FCF720F840F2A813C2F20003C4
:104E300053F82410484010BD10B504464FF001004F
:104E4000FFF748FF49F67073C0F6030353F83420A8
:104E500041F20C51C2F201010A6003EBC404606824
:104E600041F2A843C2F20103186010BD00B585B03D
:104E70004FF00000FFF7E0FF4FF00003009341F216
:104E80003452C2F2010201924FF04000029049F602
:104E90004470C0F603004FF0020144F64172C0F6C0
:104EA000020201F07BFB41F23463C2F2010318609D
:104EB00005B000BD2DE9F001804600283CD04FF040
:104EC00000034FEA8302086850F823404D6855F804
:104ED000236086EA0407886850F8235084EA050CAA
:104EE0004CEA07076FEA070CC86850F8235026EA17
:104EF000050707EA0C0705EA0C0C66EA0C063540C4
:104F000040F82350CD6855F82300384345F8230076
:104F10000D6955F82300384345F823004D690DB15C
:104F200045F82370486885588868855048688450DB
:104F300003F101034345C4D1BDE8F001704700BF50
:104F40002DE9F84341F20C58C2F2010841F238460B
:104F5000C2F2010641F23C44C2F201044FF00005E6
:104F600041F2A847C2F20107D8F8000000EB800028
:104F700001F072FC3368002B40F043812046294643
:104F80004FF0240212F044F93BE14FF0090049F6DA
:104F9000F861C0F60301FFF78DFF41F20853C2F23A
:104FA0000103197859B101F1FF3041F20852C2F200
:104FB0000102107041F23863C2F201031D6041F238
:104FC0000451C2F20101086848B941F20452C2F228
:104FD00001021560136813B1284605F00DFF41F278
:104FE0000851C2F20101087858B100F1FF3341F2D3
:104FF0000852C2F20102137041F23861C2F201019B
:105000004D6041F20450C2F2010003684BB941F215
:105010000452C2F201021560116811B1284605F070
:10502000EBFE41F20850C2F2010003785BB103F1DC
:10503000FF3141F20852C2F20102117041F23860B0
:10504000C2F20100856041F20453C2F20103196803
:1050500049B941F20452C2F201021560106810B160
:10506000284605F0C9FE41F20853C2F2010319783F
:1050700059B101F1FF3041F20852C2F20102107041
:1050800041F23863C2F20103DD6041F20451C2F221
:105090000101086848B941F20452C2F201021560E8
:1050A000136813B1284605F0A7FE41F20851C2F279
:1050B0000101087858B100F1FF3341F20852C2F201
:1050C0000102137041F23861C2F201010D6141F237
:1050D0000450C2F2010003684BB941F20452C2F21B
:1050E00001021560116811B1284605F085FE41F2F4
:1050F0000850C2F2010003785BB103F1FF3141F2C5
:105100000852C2F20102117041F23860C2F201008D
:10511000456141F20453C2F20103196849B941F2F1
:105120000452C2F201021560106810B1284605F061
:1051300063FE41F20853C2F20103197859B101F13B
:10514000FF3041F20852C2F20102107041F238639E
:10515000C2F201039D6141F20451C2F201010868EB
:1051600048B941F20452C2F201021560136813B14A
:10517000284605F041FE41F20851C2F201010878CB
:1051800058B100F1FF3341F20852C2F2010213702C
:1051900041F23861C2F20101CD6141F20450C2F224
:1051A000010003684BB941F20452C2F201021560DA
:1051B000116811B1284605F01FFE41F20850C2F2F5
:1051C000010003785BB103F1FF3141F20852C2F2F2
:1051D0000102117041F23860C2F20100056241F231
:1051E0000453C2F20103196849B941F20452C2F2F0
:1051F00001021560106810B1284605F0FDFD35600C
:10520000B2E6D4F800902846FFF70AFE40EA09010A
:105210002160D4F804904FF00100FFF701FE40EA4E
:1052200009026260D4F808904FF00200FFF7F8FD21
:1052300040EA0900A060D4F80C904FF00300FFF79B
:10524000EFFD40EA0903E360D4F810904FF004004A
:10525000FFF7E6FD40EA09012161D4F814904FF010
:105260000500FFF7DDFD40EA09026261D4F81890FD
:105270004FF00600FFF7D4FD40EA0900A061D4F822
:105280001C904FF00700FFF7CBFD40EA0903E361F4
:10529000D4F820904FF00800FFF7C2FD40EA090162
:1052A0002162306800F1010030603A689042FFF4FA
:1052B0005BAE6AE600B585B04FF00003009341F2A3
:1052C0009C62C2F2010201924FF04000029049F646
:1052D0009070C0F603004FF0060145F2F522C0F6CB
:1052E000020201F05BF941F25C63C2F20103186053
:1052F00005B000BD2DE9F04F85B041F60C031E4608
:10530000C2F2010641F2C4700746C2F2010741F23F
:105310007861C2F20101019101F0D6F83268002AE9
:10532000FAD061E1E359002B53D02846FFF778FD0E
:1053300001996258605090434BD0E35910EA030240
:1053400047D0039991F800E049F69879C0F603092F
:105350004FEA451841F26061C2F201014FF6FF7C4D
:105360004AF2B80AC0F6030A41F2A07BC2F2010B6E
:1053700000957046C2F10003134022EA030218B9F7
:1053800054F80B502B4221D15FEA136E04D01AF867
:105390000E3003F118030EE01D0C04D01AF805308E
:1053A00003F1100307E05FEA132E1ABF1AF80E305C
:1053B00008331AF80330434419F8035031F815E064
:1053C000E6451CBF0EF1010E21F815E0002AD1D1EF
:1053D000009D05F1010504F10404092DA2D1029CF0
:1053E000621E029240F0F7800399087800F10100F4
:1053F000C3B20B700B2B03D14FF000040C7002E012
:10540000002B40F0E58041F2E872C2F2010211681F
:1054100091B16FEA01003B6803403B6041F2A07527
:10542000C2F201052C682040286041F2E871C2F206
:1054300001014FF000020A6041F2E870C2F201007F
:10544000436893B16FEA03057C682C407C6041F2AD
:10545000A072C2F2010251680D40556041F2E8703D
:10546000C2F201004FF00003436041F2E875C2F25E
:105470000105AC6894B16FEA0400BA680240BA60F2
:1054800041F2A073C2F2010399680840986041F2AA
:10549000E875C2F201054FF00004AC6041F2E8701B
:1054A000C2F20100C26892B16FEA0203F9681940C2
:1054B000F96041F2A075C2F20105EC682340EB608F
:1054C00041F2E870C2F201004FF00002C26041F206
:1054D000E873C2F20103196991B16FEA01053C69F1
:1054E0002C403C6141F2A070C2F2010002691540FB
:1054F000056141F2E873C2F201034FF00001196146
:1055000041F2E875C2F201056C6994B16FEA0400DA
:105510007A6902407A6141F2A073C2F201035969CB
:105520000840586141F2E875C2F201054FF00004ED
:105530006C6141F2E870C2F20100826992B16FEAD7
:105540000203B9691940B96141F2A075C2F20105BF
:10555000AC692340AB6141F2E870C2F201004FF048
:105560000002826141F2E873C2F20103D96991B18C
:105570006FEA0105FC692C40FC6141F2A070C2F2A7
:105580000100C2691540C56141F2E873C2F201032E
:105590004FF00001D96141F2E875C2F201052C6AB1
:1055A00094B16FEA04003A6A02403A6241F2A07391
:1055B000C2F20103196A0840186241F2E875C2F2AA
:1055C00001054FF000042C624FF4FA70029002E0E3
:1055D0004FF4FA7502954FF0010001F03DF9326881
:1055E000002A3FF499AE07E04FF4FA75029541F2B4
:1055F0009C74C2F2010403944FF00004254691E626
:1056000010B54FF0000441F60C03C2F201031C6018
:1056100041F2A070C2F2010021464FF00902FAF7F0
:105620007FFD41F2C470C2F2010021464FF0090231
:10563000FAF776FD41F2E870C2F2010021464FF020
:105640000902FAF76DFD41F27860C2F201002146CD
:105650004FF00902FAF764FD41F26060C2F2010006
:1056600021464FF0180211F0D3FD41F29C70C2F2B6
:105670000100047010BD00BF70B549F65073C0F64C
:1056800003031B5C49F61072C0F6030252F8202097
:1056900041F60C00C2F20100046841F2C475C2F286
:1056A000010555F82300104206D104F1010641F628
:1056B0000C05C2F201052E6049B141F2A071C2F29F
:1056C000010151F82350154341F8235009E041F2FC
:1056D000A071C2F2010151F8235025EA020541F8F8
:1056E0002350104341F2C471C2F2010141F823007A
:1056F00041F2E871C2F2010151F8230020EA0202EE
:1057000041F8232034B941F25C63C2F20103186806
:1057100000F00CFF70BD00BF30B449F65073C0F606
:1057200003031B5C49F61072C0F6030252F82020F6
:1057300041F2C470C2F2010050F82300104229D097
:1057400041F60C04C2F20104256805F1010525604B
:1057500071B141F2E871C2F2010151F823401443E2
:1057600041F8234041F29C71C2F20101097889B9E4
:105770006FEA020241F2A071C2F2010151F8234026
:10578000144041F82340024041F2C470C2F20100CB
:1057900040F8232030BC704730B4034641F6A802DD
:1057A000C2F2010252E8000F00F1010042E80004D9
:1057B000012CF7D041F26060C2F2010030F81320F2
:1057C00039B141F26061C2F201014FF0000421F8E9
:1057D000134041F6A803C2F2010353E8004FA4F1BD
:1057E000010443E80045012DF7D053E8004FB4F120
:1057F000004F0DD14FF0000443E80045012DF4D0D7
:105800004EF60450CEF20000016841F08051016074
:10581000BFF32F8F104630BC704700BF41F29C731E
:10582000C2F201031878D0F1010038BF00207047A0
:105830002DE9F84FDFF834814B4FC8EB07004FEAF2
:10584000D00707F101074FF0000540F2982AC0F693
:10585000000A40F25839C0F6000931E044464FF0E2
:1058600000066FEA060B0BEB070101F0010B58F87D
:10587000043CAB4229D135E054F8043CAB4205D19D
:1058800054F8080C8047FBF77BFE0BE0FF2B09D98F
:10589000FF2D07D154F8040C4FF0070154F8082CE1
:1058A00000F09CFF06F1010604F1080454F8041C02
:1058B000A94240D14CE005F10105B5F5807F02D049
:1058C000CA45CBD3F7E7BDE8F88FFF2B0FD9FF2DE3
:1058D0000DD158F8040C4FF0070158F8082C00F0CF
:1058E0007DFF04E058F8082C9047FBF749FE06F1CD
:1058F000010604F10804BE42DDD0BBF1000FBBD0AD
:1059000054F8040CA8420AD0FF280DD9FF2D0BD162
:105910004FF0070154F8082C00F060FF04E054F841
:10592000081C8847FBF72CFE06F1010604F1080469
:10593000BE42A1D1BFE7FF290FD9FF2D0DD154F8E9
:10594000040C4FF0070154F8082C00F047FF04E066
:1059500054F8082C9047FBF713FE06F1010604F1FA
:105960000804BE4288D1A6E75F030008A002000831
:10597000027841F67503C2F201031B789A4206D3FE
:105980004FF000020270087800F1010008700A78F8
:1059900041F67603C2F201031878824224BF002048
:1059A0000870704710B5A0F10803052B3DD8DFE85B
:1059B00003F01F3C2C3C038341F61400C2F20100AB
:1059C0004FF020014FF0540211F022FC41F6680024
:1059D000C2F201004FF0FF314FF00C0211F018FC41
:1059E00041F67C00C2F20100026802F1010202608D
:1059F0004FF0000141F61003C2F20103197041F6A5
:105A00001100C2F20100017056E041F61001C2F22D
:105A100001014FF000030B7041F61100C2F20100CA
:105A2000027802F1010202703CE041F61002C2F27B
:105A30000102127841F61101C2F201010B7841F620
:105A40007501C2F20101097801FB032341F614013B
:105A5000C2F20101C95C81421DD041F61404C2F2B8
:105A60000104E0544FEA531041F66801C2F201010B
:105A700003F01F034FF0010404FA03F351F8204030
:105A80001C4341F8204041F67C00C2F2010001684D
:105A900001F10101016002F1010241F61003C2F2BD
:105AA00001031A7041F61000C2F2010041F6110123
:105AB000C2F20101FFF75CFF4FF0000010BD00BF14
:105AC00070B4039D049C064628B141F67800C2F2EA
:105AD00001000078307029B141F68000C2F2010067
:105AE000007808702AB141F67401C2F20101087809
:105AF00010702BB141F68102C2F2010211781970C7
:105B00002DB141F61003C2F20103187828702CB1B0
:105B100041F61102C2F201021178217070BC704787
:105B200006281DD8002808BF052041F67803C2F2D8
:105B3000010318704AF2B813C0F6030313F81010EB
:105B400041F67502C2F20102117003EB4000417888
:105B500041F67603C2F2010319704FF0010070475D
:105B60004FF00000704700BF08B541F68003C2F255
:105B700001034FF001021A704FF00500FFF7D0FF4C
:105B80004FF00C004FF00001FFF70CFF08BD00BF05
:105B900008B541F61002C2F20102107041F611037D
:105BA000C2F20103197010461946FFF7E1FE08BD65
:105BB000034628B141F67500C2F201000078187062
:105BC00029B141F67603C2F20103187808702AB1B0
:105BD00041F67C01C2F201010B68136041F614002A
:105BE000C2F20100704700BF2DE9F00141F6140731
:105BF000C2F201073F1853284BD8002A49D03B4630
:105C000007F1010702F1FF3257FA82F74FF0000661
:105C100041F66804C2F201044FF001056FEA030C7B
:105C20000CEB070202EA050C13F8018B01F1FF31BE
:105C300011F8012F90452FD13DE013F801CB01F170
:105C4000010049788C450ED003F8011C4FEA52112F
:105C500002F01F0605FA06FC54F821604CEA06061D
:105C600044F821602E4602F10102D2B2542A07D034
:105C700013F801CB00F101014078844542D150E096
:105C80003EB141F67C03C2F20103196801F1010142
:105C90001960BDE8F001704703F8012C4FEA501677
:105CA00000F01F0805FA08F854F8262048EA020216
:105CB00044F826202E4600F10100C2B2542ADFD05B
:105CC000BB42DDD0BCF1000FB7D013F801CB11F807
:105CD000010F84450ED003F8010C4FEA521002F078
:105CE0001F0605FA06FC54F820604CEA060644F844
:105CF00020602E4602F10102D2B2542AC0D0BB422B
:105D00009BD1BDE703F8010C4FEA521002F01F06C9
:105D100005FA06FC54F820604CEA060644F82060B8
:105D20002E4602F10102D2B2542AA9D0BB4284D13C
:105D3000A6E700BF003018BF012041F68003C2F281
:105D400001031870003118BF012141F67400C2F23E
:105D500001000170003218BF012241F68103C2F236
:105D600001031A70704700BF41F67703C2F20103C6
:105D70004FF000021A7070474FF05400704700BF98
:105D800041F67703C2F201034FF001021A70704727
:105D9000034628B10868834214BF002001207047E1
:105DA0004FF00000704700BF10B441F6A803C2F2E4
:105DB000010353E8002F02F1010243E80021012909
:105DC000F7D00468C4B16268824202D1926862600E
:105DD00002E04368816899602368834202D15B686E
:105DE000236002E0826841685160A26802F1FF31DD
:105DF000A1604FF00004046041F6A803C2F2010361
:105E000053E8002FA2F1010243E80024012CF7D04F
:105E100053E8002FB2F1004F0DD14FF0000243E8DC
:105E20000024012CF4D04EF60450CEF2000001689C
:105E300041F080510160BFF32F8F10BC704700BF4D
:105E400038B504460D464FF000014FF0100211F036
:105E5000DFF9E56038BD00BFF8B504460F46C668F7
:105E60008D192946FFF794FF00283CD141F6A8037D
:105E7000C2F2010353E8002F02F1010243E80021BE
:105E80000129F7D04FF0000068606168A96001B196
:105E90004D60226802B925606560BC51A36803F1BA
:105EA0000103A36041F6A803C2F2010353E8002FE7
:105EB000A2F1010243E80024012CF7D053E8002F9F
:105EC000B2F1004F0DD14FF0000243E80024012C45
:105ED000F4D04EF60450CEF20000016841F080513B
:105EE0000160BFF32F8FF8BD2DE9F04104468846CD
:105EF000C6688D199719C2B941F6A803C2F2010309
:105F000053E8002F02F1010243E800210129F7D0F4
:105F100002686A6005604FF00000A860616809B916
:105F2000656020E06B689D601DE03946FFF730FF3B
:105F300000283FD02846FFF737FF41F6A803C2F2FA
:105F4000010353E8002F02F1010243E80021012977
:105F5000F7D0B868A8606F60BD602168B9420EBF15
:105F60002560A9684D6048F80640A26802F1010268
:105F7000A26041F6A803C2F2010353E8002FA2F188
:105F8000010243E80024012CF7D053E8002FB2F1BE
:105F9000004F0DD14FF0000243E80024012CF4D053
:105FA0004EF60450CEF20000016841F080510160CD
:105FB000BFF32F8FBDE8F081C368C918486808B1E6
:105FC000C01A70474FF00000704700BF036813B15C
:105FD000C068181A70474FF00000704708B5C368D2
:105FE000C918FFF7D5FE08BD08B5C0680818FFF747
:105FF000DBFE08BD08B541F68400C2F201004FF097
:106000001C01FFF71DFF08BD70B5054600F108062D
:106010003046FFF7DBFF0446686050B1304621464A
:10602000FFF7E2FF4FF00100A861204600F07EFA82
:1060300070BD4FF00003AB6170BD00BF38B50446C2
:106040000D464FF000014FF0280211F0E1F8204614
:1060500040F8085B4FF01C01FFF7F2FE41F68400A8
:10606000C2F201002146FFF7F7FE38BD2DE9F041ED
:106070000746884642F24853C2F2010318680028D6
:1060800000F0FE8041F6A804C2F2010454E8002F9B
:1060900002F1010244E800210129F7D0796831B109
:1060A00042F24852C2F20102136899422ED142F2E2
:1060B0004850C2F2010004687C60B96901F1010135
:1060C000B96141F6A803C2F2010353E8002FA2F11F
:1060D000010243E80024012CF7D053E8002FB2F16D
:1060E000004F0DD14FF0000243E80024012CF4D002
:1060F0004EF60450CEF20000016841F0805101607C
:10610000BFF32F8F4FF00100BDE8F081B8F1FF3FE2
:1061100024D141F6A803C2F2010353E8002FA2F1F3
:10612000010243E80024012CF7D053E8002FB2F11C
:10613000004F0DD14FF0000243E80024012CF4D0B1
:106140004EF60450CEF20000016841F0805101602B
:10615000BFF32F8F4FF00000BDE8F08107F1080575
:106160002846FFF733FF0246F0B142F24856C2F22A
:106170000106306892F8294090F829108C4208D91D
:1061800012E0336892F8290093F82940A04204D91C
:106190000AE042F24856C2F2010628461146FFF7CD
:1061A0000BFF02460028ECD1284642F24851C2F2C9
:1061B00001010968FFF798FE41F6A806C2F2010640
:1061C00056E8002FA2F1010246E80024012CF7D086
:1061D00056E8002FB2F1004F0DD14FF0000246E813
:1061E0000024012CF4D04EF60450CEF200000168D9
:1061F00041F080510160BFF32F8FB8F1000F04D040
:1062000008EB880000F028FB01E000F05DF941F6A2
:10621000A804C2F2010454E8003F03F1010344E87A
:106220000032012AF7D042F24856C2F2010628464F
:106230003168FFF7D9FE54E8003FA3F1010344E8B9
:106240000032012AF7D054E8003FB3F1004F0DD1DE
:106250004FF0000344E80032012AF4D04EF6045017
:10626000CEF20000016841F080510160BFF32F8F32
:1062700078683268904214BF00200120BDE8F081A8
:106280004FF00100BDE8F08110B5044642F24853DA
:10629000C2F201031868002860D06268904201D001
:1062A000F9F72EFF41F6A803C2F2010353E8002FCD
:1062B00002F1010243E800210129F7D0A16901F1AF
:1062C000FF30A06118B341F6A803C2F2010353E8FE
:1062D000002FA2F1010243E80024012CF7D053E87B
:1062E000002FB2F1004F0DD14FF0000243E800241F
:1062F000012CF4D04EF60450CEF20000016841F0BB
:1063000080510160BFF32F8F4FF0000010BD204679
:10631000FFF77AFE41F6A803C2F2010353E8002F0B
:10632000A2F1010243E80024012CF7D053E8002F2A
:10633000B2F1004F0DD14FF0000243E80024012CD0
:10634000F4D04EF60450CEF20000016841F08051C6
:106350000160BFF32F8F4FF0010010BD4FF001001F
:1063600010BD00BFF8B5054641F6A803C2F201030F
:1063700053E8002F02F1010243E800210129F7D080
:1063800041F68400C2F20100FFF720FE0446E0B1AE
:1063900041F68407C2F201076068A84203D1204693
:1063A000FFF732FE0AE004F1080630462946FFF7FF
:1063B00015FE18B130462946FFF716FE384621462D
:1063C000FFF7FAFD04460028E6D141F6A803C2F221
:1063D000010353E8002FA2F1010243E80024012C3D
:1063E000F7D053E8002FB2F1004F0DD14FF000026B
:1063F00043E80024012CF4D04EF60450CEF2000005
:10640000016841F080510160BFF32F8FF8BD00BFDC
:1064100008B54AF2C413C0F60303195C012906D07B
:1064200011B102290BD105E0FDF7FEFA08BD02F01B
:1064300001F908BDF9F764FE4FF0000008BD4FF008
:10644000000008BD4EF60453CEF200031A6842F075
:1064500080501860704700BF4FF0010280F828207C
:1064600041F6A403C2F2010390F8291002FA01F2E6
:10647000188802431A80704710B441F6A003C2F294
:1064800001031A68C2B1904213D104E088420FD1CF
:1064900002F1140203E041F6A002C2F201024369D4
:1064A0001BB19C698169611899614369136003E0BC
:1064B0000A4651690029E9D14FF0000282614FF08C
:1064C000FF31416110BC704710B5F9F76FFE04460B
:1064D00042F24853C2F20103186890F82820032AB8
:1064E0001BD0F9F763FE42F24853C2F20103196868
:1064F0004FF0000281F8282091F82920096941F61F
:106500009413C2F2010343F82210F9F759FE204612
:10651000F9F756FEFFF796FF10BD4FF0020180F825
:1065200028102046F9F74CFE10BD00BF38B50446D0
:1065300090B3036883B3F9F739FE054694F8280051
:1065400010BB2046FFF788FF42F24851C2F201011A
:106550000B6843B194F8292093F8290020F0010139
:10656000531A002B15DA41F6A802C2F20102106894
:1065700038B140F0004141F6A803C2F201031960AE
:1065800007E0FFF75FFF04E0022804BF032084F860
:1065900028002846F9F714FE38BD00BF2DE9F04F5A
:1065A00085B006460F46934698460F9DDDF840900D
:1065B000F9F7FCFD824641F6EC03C2F201031968CB
:1065C000504881420FD240F20002C2F2020252F859
:1065D0002C4C54B14C4B1C468B4207D953F82C0918
:1065E0000028F8D102E0474C00E0464CA14206D119
:1065F000A1F12C0141F6EC02C2F201021160204629
:106600004FF000014FF02C0210F002FE4FF0FF316E
:1066100061611EB94AF2C826C0F603062660B8F1C9
:10662000000F08D00E9B042B08D9184600F1030078
:106630004FEA900604E04FF0000601E04FF000063C
:106640000DBB43F24C09C2F2010941F69405C2F2B6
:106650000105296846F6B920C0F602000090CDF881
:106660000480029648464FF000025B46FAF7D6F8DF
:106670002A68A260E0604FEA800153182B60C1EBEA
:106680000900606020E028464FF0FF314A46F9F7E4
:1066900047FD4AF2ED52CDF6CE622A60E56005EB89
:1066A0008905656046F6B921C0F602010091CDF872
:1066B00004800296284629464FF001025B46FAF70D
:1066C000ADF8A5EB800363606FEA0702C2F3C01167
:1066D00001EB470707F0FF0784F8297041F6AC0388
:1066E000C2F2010353F82700206143F827405046C7
:1066F000F9F766FD2046FFF719FF204605B0BDE813
:10670000F08F00BFD4FF0120A8FF012030B585B075
:106710004FF0000142F24853C2F201031960284CC5
:1067200040F20005C2F202052A1B20464FEAA202EF
:10673000F9F7F6FC41F69400C2F201000460A5F1FD
:106740002C0541F6EC01C2F201010D6042F64C034A
:10675000C2F201034FF0B504CBF26B141C6003F1DD
:106760004C004FF0FF3243F8042F43F8042F43F856
:10677000042F8342F9D14FF00004009441F6F00158
:10678000C2F2010101914FF0280302934AF2D42092
:10679000C0F603004FF0070146F63902C0F60202C8
:1067A0002346FFF7FBFE41F69012C2F20102106091
:1067B00041F6AC00C2F20100C46305B030BD00BFB9
:1067C0005030012010B584B0069C00944FF00004B6
:1067D00001940294FFF7E2FE04B010BD00B585B04D
:1067E0004FF00003009301930293FFF7D7FE05B02B
:1067F00000BD00BF38B542F24853C2F20103186829
:10680000C0B1F9F7D3FC054642F24854C2F2010484
:106810002068FFF721FE216891F82920086941F6D8
:106820009413C2F2010343F822002846F9F7C8FC8A
:10683000FFF708FE38BD00BF38B542F24855C2F236
:10684000010541F6AC04C2F201042B6822681A610A
:10685000FFF7D0FFF9E700BF38B542F24853C2F264
:1068600001031968002900F0918020B9FFF7C2FFE9
:106870004FF001029AE0B0F1FF3F04D1FFF724FE90
:106880004FF0000292E041F6A804C2F2010454E87D
:10689000002F02F1010244E800210129F7D041F65E
:1068A000A002C2F201021568002D7AD0AB699842AD
:1068B0006FD3C01A05F114016D691DB1AB69834234
:1068C000F7D96AE042F24855C2F201052B68986197
:1068D000086858611846F9F717FC41F6A804C2F297
:1068E000010454E8003FA3F1010344E80032012A07
:1068F000F7D054E8003FB3F1004F0DD14FF0000343
:1069000044E80032012AF4D04EF60450CEF20000E2
:10691000016841F080510160BFF32F8FFFF7D4FD74
:1069200054E8003F03F1010344E80032012AF7D0A4
:1069300028684169B1F1FF3F04D0FFF79DFD4FF09A
:10694000000201E04FF0010241F6A803C2F2010388
:1069500053E8004FA4F1010443E80045012DF7D0AE
:1069600053E8004FB4F1004F0DD14FF0000443E85D
:106970000045012DF4D04EF60450CEF2000001681F
:1069800041F080510160BFF32F8F0FE04FF0010203
:106990000CE041F6A001C2F20101AC69221AAA6121
:1069A00090E741F6A001C2F201018BE7104638BD25
:1069B000F8B5044600287AD0F9F7F8FB064641F608
:1069C000EC03C2F2010319683948814211D240F246
:1069D0000002C2F2020252F81C5CA54263D0354BA1
:1069E0001D468B4205D9A3F12C03D86BA042F7D1E9
:1069F0005AE094F8293041F6AC02C2F2010252F892
:106A00002300A04206D1016941F6AC02C2F20102A4
:106A100042F823102046FFF72FFD2046FFF7A2FC87
:106A200094F82900236941F69411C2F2010141F85A
:106A3000203042F24852C2F201021068A04229D02E
:106A4000A06838B3E76800EB870541F69407C2F207
:106A500001073B685A1B29464FEAA2024FF0000388
:106A6000FBF7D6FDE1683868A0EB81033B6041F697
:106A7000EC02C2F2010211680D4B99420AD29A68E7
:106A8000954203D8E068A2EB80029A60A3F12C0340
:106A90008B42F4D84FF00001216084F82810304672
:106AA000F9F78EFBF8BD024D21692961A1E7F8BD18
:106AB000D4FF0120A8FF012000BFF04772B642F2C8
:106AC0004854C2F201042068FFF772FF4FF0000340
:106AD0002360F9F7F3FE00BF41F6A003C2F2010301
:106AE000196849B1886950B100F1FF328A61D2F169
:106AF000010038BF002070474FF0000070474FF092
:106B00000000704770B541F6A003C2F201031C6893
:106B1000A4B1A06990B941F6A005C2F201054FF0F9
:106B2000FF3660692946F9F7EFFA66612046FFF7FC
:106B3000FDFC2C6814B1A1690029F2D070BD00BF22
:106B4000F0B472B641F6A403C2F201031C882CB95A
:106B500041F69013C2F2010318685FE04AF2C81CC4
:106B6000C0F6030C41F69415C2F2010541F6AC06DD
:106B7000C2F20106C4F1000323401A0A1ABF1CF82E
:106B8000021008311CF8031011F0010F0AD141F076
:106B9000010055F8200038B190F82820012A38D893
:106BA0001F4602E01F4600E01F4655F82120B2B103
:106BB00092F828307BB141F6A400C2F201000480B3
:106BC00010462BE090F8283033B141F6A402C2F20F
:106BD0000102148022E0104600690028F2D156F824
:106BE0002100824207D1BC43C4D141F6A401C2F2C4
:106BF00001010C80ACE745F8210011F0010FD4D160
:106C000014EA4703D1D04FEA4707BFB241F0010170
:106C1000CBE741F6A401C2F201010C8062B6F0BCE0
:106C2000704700BF70B542F24853C2F201031B68BF
:106C300083420FD193F82820012A9CBF022283F8B7
:106C4000282093F8291041F69410C2F2010040F870
:106C5000213070BD41F69802C2F20102136042F287
:106C60004851C2F20101086090F8292041F69413BE
:106C7000C2F2010343F8220090F8281001299CBFBA
:106C8000022180F828108268AAB9C1684AF2ED533F
:106C9000CDF6CE630868984201D0F9F731FA42F296
:106CA0004852C2F2010211684868CB6898427ED20D
:106CB000F9F726FA70BD41F69C03C2F201031B6886
:106CC000984274D093B3586843F24C04C2F2010462
:106CD000251A4FEAA501D96042F64C02C2F2010220
:106CE00090420AD34FF0B503CBF26B1342F64C003F
:106CF000C2F2010004689C4201D0F9F701FA41F6A2
:106D00009C05C2F201052A6841F69404C2F201040E
:106D100020685168D2684FF00003FBF779FC2968BE
:106D200023688B60C86803EB8002226042F24851FE
:106D3000C2F201010B6841F69C00C2F2010003603F
:106D4000DA68002A33D0586899684FF00103FBF7DE
:106D50005FFC42F24856C2F201063568A868EC684A
:106D600000EB840441F69406C2F201063268131B5C
:106D700021464FEAA3024FF00003FBF749FCE96804
:106D80003068A0EB8102326041F6EC03C2F20103ED
:106D90001968074B99420AD29A68944203D8E86866
:106DA000A2EB80029A60A3F12C038B42F4D870BD51
:106DB000D4FF012000B585B041F63030C2F20100A9
:106DC0004FF00001FFF73CF841F6D810C2F2010085
:106DD0004FF00001FFF734F84FF00003009341F645
:106DE000F012C2F2010201924FF0500002904AF2FA
:106DF000DC20C0F60300194647F20912C0F6020271
:106E0000FFF7CCFB41F6D413C2F20103186005B0C2
:106E100000BD00BF08B5FFF7D9F8034648B1C06808
:106E200050B100F1FF31D960D1F1010038BF00202D
:106E300008BD4FF0000008BD4FF0000008BD00BFC6
:106E400070B505460E46144641F6A803C2F201038A
:106E500053E8002F02F1010243E800210129F7D095
:106E6000FFF7B4F80246002839D0C06884422DD319
:106E7000241A28461146FFF79FF8024600282ED014
:106E8000C068A042F4D921E041F6A803C2F2010390
:106E900053E8002FA2F1010243E80024012CF7D0AF
:106EA00053E8002FB2F1004F0DD14FF0000243E83C
:106EB0000024012CF4D04EF60450CEF200000168FC
:106EC00041F080510160BFF32F8F70BDF460D16835
:106ED0000B1BD36028463146FFF706F8D4E7F46071
:106EE00028463146FEF7B8FFCEE700BFF8B50646A4
:106EF000FFF76CF80446F8B1C368EBB93046214699
:106F0000FFF75AF80546F9F751F90746304621468A
:106F1000FFF76AF83846F9F753F922691AB1304693
:106F20002146FFF78DFF04F11400FDF7B3FE1DB1FC
:106F30002C46E8680028E1D0F8BD00BF08B541F64E
:106F4000EC13C2F201031A6802F101021A6041F661
:106F5000D810C2F20100FFF75DFF28B141F6D8104A
:106F6000C2F20100FFF7C2FF08BD00BF08B501462D
:106F700041F63030C2F20100FFF730F820B141F69F
:106F80003030C2F2010008BD41F6D810C2F2010053
:106F900008BD00BF70B5044641F6A803C2F2010364
:106FA00053E8002F02F1010243E800210129F7D044
:106FB000FFF7DCFF05462146FFF710F8002845D013
:106FC00041F6A800C2F2010050E8002F02F10102D0
:106FD00040E800210129F7D028462146FEF7ECFFC2
:106FE00018B1C168E2688B18C360F9F7DFF806468C
:106FF00028462146FEF7F8FF3046F9F7E1F84FF052
:10700000FF35E56041F6A803C2F2010353E8002F03
:10701000A2F1010243E80025012DF7D053E8002F2B
:10702000B2F1004F0DD14FF0000243E80025012DD1
:10703000F4D04EF60450CEF20000016841F08051C9
:107040000160BFF32F8F4FF0010501E04FF0000505
:1070500004F11400FDF718FE41F6A803C2F2010383
:1070600053E8002FA2F1010243E80024012CF7D0DD
:1070700053E8002FB2F1004F0DD14FF0000243E86A
:107080000024012CF4D04EF60450CEF2000001682A
:1070900041F080510160BFF32F8F284670BD00BFC3
:1070A0002DE9F04105460F4614469846FFF772FF5A
:1070B000064694B19DF82030002B14BF20460020D6
:1070C000286105F114004146069A079BFDF7C2FDB1
:1070D000384629462246FFF7B3FE3046BDE8F08128
:1070E00070B584B00E4615460093089C01949DF837
:1070F0002430029341F63031C2F2010132462B4670
:10710000FFF7CEFF04B070BD00B583B04FF00003B1
:1071100000934FF00100019041F64030C2F20100AF
:1071200041F288314FF0FF0246F63D73C0F602038C
:10713000FFF7D6FF41F63034C2F20104FFF7E2FC5C
:107140002046FFF7D3FEFFF7BFF9F7E741F6E81354
:10715000C2F2010318681A689042FBD1704700BF61
:1071600010B541F6E813C2F201031A6802F10102F8
:107170001A60FFF7B1FC044641F63030C2F201005C
:10718000FFF748FE204310F0FF0F06D041F6D41061
:10719000C2F201000068FFF7C9F910BD08B54AF254
:1071A0001030C0F603004FF0060147F2D952C0F686
:1071B0000202FFF713FB41F66833C2F201031860C5
:1071C00008BD00BF38B504460D4641F6B433C2F2DF
:1071D0000103586AA0420AD041F6B431C2F201015B
:1071E0004C620A681AB115B14948FDF753FD41F6E2
:1071F000B433C2F20103186F84420AD041F6B431AD
:10720000C2F201010C67CA6C1AB115B14148FDF711
:1072100041FD41F6B433C2F20103D3F8BC0084420D
:107220000CD041F6B431C2F20101C1F8BC40D1F832
:1072300098201AB115B13848FDF72CFD41F6B4334A
:10724000C2F20103D3F8080184420CD041F6B431F4
:10725000C2F20101C1F80841D1F8E4201AB115B118
:107260002E48FDF717FD41F6B433C2F20103D3F8FF
:10727000540184420CD041F6B431C2F20101C1F88C
:107280005441D1F830211AB115B12548FDF702FD5E
:1072900041F6B433C2F20103D3F8A00184420CD00A
:1072A00041F6B431C2F20101C1F8A041D1F87C210C
:1072B0001AB115B11B48FDF7EDFC41F6B433C2F22B
:1072C0000103D3F8EC0184420CD041F6B431C2F290
:1072D0000101C1F8EC41D1F8C8211AB115B1124829
:1072E000FDF7D8FC41F6B433C2F20103D3F83802FB
:1072F000A0420CD041F6B431C2F20101C1F83842CB
:10730000D1F814221AB115B10848FDF7C3FC38BDF5
:10731000C41B0120101C01205C1C0120A81C0120A2
:10732000F41C0120401D01208C1D0120D81D0120CE
:107330002DE9F04707460D4691460898DDF828806C
:107340000C683E68D8F800108A19944202D80219D5
:10735000964203D304192C60BDE8F087341B061B4A
:10736000B14234BF8A46B246099931B1D9F800001A
:107370000818191952460FF027FFD8F80030CAEB49
:107380000302C8F800203E6806EB0A013960D9F80C
:10739000000000EB0A03C9F800302E68A419544419
:1073A0002C60BDE8F08700BF70B584B09CF8196010
:1073B000157A947B4FF007038CF810304FF00502DC
:1073C0008CF8112006F00F0260F3C7128CF812201F
:1073D0004FF0000065F301008CF813004FF000023D
:1073E00061F30A02ACF814208CF81640DCF80C109B
:1073F0000093DCF804300193CDF808C001F10400DB
:107400000CF108020CF11003FFF792FF04B070BDFD
:107410002DE9F04F8FB00746059114464FF0000359
:107420000793136012896068131A8B4238BF059363
:107430000599002900F0AA8041F6AC35C2F2010599
:107440002D6815B34FEAC5054FF000024FF0FF015C
:10745000134641F62C60C2F20100A5F10806C6F3FE
:10746000C00E1658F6798E4240F0958096E0165878
:10747000F6798E421CBF0133314602F1080286586C
:10748000F6798E4240F09F80A0E04FF0000303EBBE
:1074900043024FEAC20000F1100008904FF48071DF
:1074A000ADF824104FF00402ADF826208DF82830F6
:1074B0000DF129004FF000014FF007020FF0A8FE78
:1074C00004F1040B04944FF010030093019705A8F6
:1074D00002905846214607AA08ABFFF729FF0599F5
:1074E000002951D04FF001028DF821200DF132001A
:1074F0004FF000014FF006020FF08AFE41F6AC3368
:10750000C2F20103186800283ED04FF0FF014FF08F
:10751000000441F62C69C2F201094AF22038C0F693
:10752000030841F6AC3AC2F2010A59F83450ED7939
:107530008D4223D08DF820404FEA05160DF1220030
:1075400008EB06014FF008020FF03EFE06F10801BD
:107550000DF12A0041444FF008020FF035FE4FF0C4
:1075600018020092019705AB02935846049907AAA6
:1075700008ABFFF7DDFE059830B1294604F10104A0
:10758000DAF80020A242D0D8079801E04FF0FF308F
:107590000FB0BDE8F08F03F10103314602F108029C
:1075A000AA423FF474AFBEF1000F3FF460AF16582B
:1075B000F6798E421CBF0133314602F10802AA421D
:1075C0007FF455AF63E703F10103314602F108028E
:1075D000AA427FF44CAF5AE72DE9F0414FF0010089
:1075E000FDF726FA4AF20030C0F60300FDF7A4F8D2
:1075F00041F66433C2F201034FF001021A7041F602
:107600009830C2F20100016841B941F69834C2F2E3
:107610000104FEF759FF2568002DFAD041F6A9377D
:10762000C2F2010741F66434C2F2010441F6A83601
:10763000C2F2010641F61565C2F2010541F628685D
:10764000C2F201083B783BB14FF000023A704FF0B4
:1076500002002070FDF7E6F9317859B14FF00003D0
:107660003370227862F07F0020704FF001000146F5
:10767000FFF7A8FD297851B14FF00000287023785A
:1076800003F07F0222704FF00101FFF79BFD98F895
:10769000000010B9FEF718FFD4E741F66431C2F2DA
:1076A00001014FF002030B704FF00000FDF7C0F92D
:1076B000BDE8F08108B541F69833C2F201031860C5
:1076C00041F66830C2F201000068FEF72FFF08BDE6
:1076D00070B505460E4641F6B033C2F20103186894
:1076E000032801D9F8F70CFD41F6B032C2F20102CD
:1076F000116841F67834C2F2010444F8316004EBB9
:10770000C104656001F10101116070BD70B50546ED
:107710000C461646032801D9F8F7F2FC41F62C6313
:10772000C2F2010353F8350008B1F8F7E9FC41F65D
:107730002C61C2F2010141F8354001EBC5056E60D4
:1077400041F6AC33C2F201031A6802F101021A6079
:10775000206930B1FCF7F0FF04F10404206900282F
:10776000F8D170BD08B541F6B433C2F2010319680F
:1077700081425AD041F6B432C2F20102D36C834244
:1077800034D041F6B431C2F20101D1F898208242DE
:107790002FD041F6B433C2F20103D3F8E410814292
:1077A0002AD041F6B432C2F20102D2F8303183421B
:1077B00025D041F6B431C2F20101D1F87C218242D8
:1077C00020D041F6B433C2F20103D3F8C81181428C
:1077D0001BD041F6B432C2F20102D2F81432834215
:1077E00016D0F8F78DFC4FF0080013E04FF00100C1
:1077F00010E04FF002000DE04FF003000AE04FF000
:10780000040007E04FF0050004E04FF0060001E03F
:107810004FF0070041F6B431C2F201014FF04C02C3
:1078200002FB001090F8200008BD4FF00000F1E7C7
:107830002DE9F04F8FB0089007910A924FF00003A6
:1078400009931360546813891B1B8B4238BF07933D
:107850000799002900F04A81082C69D841F6AC3418
:10786000C2F20104D4F800E041F6B035C2F20105DD
:107870002E680EEBCE0707EBC60404F109044FF0A7
:10788000000141F62C67C2F20107CB598BB1DD68CC
:10789000641903F110051B695BB15E890EB104F137
:1078A00007049B890BB104F1070455F8043F002B32
:1078B000F3D101F108012029E7D141F69831C2F254
:1078C00001010D682F7E6E7EEB8A03F10103C3F385
:1078D00047054FF000010C914FF009038DF82C3053
:1078E0004FF002018DF82D10ADF82E408DF830E0EC
:1078F0004FF001018DF831104FF0000167F3451191
:1079000066F3861161F07F018DF833108DF83450E5
:107910000093019007A8029002F10400114609AA01
:107920000BABFFF705FD079A002A00F0DD80E0E0D1
:107930004FF009001060DCE05BF83640002C00F0EE
:10794000CE80059D286800284BD07A68B2420CD0C2
:107950004FF0000310F0010F3ED1DFE007EBC30250
:107960005268B24240F0E38001E04FF0000357F864
:107970003300D2B290F8048090F805C090F806E089
:10798000C579016819B143F01000C3B201E04FF0AE
:1079900000034FF008008DF82C004FF00B018DF81C
:1079A0002D108DF82E208DF82F808DF830C08DF899
:1079B00031E08DF832508DF833300A990090089AF2
:1079C000019207AB029301F1040009AA0BABFFF788
:1079D000AFFC079828B987E003F101052B468542E3
:1079E000BCD104F1100523697BB129464FF0000298
:1079F000588908B102F101029B890BB102F1010221
:107A000051F8043F002BF3D101E04FF000025FFA80
:107A100086FCD2B294F804E06079A17923681BB1A6
:107A200046F02003DBB201E04FF000038DF82CA0FC
:107A30004FF004088DF82D808DF82EC04FF0000C0B
:107A40008DF82FC08DF830208DF831E08DF83200A0
:107A50008DF833108DF834300A99CDF800A0089ACB
:107A6000019207A8029001EB080009AA0BABFFF7EF
:107A70005FFC0799002937D0A3686BB10A99E268C7
:107A800000920898019007AA029201EB080009AA47
:107A9000FFF74EFC079B3BB3246904B34FF001088A
:107AA0004FF000092046FFF75DFE8DF83500618933
:107AB00039B10DF11C0C40462246FFF775FC0799C1
:107AC00091B1A18939B10DF11C0C48462246FFF74E
:107AD0006BFC079840B155F8044F002CE2D106F139
:107AE0000106042E7FF428AF099814E04FF0FF3010
:107AF00011E04FF0000641F62C6BC2F2010B41F68B
:107B0000B034C2F2010405944FF0090A41F6783707
:107B1000C2F2010710E70FB0BDE8F08F03F10103D7
:107B200007EBC3014A68B2427FF456AF1FE705F185
:107B3000010307EBC3014A68B2427FF44DAF16E779
:107B400008B541F61863C2F201031A5C41F6B4317C
:107B5000C2F201014FF04C0000FB0210436AD3F166
:107B6000010238BF002242634FF00001C16301648B
:107B7000416400F11000FDF78DF808BD2DE9F047D4
:107B800090B081468A4641F61863C2F201031A5C3E
:107B900041F6B430C2F201004FF04C0404FB020481
:107BA00004F148064FF001084FF000073546404603
:107BB0003146F8F7A9FA28B14FF002003146F8F73C
:107BC000A3FA36E0BAF1000F05D148464146FCF76A
:107BD000DFFC032827D0256C75B16846A168E26BED
:107BE000A8470546B0F1FF3F14D060644846694697
:107BF0002A46FCF7F3FC0EE0616CA5688D4228BFB5
:107C00000D464846E16B2A46FCF7E8FCE36B5A193F
:107C1000E26300E03D46606CA16888423CBFE763D8
:107C20002764451B656438463146F8F76DFA02282B
:107C3000BCD010B0BDE8F087F8B505460E46174633
:107C400041F61863C2F201031A5C41F6B430C2F285
:107C500001004FF04C0404FB02044FF00000FCF75D
:107C6000EFFBE76326644FF00001616428464FF0A4
:107C70000101FFF783FF4FF00100FCF7E1FBF8BDC6
:107C8000F8B505460F46164641F61863C2F20103E1
:107C90001A5C41F6B430C2F201004FF04C0404FB10
:107CA0000204A168B1420DD242F64C03C2F20103B4
:107CB0009F4207D343F24C02C2F20102974201D223
:107CC000F8F71EFA4FF00000FCF7BAFBE7634FF03D
:107CD00000002064666428464FF00101FFF74EFF64
:107CE0004FF00100FCF7ACFBF8BD00BF08B5FCF796
:107CF000FDFC08BD70B586B005460C46164602A8C8
:107D0000F9F744FB01462EB102A82A46234600F0AB
:107D10009BFD07E04FF00103009302A82A4623468B
:107D200000F044FE06B070BD70B58AB00378212B18
:107D300000F0938004D86BB1012B40F0D88186E02D
:107D4000A12B00F0A781C02B00F0B481802B40F064
:107D5000CE8195E04178052903D0092940F0CA81F8
:107D600046E0408841F66432C2F201021378022BE9
:107D700002D0032B33D118E000F1FF318AB27E2A02
:107D800030D8C0B241F61463C2F2010318704FF04C
:107D90000201FCF7B7FD41F66430C2F201004FF07A
:107DA000030101704FF00100C3E170B941F61462A4
:107DB000C2F20102107041F66430C2F201004FF0CD
:107DC000020303704FF00100B3E17F280DD841F6A4
:107DD0001461C2F2010108704FF00100A9E14FF0F7
:107DE0000200A6E14FF00200A3E14FF00200A0E183
:107DF000827841F66433C2F201031978022923D94B
:107E000072B941F66433C2F201034FF003011970F5
:107E10004FF001000146FFF7D5F94FF0010088E16E
:107E2000012A18BF022040F0848141F66430C2F27A
:107E300001004FF0040202704FF000000146FFF70E
:107E4000C1F94FF0010074E14FF0020071E1407898
:107E50000B280CBF012002206BE18388032B00F26A
:107E60004C8141F62C64C2F2010404EBC3035B684D
:107E7000002B00F045819847002808BF022058E1F8
:107E800042781AB1062A40F03E8121E0C1880229D9
:107E90001BD14FF00000ADF8040041F69832C2F259
:107EA000010212680346517E61F30003ADF804300D
:107EB000127E62F341030AA921F8243D4FF0020229
:107EC000FFF7DEFE4FF0030033E14FF0020030E138
:107ED0008278C1888CB2C378022B2ED0032B3DD080
:107EE000012B40F0D48041F64C65C2F201052846D2
:107EF0004AF2EC21C0F603014FF012020FF064F9D0
:107F000041F69830C2F2010001688A892A81CB8942
:107F10006B81088AA8818A7C2A71CB7C6B71097D70
:107F2000A9714FF000002946122C34BF22461222BC
:107F3000FFF7A6FE4FF00300FBE041F69C32C2F2D1
:107F4000010211814FF00000506047F63101C0F688
:107F50000201FFF771FE4FF00300EAE0D2B941F6EB
:107F60004C64C2F2010404F102004AF2E821C0F6B6
:107F700003014FF002020FF027F94FF004022270C4
:107F80004FF0030565704FF000002146FFF778FEC3
:107F90002846CEE0012A06D141F69833C2F2010309
:107FA000196809682FE0022A06D141F69832C2F218
:107FB00001021068416826E0032A06D141F6983391
:107FC000C2F20103196889681DE002F00F0022F077
:107FD0000F03102B08D15A4B196888420EDA594A00
:107FE00052F8300001680EE0202B07D1032805D895
:107FF000554951F8300008B1016804E0EE2A04D078
:108000004FF0020095E009B93EE05049B1F1FF3F61
:1080100040F0888001A84FF020014FF00102FFF7E7
:1080200069FE0AAD2A184FF0000002F8240C01A9DD
:1080300078E000F10206428003F10102134611F8D4
:10804000015F5DB100F10400758002F1010311F8D8
:10805000012F002A6FD101E04FF0000341F64C617F
:10806000C2F201014FF003054D7003F101034FEA25
:108070004303DAB20A704FF00000A24228BF224642
:10808000FFF7FEFD284654E04FF0020051E04FF0AC
:1080900002004EE08388032B38D841F62C64C2F2EC
:1080A000010404EBC3035B689BB39847002808BF37
:1080B00002203EE04378212B2ED1C18841F69C332B
:1080C000C2F2010319814FF000025A60808804282F
:1080D00025D1104647F21141C0F6020141F69C320B
:1080E000C2F20102FFF7A8FD4FF0030021E04FF0BC
:1080F00002001EE04FF002001BE04FF0020018E00B
:108100004FF0020015E04FF0020012E04FF00200C5
:108110000FE04FF002000CE04FF0020009E04FF0DA
:10812000020006E00A78002A96D009484FF00003C2
:108130007FE70AB070BD1E2B7FF47BAF8EE700BFD8
:10814000B01B0120781B01202C1E012014A3030862
:108150004C1E012010B50446436993B14FF0000056
:10816000606141F66431C2F201010A78032A08D144
:1081700041F61463C2F2010318784FF00301FCF7D3
:10818000C1FB206958B34FF000002061E06041F668
:108190007431C2F20101087041F66C31C2F2010182
:1081A0004FF00802FFF7A2FD082853D141F66C32C8
:1081B000C2F20102137813F0800F06D141F66C3041
:1081C000C2F20100C188002944D141F66C30C2F2EC
:1081D00001004FF000010A46FFF7A6FD2DE0E1681F
:1081E000002937D04FF00000E06041F67432C2F24F
:1081F0000102137841F64C61C2F20101C3F1400261
:10820000FFF774FD034628B341F67430C2F2010053
:1082100001785A18D2B2027041F66C33C2F20103EF
:10822000D888904216D141F66C30C2F2010041F676
:108230004C61C2F20101FFF777FD012804D002284A
:1082400008D1FCF7B5F910BD4FF000000146024619
:10825000FFF716FD10BD00BF08B541F68C63C2F2F2
:1082600001031B693BB14FF0000141F68C62C2F281
:1082700001025269984741F68C60C2F201004FF04A
:108280000001017041608160C1600161416108BD10
:1082900041F68C60C2F2010081614AF20841C0F6E9
:1082A00003018A5C42778377037F6FF307030377C9
:1082B0004FF000014162704730B583B041F68C64E5
:1082C000C2F201042070089D6560099DA5600A9DA9
:1082D000E5600B9D25610C9D65619DF8184000943B
:1082E0009DF81C400194FFF7D3FF03B030BD00BFE1
:1082F00041F68C63C2F201035B6AB3F1FF3F09D11F
:1083000041F68C61C2F201014FF000034B624FF065
:10831000010070473F2B0BD841F68C62C2F201027C
:10832000106AC15403F1010353624FF0010070471A
:108330004FF00000704700BF704700BF70B541F6B6
:108340008C64C2F2010404F118004AF27841C0F6CC
:1083500003014FF007020EF037FF4FF000004AF222
:108360004441C0F60301FFF7B3F948F29956C0F64D
:1083700002064FF000004AF2F031C0F60301324627
:10838000FFF7C4F94AF24C45C0F603054FF001006F
:1083900029463246FFF7BAF92869FFF7E3F984F86E
:1083A000280041F6B860C2F201004FF0070148F220
:1083B000C132C0F602024FF00003FCF74BFC70BD67
:1083C00038B541F6EC63C2F201034FF001021A70B6
:1083D00041F68C64C2F2010494F828004FF00001C9
:1083E0000A46FFF74DFC606868B141F68C64C2F242
:1083F00001044FF0FF356562636820786169984732
:10840000616A0029F7D041F68C60C2F201004FF09A
:1084100000024262836833B141F68C61C2F201010D
:1084200008784969984738BD2DE9F047A2B08046E1
:1084300043680BB9806828B14FF00001C8F80810F4
:10844000FFF7BEFFD8F80C20002A3ED04FF00007FF
:10845000C8F80C70D8F8000012A94FF04002FFF7DE
:1084600045FC074641F68C63C2F20103D86860B34D
:108470005FB341F68C64C2F201044FF0000507F1CE
:10848000FF3606F0010A20789DF848102A466369F5
:10849000E668B0474FF001094F456CD115E0E6683A
:1084A000207812AA12F809102A466369B04709F128
:1084B0000109E668207812AB13F809102A466369AF
:1084C000B04709F101094F45E9D1D8F81400002857
:1084D0004ED04FF0000441F6EC61C2F201010C7085
:1084E000C8F8144041F6C860C2F20100FEF752FD20
:1084F00041F68C62C2F2010254625368002B30D004
:1085000041F68C65C2F2010502AC2C622C46656A0C
:108510006268207861699047606A8542F7D105B347
:10852000D8F8000002A92A46FFF7AAFB4FF0000185
:108530000091019141F6C860C2F201004FF04B0179
:108540004FF0FF0248F2C133C0F60203FEF7C8FD48
:108550000EE041F68C62C2F2010210785169984730
:1085600006E041F68C63C2F201039B68002BF0D158
:1085700022B0BDE8F087BAF1000F90D0E66820780D
:1085800012A911F809102A466369B04709F10109D7
:108590004F4584D199E700BF10B544780378212B6B
:1085A00002D0A12B19D10CE0202C02D0222C08D112
:1085B00019E0072A1AD10F480EF006FE4FF001000D
:1085C00010BD212C0CD14FF000000A494FF00702DA
:1085D000FFF756FB4FF0030010BD4FF0000010BD39
:1085E0004FF0000010BD4FF0010010BD4FF0020031
:1085F00010BD00BFA41E012008B541F6EC63C2F215
:108600000103187870B941F68C61C2F201014A6A1F
:1086100072B941F68C63C2F2010393F82800FFF7A8
:108620008FFA08BD41F6B860C2F20100FCF732FBD8
:1086300008BD00BF4AF2C030C0F60300704700BF5B
:1086400070B4037801298CBF4478002402298CBFC0
:1086500085780025DCF8000048B34FEA93064AF21B
:108660008050C0F60300365C16704FEA031343EAED
:10867000141303F03F031B5C5370012907D94FEA21
:10868000840444EA951303F03F04205C01E04FF0BA
:108690003D009070022907D905F03F054AF280534A
:1086A000C0F60303E95C01E04FF03D01D17070BCFE
:1086B000704700BF82B04FF00A010CE00191019BAE
:1086C00003F1FF32019233B100BF019B03F1FF328E
:1086D0000192002BF8D100F1FF30B0F1FF3FEDD156
:1086E00002B0704770B4C4B24FEA10204AF280461C
:1086F000C0F603064AF21465C0F6030511F8013B03
:108700001AB94BB944EA00200BE06340F45C4440E2
:10871000E85C013AF2D1F5E76340F45C4440E85C80
:10872000ECE770BC704700BF10B444F6FB43C0F2E6
:10873000861311F8014B02B9ACB380EA04404FEA4A
:10874000400010F0807F18BF58404FEA400010F002
:10875000807F18BF58404FEA400010F0807F18BF5C
:1087600058404FEA400010F0807F18BF58404FEA51
:10877000400010F0807F18BF58404FEA400010F0D2
:10878000807F18BF58404FEA400010F0807F18BF2C
:1087900058404FEA400010F0807F18BF5840002A30
:1087A000C7D0013AC5D120F07F4010BC704700BF50
:1087B00082B001909DF806304FF0000063F307008F
:1087C0009DF8052062F30F209DF8042062F3174006
:1087D0009DF8072012F0800F14BF63F07F0103F0B3
:1087E0007F0161F307004FEA4201CAB262F31F60E2
:1087F00013F0800F18BF42F0010262F31F6002B055
:10880000704700BF84B0C0F307438DF80C30C0F34D
:1088100007228DF80D20C3B24FEA10604FEA5002D4
:1088200010F0010F14BF63F07F0103F07F018DF89A
:108830000E1013F0800F18BF62F07F028DF80F202A
:10884000039804B0704700BF2DE9F04F83B0054690
:108850000F4614461E46019201F1FF3313F1050F36
:1088600044D8032E43D9A6F10400C0F380080DF1CB
:10887000040C2846FFF7E4FE05F10305A7F1030108
:1088800004F10404A6F10406A7F1040717F1050F8B
:1088900067D92CE00DF1040C284639462246FFF733
:1088A000CFFE05F1030B5D46A7F1030104F1040AB5
:1088B0005446A6F104094E46A7F1040717F1050F27
:1088C00015D80F460DF1040C58465246FFF7B8FE76
:1088D0000BF10305A7F103010AF10404A9F1040651
:1088E000A7F1040818F1050F59D900E0FFE799B383
:1088F00096B30DF1040C28466A46FFF7A1FE022E3E
:1089000011D0032E02D0012E26D11AE0019929B1EF
:108910009DF8002022704FF0010301E04FF00003AA
:1089200004F1010401E04FF00003019830B102A905
:10893000CA1812F8080C207003F1010304F10104B5
:1089400001E04FF00003019921B102AAD31813F8F6
:10895000080C207004F101040199601A03B0BDE80D
:10896000F08F0F46032EC2D9B8F1000F92D00DF14F
:10897000040C28462246FFF763FE05F10305A7F124
:10898000030104F10404A6F10406A7F1040717F19A
:10899000050FACD80F46032E3FF67CAFA7E7A7F133
:1089A0000307032E3FF676AFA1E700BFF0B49DF8B2
:1089B0001040ECB14FEA41079F421CD2DD1B1DD095
:1089C00056194FF030046FEA0203F31803F0010365
:1089D00002F8014BB24240F0928007E0134603F8E0
:1089E000014B547003F10102B242F7D13B4607E05C
:1089F0004FF0000504E04FF0000501E04FF00005E6
:108A000000293CD003F1FF34002B3AD000F10103E0
:108A100041182846521B04F1FF3515F0020F10D003
:108A200032E0A4F1020603F101031F46012C29D014
:108A30003446B44613F8016C4FEA1616092E42D993
:108A400044E01E4613F8015C4FEA1515092D8CBF52
:108A500037353035155414B900F1010012E013F820
:108A6000016C06F00F05092D8CBF3735303516180F
:108A7000757000F1020528468B42D2D102E02846EB
:108A800000E02846F0BC70471E4613F8015C4FEA30
:108A90001515092D94BF303537351554002CDBD012
:108AA00013F8016C06F00F05092D94BF30353735EA
:108AB0001618757000F102008B42E3D003F1010338
:108AC000A4F10204BDE706F1300601E006F1370625
:108AD0005655BCF1000FBFD013F8016C06F00F061D
:108AE000092E94BF303637361018467005F1020053
:108AF0008F42C7D003F10103A4F10204A1E7002BC8
:108B00003FF46CAF02F8014BB2427FF467AF6DE700
:108B1000DCF8143093F8452083F84420DCF8141076
:108B200091F8463081F84530DCF8141091F8472070
:108B300081F84620DCF8143083F84700704700BF06
:108B4000DCF8143093F8470093F8462083F8472068
:108B5000DCF8141091F8453081F84630DCF8141038
:108B600091F8442081F84520704700BF42F2A412DA
:108B7000C2F20102136840F20001C0F60101C85CB4
:108B8000C918497803F10203136041EA00207047D5
:108B9000DCF80430DCF8082002EBD300CCF8080045
:108BA00003F007014FF0010303FA01F2CCF80420AF
:108BB000704700BF2DE9F04F83B004468A469346C4
:108BC0001E46CDF804C04FF00007B846B9463DE058
:108BD00025463046D047034600283DD0B9F1000F66
:108BE0000CD1202829D0092829D00A2829D00D28DD
:108BF00029D0022D4FF0010988BF0225A3F13002D0
:108C0000D1B2092910D9A3F14100C1B2052903D875
:108C1000A3F13703D9B207E0A3F16102D0B205286E
:108C20001AD8A3F15703D9B24FEA0717FCB241EAA9
:108C3000040708F101082C4606E02C4604E02C4607
:108C400002E02C4600E02C463046D847FF2CBFD02F
:108C500004F1FF35002CBCD1DDF804C03846FFF725
:108C600057FF019B5A69D8F1010838BF4FF000083F
:108C700082F8508003B0BDE8F08F00BF42F240039D
:108C8000C2F201031B684B634BB19A68824209D060
:108C9000DB684B631BB19A688242F9D102E04FF066
:108CA0001E0070474FF00000704700BF884204D894
:108CB000884234BF0220002070474FF00100704707
:108CC000D0F80431D0F80021934214BFC05C0020DA
:108CD000704700BFD0F80431FF2B14BF01330023CD
:108CE000C0F80431704700BF10B4DCF81420D16C18
:108CF0000B46044658B14FEA016343EA116301F49D
:108D00007F4043EA002301F47F0143EA1123DCF8AA
:108D1000040030B199B24FEA134060F30F0361F3DE
:108D20001F435CB94FEA036141EA136103F47F40DA
:108D300041EA002103F47F0341EA1323D36410BC0A
:108D4000704700BFDCF80030FA2B05D841F6F0621E
:108D5000C2F20102D05C70474FF00000704700BFC4
:108D6000DCF8003003F10103CCF80030DCF814002B
:108D700090F8512002F1010280F85120704700BFA5
:108D800070B404460846A1B199188C4211D2251836
:108D9000AA420ED294423ABFC4EB0206F6B20026B3
:108DA000A94205D20019821AD31AF118C8B200E0FC
:108DB000304670BC704700BFF0B583B042F2480344
:108DC000C2F201034FF00C021A7042F23400C2F2F8
:108DD000010004683CB3154642F24807C2F201079D
:108DE0004FF0000621680B6873B10DF107000DF11B
:108DF000060198479DF807009DF8061032463B781B
:108E0000FFF7BEFF4519EDB26468002CEAD142F2CB
:108E10004802C2F201021078A84204D242F248018C
:108E2000C2F201010D7042F24803C2F201034FF099
:108E30000A025A7042F26004C2F2010424683CB390
:108E4000154642F24807C2F201074FF000062068BB
:108E5000036873B10DF107000DF1060198479DF805
:108E600007009DF8061032467B78FFF789FF451909
:108E7000EDB26468002CEAD142F24801C2F201016D
:108E80004A78AA4204D242F24800C2F20100457078
:108E900042F24803C2F201034FF00501997042F219
:108EA000A014C2F2010424683CB30D4642F2480704
:108EB000C2F201074FF000062268136873B10DF18A
:108EC00007000DF1060198479DF807009DF8061070
:108ED0003246BB78FFF754FF4519EDB26468002CA9
:108EE000EAD142F24800C2F201008178A94204D2DC
:108EF00042F24802C2F20102957042F24803C2F205
:108F000001034FF00100D87042F2AC14C2F2010428
:108F100024683CB3054642F24807C2F201074FF00D
:108F2000000621680A6872B10DF107000DF1060113
:108F300090479DF807009DF806103246FB78FFF732
:108F40001FFF4519EDB26468002CEAD142F24803D4
:108F5000C2F20103D878A84204D242F24801C2F218
:108F60000101CD7003B0F0BD42F29C13C2F20103C7
:108F7000196840F20000C0F60200401A704700BFB6
:108F8000034610B182688A4218D042F24403C2F20A
:108F90000103186860B182688A4203D10BE08368DC
:108FA0008B420AD040680028F9D14FF0000305E059
:108FB0004FF0000302E0034600E003461846704706
:108FC00010B540F2A064C1F200044FF4117303FB2A
:108FD0000044D4F80811B1F1FF3F03D0D4F80421C4
:108FE00091420DD123689A6A4FF0FF019047002803
:108FF00034D0D4F8080100F10100C4F8080110BD14
:1090000091422BD86318197942F22C02C2F2010264
:1090100013787BB9FD290FD923689A6A4FF0FE01B6
:109020009047D8B142F22C00C2F201004FF001018A
:10903000017010BD6FEA01012268936AC9B29847B6
:1090400060B1D4F8080100F10100C4F8080142F24F
:109050002C01C2F201014FF000020A7010BD00BFE6
:1090600070B5064640F2A065C1F200054FF41174D8
:1090700004FB00F42B194FF00101C3F80C112A591D
:10908000936998472859016A3046884770BD00BFE8
:1090900038B540F2A061C1F200014FF4117202FB39
:1090A00000F28C18D4F80831D4F80451AB420DD03A
:1090B0008958E3188A6A1979904738B1D4F80801B9
:1090C000FF2814BF01300020C4F8080138BD00BFDC
:1090D00038B540F2A064C1F200044FF4117202FBF3
:1090E00000F2A318D3F80451D3F808118D4206D129
:1090F0004FF00001C3F80C11A2589369984738BD8E
:1091000010B440F2A063C1F200034FF4117202FBED
:10911000003000F58870D0F80031FF2B14BF5A1CC6
:109120000022D0F80441A2421CBFC154C0F8002163
:1091300010BC7047F8B542F29C14C2F201042468D6
:109140008568C768466807FB05604518611911D234
:10915000CE180B48864210D8012B04D1635D1370E2
:109160004FF00000F8BD10461A460EF02DF84FF0F3
:109170000000F8BD4FF01F00F8BD4FF01F00F8BD14
:109180000100020810B542F24C03C2F201031A7842
:1091900040F2A060C1F200004FF4117404FB02041D
:1091A000F7F704F84FF0FF31C4F810124FF0000346
:1091B000C4F8183204F58874F7F702F810BD00BF40
:1091C000F8B506464FF00203037044F20000C0F603
:1091D0000000C28B4FF6FF718A4221D03F4C404BBA
:1091E000A34222D203F110033E4DEF1A4FEA1712A9
:1091F0004FF6FF7502F1010002F001071C46D98B02
:10920000A9424FD115E01C46D98BA94211D002F1D9
:10921000010203F110031C46D98BA94257D108E083
:1092200044F20004C0F6000403E044F20004C0F677
:1092300000044FF6FF7021464FF00D02FFF752FA7F
:109240004FF6FF73984208BF0020E28982421BD08C
:10925000A4F1100544F20000C0F6000085421AD3C4
:109260004FF6FF7029464FF00D02FFF73BFA4FF61D
:10927000FF71884208BF002034F8024C84420AD1B2
:109280002C464FF0010201E04FF00002607BFF2806
:1092900006D1327004E04FF0020333704FF0000447
:1092A0002046F8BD4FF0000202F1010203F1100365
:1092B0008242BED0002FA6D01C46D98BA942B8D07E
:1092C00002F1010203F1100382429CD1B1E702F1E5
:1092D000010203F11003824295D1AAE70080000841
:1092E000004000080F80000870B5C0B005460E466B
:1092F00020F0FF04684621464FF04002F9F718F9C4
:1093000000AB53FA85F031464FF010020DF05CFFD0
:10931000684621464FF48072F9F75EFA40B070BD9E
:1093200038B5054640F2A064C1F200044FF4117351
:1093300003FB0044D4F81C02FDF73AFB42F24C0058
:10934000C2F201000178A94206D142F24C03C2F2F6
:1093500001034FF0FF021A704FF00000C4F81C0226
:1093600038BD00BF10B54FF00000FBF7B3FC42F270
:109370003403C2F201031C6834B12068016901B1F1
:1093800088476468002CF8D110BD00BF10B50446B2
:10939000072827D8032894BF4FF4FA73322303FB1E
:1093A00001F140F2A063C1F2000303EBC000C0F87A
:1093B000141969B1FDF7CAFE002808BF012040F268
:1093C000A063C1F2000303EBC404C4F8100910BD8C
:1093D00040F2A061C1F2000101EBC4044FF00002B1
:1093E000C4F8102910BD00BF38B50446072851D86D
:1093F00040F2A063C1F2000303EBC000D0F814599F
:1094000035B340F2A061C1F2000101EBC402D2F811
:109410001039EBB1FDF79AFE002808BF012040F299
:10942000A061C1F2000101EBC402D2F81039C01AE8
:1094300085420CD240F2A065C1F2000505EBC401E3
:109440004FF00005C1F81459C1F8105900E02D1A69
:1094500005F104054CF6CD42CCF6CC42A2FB052327
:109460004FEA9300032C0AD800F1630348F21F511E
:10947000C5F2EB11A1FB03324FEA521038BD00F1E7
:1094800009014CF6CD42CCF6CC42A2FB01304FEAAA
:10949000D00038BD4FF0000038BD00BF70B50646A3
:1094A0006446DCF814305D6AFDF750FE6169CA6AF3
:1094B0000AB9C86208E0801A05EB850506FB05F6C7
:1094C000B04224BF0020C8626369D96AD1F10100AB
:1094D00038BF002070BD00BF10B540F2A063C1F2DC
:1094E00000034FF4117404FB003303F58873D3F8C1
:1094F0000841002C5FD15AB14FF0FF31C3F8001181
:1095000042F22D03C2F201034FF00000187010BDAB
:10951000D3F80021B2F1FF3F06D1FF294BD14FF024
:109520000002C3F8002110BDFF291ED142F22D0117
:10953000C2F201014FF000040C70012A10D94FF063
:109540000102C3F8082140F2A063C1F200034FF406
:10955000117101FB0030D0F81C02FCF7E7FF10BDD1
:109560004FF00000C3F8000110BDFE2907D142F200
:109570002D03C2F201034FF00101197010BD42F238
:109580002D00C2F20100007848B16FEA0101C9B2B2
:1095900042F22D00C2F201004FF000040470FF2AD5
:1095A00005D8995402F10102C3F8002110BD4FF013
:1095B000FF32C3F8002110BD08B540F2A063C1F22C
:1095C00000034FF4117202FB0030D0F80811D0F8FC
:1095D000043100F1040099420AD94FF00002C0F8AA
:1095E000002142F27800C2F201004068FCF79EFFC1
:1095F00008BD00BFF8B5654642F2B013C2F20103E0
:109600001C7804F00802D7B227B1DCF8146096F891
:10961000516007E014F0110F06BFDCF8144094F815
:109620005260002601EB800411F820304FEA9312BB
:10963000012A08D0022A10D111F82070C7F3C20302
:1096400003FB06F70BE06A6992F8513011F82070BD
:10965000C7F3C20202FB03F701E04FF0000711F865
:10966000200000F00701042950D8DFE811F0940130
:1096700040003B002200050042F2A411C2F20101A9
:109680000B6840F20007C0F60107FA1892F802E0F2
:10969000D0784FEA006040EA0E40527840EA02205B
:1096A000FF5C03F104030B603843FFF7ABF868601D
:1096B0002CE042F2A412C2F20102136840F2000050
:1096C000C0F60100C11891F801C0C05C4FEA00402B
:1096D00040EA0C208978084303F1030313603F1824
:1096E0006F6013E0FFF742FAC2196A600EE042F2BF
:1096F000A413C2F20103186840F20001C0F6010190
:109700000A5CBF186F6000F10100186063784FEACF
:109710009310012807D002280ED16178C1F3C2024C
:1097200002FB06F70AE06F6997F851306078C0F3E2
:10973000C20101FB03F701E04FF00007627802F07D
:109740000703042B50D8DFE813F0260140003B004C
:109750002200050042F2A411C2F201010B6840F29E
:109760000007C0F60107FA1892F802E0D0784FEA35
:10977000006040EA0E40527840EA0220FF5C03F1AC
:1097800004030B603843FFF73DF8A8602CE042F279
:10979000A412C2F20102136840F20000C0F60100F8
:1097A000C11891F801C0C05C4FEA004040EA0C20AB
:1097B0008978084303F1030313603F18AF6013E097
:1097C000FFF7D4F9C219AA600EE042F2A413C2F264
:1097D0000103186840F20001C0F601010A5CBF18DD
:1097E000AF6000F101001860A3784FEA93100128E0
:1097F00007D002280ED1A178C1F3C20202FB06F7FE
:109800000AE06F6997F85130A078C0F3C20101FBFC
:1098100003F701E04FF00007A27802F00703042BE2
:109820004ED8DFE803F0B83E3920030042F2A4111D
:10983000C2F201010B6840F20007C0F60107FA18F6
:1098400092F802E0D0784FEA006040EA0E40527889
:1098500040EA0220FA5C03F104030B601043FEF7B8
:10986000D1FFE8602CE042F2A412C2F201021368B8
:1098700040F20000C0F60100C11891F801C0C05CC0
:109880004FEA004040EA0C208978084303F10303C3
:1098900013603F18EF6013E0FFF768F9C219EA6040
:1098A0000EE042F2A413C2F20103186840F2000174
:1098B000C0F601010A5CBF18EF6000F101001860FA
:1098C000E3784FEA9310012802D002280FD108E074
:1098D0006E6996F85130E078C0F3C20101FB03F6DF
:1098E00007E0E178C1F3C20202FB06F601E04FF0A7
:1098F0000006E27802F00703042B4CD8DFE803F0FF
:109900004B031318300042F2A413C2F2010318688B
:1099100040F20001C0F601010A5CB6182E6100F1A8
:1099200001001860F8BDFFF721F982192A61F8BD1E
:1099300042F2A412C2F20102136840F20000C0F623
:109940000100C1184C78C05C4FEA004040EA042096
:109950008978084303F10303136036182E61F8BDBC
:1099600042F2A411C2F201010B6840F20004C0F6F9
:109970000104E2189678D0784FEA006040EA064089
:10998000527840EA0220E25C03F104030B601043CA
:10999000FEF738FF2861F8BD08B503281ED8DFE8B8
:1099A00000F0020910174AF6D050C0F603000FF07D
:1099B000FBF908BD4AF6D450C0F603000FF0F4F9E5
:1099C00008BD4AF6E850C0F603000FF0EDF908BDF7
:1099D0004AF60060C0F603000FF0E6F908BD00BFCC
:1099E0002DE9F8430546884616461F4642F24C03C9
:1099F000C2F2010393F8009042F24850C2F2010013
:109A0000016842F23002C2F201021368994201D0A9
:109A1000FFF7B8FB072D6ED81F2E6CD840F2A0645C
:109A2000C1F200044FF4117000FB094442F27800C7
:109A3000C2F201004FF00001FCF718FB217965F339
:109A40004711072D14BF00250125AA1962F304014F
:109A50002171CBB22DB184F8058043444FF0020050
:109A600001E04FF0010006F1FF3E5FFA8EFE46B3C3
:109A700002463F1A0EF0010C3D5C04F10406355419
:109A80005B1902F101020EF1FF31C9B2FF2934D195
:109A900014E0BD5C04F10406B5545B1902F1010247
:109AA00001F1FF3101F0FF01BD5CB5545B1902F11A
:109AB000010201F1FF31C9B2FF29EAD100F1010031
:109AC00070442218137100F10100C4F804014FF032
:109AD000FF33C4F8083121680B6A42F24C00C2F22D
:109AE000010000789847FCF7EFFC42F27800C2F2E0
:109AF0000100FCF7C9FBBDE8F8834FFA8CF5002D97
:109B0000C7D0BD5C04F10406B5545B1902F1010233
:109B100001F1FF31C9B2FF29BBD1CFE738B5054606
:109B200041F6F074C2F201042046FCF7ADFBF7F7F2
:109B300027FD2846FCF790FE20464FF00001FCF779
:109B400095FA38BD10B586B00DF10700FFF738FB68
:109B5000044618B19DF8073023B90FE044F2000421
:109B6000C0F60004E2894FF6FF7082422BD048F223
:109B70000001C0F600018C4209D32AE0304821469A
:109B80004FF00D020CF0CAFE002848D0EAE74FF66D
:109B9000FF7248F20000C0F600006FEA0403C1182B
:109BA000C1F3001104F11004E389934239D10AE0B2
:109BB00004F110031C46D989914204D003F110042A
:109BC000E389934239D148F20002C0F60002944280
:109BD00007D344F20004C0F6000420462146F8F7FB
:109BE0008FFD02A816494FF00D020DF0EDFA4FF06F
:109BF000FF008DF815004FF6FF7002A94FF00D021F
:109C0000FEF770FD4FF6FF71884212BFADF81600E7
:109C10000021ADF81610204602A9FFF765FB06B03B
:109C200010BD8442D5D20029C2D004F11004E189CC
:109C30009142C8D08442BBD3CBE78442B8D3C8E7B3
:109C4000F61E01202DE9F04F85B0884691461D464D
:109C5000E2464FF0000426464FF0020B2DE0074687
:109C60002846C047034670B324B9202822D00928CB
:109C700002D11FE0012C05D12B2B0DD02D2B0DD0A7
:109C80005C4601E0022C01D12E2B09D0A3F1300259
:109C9000D0B2092817D805E05C4603E05C4601E035
:109CA0004FF003040E2E05D804A98A1902F8103CBF
:109CB00006F101062846C8473846FF28CFD000F1F4
:109CC000FF370028CCD1012C12D98EB104ACA619D3
:109CD0004FF0000406F8104C684621460CF078FE60
:109CE000DAF81410C864DAF8142082F8504005E05D
:109CF000DAF814304FF0010083F8500005B0BDE8E9
:109D0000F08F00BF10B586B040F20000C0F6010031
:109D10003449F8F7F5FC00284BD1334B334A9A42CB
:109D20001DD240F20001C0F601010B68B3F1FF3F04
:109D300042D102F104032E4AD01A20F003029918EE
:109D400012F0040F3FD118468B420CD003F10402ED
:109D50001B68B3F1FF3F3ED04FF0000031E040F20E
:109D60000000C0F6010040F20003C0F60203984272
:109D700025D10DF10700FFF723FA0446B0B19DF895
:109D80000710022912D002A821464FF010020DF050
:109D90001BFA9DF815006FF307008DF8150020469B
:109DA00002A9FFF7A1FA4FF001000AE04FF001000D
:109DB00007E04FF0000004E04FF0000001E04FF03A
:109DC000000006B010BD184603F104030268B2F1AA
:109DD000FF3FB8D0C0E702F104031068B0F1FF3FC5
:109DE000B1D0B9E7FFFF0108000002080000010838
:109DF000030002082DE9F007034600284AD040F28C
:109E00000022C0F6000292F8469092F8478042F293
:109E10004800C2F2010090F801C092F848A005780D
:109E200042F26402C2F201021468177A567A50684C
:109E30004FF000021A7083F8019083F80280DA7004
:109E40004FF0FB0883F804804FF0060883F8058084
:109E50009D7183F807C04FF0040C83F808C083F8A5
:109E600009C083F80AA0DD721A734FEA14255D73E6
:109E70009C73DF731E745A744FF01D029A744FF076
:109E80000202DA744FF0FE021A755A754FEA102278
:109E90009A75D87529B142F24803C2F201031868D5
:109EA0000860BDE8F0077047034628B142F264023B
:109EB000C2F201021068186042F26401C2F20101AC
:109EC000087A704770B505460E4614464FF00000FC
:109ED0002946FFF755F808B1F6F712F942F24403A4
:109EE000C2F201031A686260A56026601C6070BD42
:109EF00008B539B142F23403C2F201031A68426074
:109F000018601EE042F23403C2F201031B68834270
:109F10000FD1586842F23401C2F20101086010E02A
:109F200042685A6041605A688242F9D013461BB9B0
:109F300007E033B14FF000015A688242F0D0134677
:109F4000F5E7FEF739FF08BD08B539B142F2600305
:109F5000C2F201031A68426018601EE042F2600318
:109F6000C2F201031B6883420FD1586842F26001BC
:109F7000C2F20101086010E042685A6041605A680C
:109F80008242F9D013461BB907E033B14FF000010C
:109F90005A688242F0D01346F5E7FEF70DFF08BD80
:109FA00008B539B142F2A013C2F201031A68426047
:109FB00018601EE042F2A013C2F201031B68834244
:109FC0000FD1586842F2A011C2F20101086010E0FE
:109FD00042685A6041605A688242F9D013461BB900
:109FE00007E033B14FF000015A688242F0D01346C7
:109FF000F5E7FEF7E1FE08BD08B539B142F2AC1352
:10A00000C2F201031A68426018601EE042F2AC130B
:10A01000C2F201031B6883420FD1586842F2AC11AF
:10A02000C2F20101086010E042685A6041605A685B
:10A030008242F9D013461BB907E033B14FF000015B
:10A040005A688242F0D01346F5E7FEF7B5FE08BD28
:10A0500001604360826042F24003C2F201031A6869
:10A06000C2601860704700BF70B582B006464FF0FE
:10A0700000038DF807300D4601B10B7042F2340039
:10A08000C2F20100046874B121684B6843B13046E4
:10A090000DF107012A46984710B19DF8070011E01D
:10A0A0006468002CF0D10B2E03D83046FAF756FE28
:10A0B00008E02DB14FF005022A704FF0000001E0DA
:10A0C0004FF0000002B070BD70B582B006464FF090
:10A0D00000038DF807300D4601B10B7042F23400D9
:10A0E000C2F20100046874B121688B6843B1304644
:10A0F0000DF107012A46984710B19DF8070019E0B5
:10A100006468002CF0D10B2E0BD83046FAF73CFED9
:10A110008DF8070010B13046FAF77CFE9DF8070075
:10A1200008E02DB14FF005022A704FF0000001E069
:10A130004FF0000002B070BD70B582B006464FF01F
:10A1400000038DF807300D4601B10B7042F2340068
:10A15000C2F20100046874B12168CB6843B1304693
:10A160000DF107012A46984710B19DF8070011E04C
:10A170006468002CF0D10B2E03D83046FAF7D4FDDA
:10A1800008E02DB14FF005022A704FF0000001E009
:10A190004FF0000002B070BD70B582B006464FF0BF
:10A1A00000038DF807300D4601B10B7042F26000DC
:10A1B000C2F2010004685CB121688B682BB13046A3
:10A1C0000DF107012A46984758B96468002CF3D16D
:10A1D000092E0CDC0A2E0AD83046F6F72BFE8DF835
:10A1E00007009DF80700003018BF012008E02DB1DE
:10A1F0004FF006022A704FF0000001E04FF000001F
:10A2000002B070BDF0B583B005460E464FF00003B6
:10A210008DF8073042F26000C2F201000468E4B138
:10A220004FF000072168CA681AB1284631469047A6
:10A23000F0B923689B6833B128460DF106010DF192
:10A240000702984700E038469DF8071099B96468FE
:10A2500014B10028E6D004E018B9092D0DDC0A2D50
:10A260000ED82846314606F0D9FA4FF0000009E032
:10A270004FF0000006E0084604E04FF0060001E061
:10A280004FF0060003B0F0BD70B582B005460E4633
:10A290004FF000038DF8073012B11946FFF7B2FFF7
:10A2A00042F26000C2F2010004686CB121684B68A0
:10A2B000284631460DF10702984710B19DF8070076
:10A2C00012E06468002CF1D1092D08DC0A2D09D8B0
:10A2D00028463146F6F7D0FD4FF0000004E04FF07D
:10A2E000060001E04FF0060002B070BD08B54FF067
:10A2F000000001464FF00102FFF7C6FF08BD00BF96
:10A3000070B582B005460E464FF000038DF8073059
:10A3100042F2A010C2F2010004689CB121684B68AF
:10A32000284669460DF10702984728B10EB10098FA
:10A3300030609DF8070014E064681CB19DF80720A8
:10A34000002AEBD0042D07D84EB12846F7F770FB52
:10A3500030604FF0000004E04FF00F0001E04FF0DC
:10A36000000002B070BD00BF70B582B005460E4659
:10A370004FF000038DF8073042F2AC10C2F201003A
:10A38000046884B121684B68284631460DF1070204
:10A39000984710B19DF8070010E064681CB19DF863
:10A3A0000720002AEED03DB94FF000003146F7F704
:10A3B000EDF94FF0000001E04FF00E0002B070BD6B
:10A3C00070B582B005460E464FF000038DF8073099
:10A3D00042F2AC10C2F201000468A4B121688B689B
:10A3E0005BB1284669460DF10702984728B10EB1C6
:10A3F000009830609DF8070014E064681CB19DF877
:10A400000720002AEAD045B956B14FF00000F7F70F
:10A4100033FB30604FF0000004E04FF0060001E035
:10A420004FF0000002B070BD2DE9F04F2DED048B10
:10A430008BB007461546914259D289464FF0000B22
:10A440004FF000089FED908B9FED919B6FEA010606
:10A45000B01800F00106CDF804B0022F4CD150E046
:10A46000CDF804B0022F05D15FFA89F001A9FFF7FA
:10A47000A7FF04E05FFA89F001A9FFF741FF04EBB1
:10A4800044060AA88119A1F1200601F8209C01F8D0
:10A490001F8C01980BF0FCFC53EC182B0BF096FE74
:10A4A00053EC192B0BF04EFD0BF0B8FC83B2FF2BD5
:10A4B00028BFFF23B37004F101040A2C04D005F176
:10A4C000FF324A450AD14CB104EB44044FF0070077
:10A4D0003946E2B202ABFFF783FA444609F10109BB
:10A4E0004E46CDF804B0022F40F089808DE00BB0CD
:10A4F000BDEC048BBDE8F08FC8B201A9FFF700FFE7
:10A5000003E0C8B201A9FFF75BFF0AAC04F8209D85
:10A5100084F8018001980BF0BBFC53EC182B0BF076
:10A5200055FE53EC192B0BF00DFD0BF077FC81B2AF
:10A53000FF2934BF0B46FF23A3704FF0000404F142
:10A54000010405F1FF324A450DD10AE004EB440451
:10A550004FF007003946E2B202ABFFF741FA44463A
:10A5600001E0002CF2D109F101094D45BFD9002EBF
:10A570003FF476AFCDF804B0022F05D05FFA89F032
:10A5800001A9FFF7BDFE04E05FFA89F001A9FFF71A
:10A5900017FF04EB44060AA8861906F8209D86F8E2
:10A5A000018001980BF074FC53EC182B0BF00EFE9D
:10A5B00053EC192B0BF0C6FC0BF030FC81B2FF29D9
:10A5C00034BF0B46FF23B37004F101040A2C0AD1F7
:10A5D00004EB44044FF007003946E2B202ABFFF748
:10A5E000FFF9444605E005F1FF324A4501D1002C50
:10A5F000EED109F101094D453FF632AF77E75FFA39
:10A6000089F001A9FFF77CFE04E05FFA89F001A957
:10A61000FFF7D6FE04EB44000AA90B18A3F1200AA9
:10A6200003F8206C03F81F8C01980BF031FC53ECFD
:10A63000182B0BF0CBFD53EC192B0BF083FC0BF01C
:10A64000EDFB82B2FF2A28BFFF228AF8022004F124
:10A6500001040A2C0AD104EB44044FF007003946E8
:10A66000E2B202ABFFF7BCF9444605E005F1FF306A
:10A67000B04201D1002CEED109F101094D453FF660
:10A68000EFAE34E7AFF300800000000000E06F4061
:10A69000000000000000E03F2DE9F04F95B040F6CB
:10A6A000C410FCF7D9F84FF002004FF0000142F25D
:10A6B0004803C2F20103DA78FFF7B6FE4FF0000B51
:10A6C000DA46D9464FF001074CF6CD44CCF6CC44DF
:10A6D00001944FF07D00FCF7BFF88DF82F90C8462D
:10A6E0004E464C4613E045F0800504F10804E4B200
:10A6F0000CABF05CA84202D00CA97554B84606F128
:10A7000001069DF82F50002D50D1202E4ED020460E
:10A710000DF12F01FFF7A8FC051C18BF012504F15E
:10A720000100C0B20DF12F01FFF79EFC10B145F002
:10A730000205EDB204F10201C8B20DF12F01FFF7DD
:10A7400093FC08B145F0040504F10302D0B20DF109
:10A750002F01FFF789FC08B145F0080504F1040357
:10A76000D8B20DF12F01FFF77FFC08B145F01005BD
:10A7700004F10500C0B20DF12F01FFF775FC08B11F
:10A7800045F0200504F10601C8B20DF12F01FFF7D5
:10A790006BFC08B145F0400504F10702D0B20DF1A1
:10A7A0002F01FFF761FC00289DD19EE7B8F1000F53
:10A7B00002D1BAF1000F0AD14FF002004946F2B2BD
:10A7C0000CABFFF70DF94FF03200FCF745F842F201
:10A7D0004802C2F2010292788AB1019EA6FB0A43A6
:10A7E0004FEA131404EB8400BAEB800F07D138460C
:10A7F0004946FFF719FE4FF03200FCF72DF8BBF188
:10A80000000F40F09B8003A849464FF020020CF057
:10A81000FFFC42F24801C2F201018D78ADB34E4611
:10A820006FEA0902531903F0010009F0070407FA5F
:10A8300004F29DF80C1042EA01038DF80C3006F189
:10A840000106AE42C0F299801FE014AA02EBD603C3
:10A8500006F0070407FA04F013F8441C40EA01026A
:10A8600003F8442C06F1010614AC04EBD60006F004
:10A87000070107FA01F210F8443C42EA030400F829
:10A88000444C06F10106AE42DFDB4FF007004FF00B
:10A8900011014FF01E0203ABFFF7A2F84FF0320098
:10A8A000FBF7DAFF03A849464FF020020CF0B0FC9A
:10A8B00042F24805C2F20105EE78A6B348466FEAB7
:10A8C00009018A1902F0010309F0070407FA04F5E7
:10A8D0009DF80C1045EA01028DF80C2000F10100F2
:10A8E000864236DC1FE014AD05EBD00200F0070411
:10A8F00007FA04F312F8441C43EA010502F8445C29
:10A9000000F1010014AA02EBD00500F0070407FAD9
:10A9100004F315F8441C43EA010205F8442C00F145
:10A9200001008642DFDC4FF007004FF012014FF0CC
:10A930001E0203ABFFF754F84FF0060BBAF1000FFD
:10A9400004D10BF1FF3B4FF0280AC2E60AF1FF3AAF
:10A95000BFE6002BC7D014AB03EBD00500F0070413
:10A9600007FA04F215F8441C42EA010305F8443CD6
:10A9700000F101008642B6DCD5E700283FF465AF60
:10A9800014A800EBD60206F0070407FA04F312F845
:10A99000441C43EA010002F8440C06F10106AE42F1
:10A9A000FFF653AF71E700BF2DE9F04F2DED028B9D
:10A9B00087B008EE100A0C4617469946129E139966
:10A9C000B5EEC08AF1EE10FA54BF00250125A84665
:10A9D00004F1FF33D8B2082807D8092A05D8A246BF
:10A9E00001F1FF32944205D808E001F1FF339C42A7
:10A9F00040F2CD8001F1FF34E4B2C8E018EE100A55
:10AA00000BF01AFE48B930464FF03F0122460CF0D9
:10AA1000FFFB4FF000013155C4E018EE100A0BF0B7
:10AA200077FE06EE900AF2EE047AF4EEE76AF1EEB3
:10AA300010FA0DDB4FF00100B0EE677A00F1010073
:10AA400067EE877AF4EEE76AF1EE10FAF6DA03E0E1
:10AA50004FF00100F2EE047A21464319A34200F3BD
:10AA60009680C0EB040EC5EB0E0202F1FF3E4AF6E3
:10AA7000B00AC0F6030ADFED9C4AF6EE003AB2EEE9
:10AA8000044AC0EB040CC5EB0C0303F0010BBEF150
:10AA9000000F00F38F808AE0BEF1000F04DDBE4599
:10AAA000B4BF72463A4601E04FF000025AF8223035
:10AAB00003EE103AB8EE430A20EE027AB4EEE47ADE
:10AAC000F1EE10FA48BF37EE237ABDEEC73A13EE27
:10AAD00010CABCFBF3FB06EE10BAB8EEC65AB4EED1
:10AAE000E75AF1EE10FA0DDB00F1010C87EE006A77
:10AAF00067EE847A0EF1FF3E6046BEF1000200F37D
:10AB0000C380BEE013EE105AB5FBF3F403FB1454FC
:10AB10002CB916EE107A002F08BF4FF00008B9F1DB
:10AB2000000F07D0C8EB0103181A002A18BF01381C
:10AB3000831A01E04FF0000301F10101B8F1000FA9
:10AB400004D04AF62467C0F6030703E048F690678E
:10AB5000C0F6030722B14AF62860C0F6030003E0FE
:10AB600048F69060C0F603004AF63C65C0F603055F
:10AB7000009501978DED026A03900492059430468A
:10AB80004AF62C62C0F603020BF00CFF0AE03046D6
:10AB9000002D0CBF2B212D2122460CF039FB4FF04C
:10ABA0000000305507B0BDEC028BBDE8F08F4FF0D0
:10ABB000000203E0BE45B4BF72463A465AF822305E
:10ABC00000EE103AB8EE405A65EE260AF4EEE40ABA
:10ABD000F1EE10FA48BF70EEA30ABDEEE03A13EEB4
:10ABE00010CABCFBF3FC06EE10CAF8EEC65AF4EE2F
:10ABF000E75AF1EE10FA85DB00F1010080EE852ABC
:10AC000067EE847A0EF1FF3E42199142BFDBBBF141
:10AC1000000F3FF441AFBEF1000F02DC4FF0000225
:10AC200003E0BE45B4BF72463A465AF8223001EE00
:10AC3000103AF8EE411A21EE822AB4EEE42AF1EE3F
:10AC400010FA48BF32EE232ABDEEC23A13EE10BA14
:10AC5000BBFBF3FB06EE10BAF8EEC62AF4EEE72AC9
:10AC6000F1EE10FAFFF64EAF00F1010082EE212A5C
:10AC700067EE847A0EF1FF3E43199942BFF60CAF9E
:10AC800085E74FF0000202E0BA42A8BF3A465AF800
:10AC9000223006EE903AF8EE660A20EE861AB4EEFE
:10ACA000E41AF1EE10FA48BF31EE231ABDEEC13AB4
:10ACB00013EE10BABBFBF3FB06EE10BAF8EEC65A61
:10ACC000F4EEE75AF1EE10FAFFF61CAF0CF10100BA
:10ACD00081EE202A67EE847A0EF1FF3E42199142FE
:10ACE000BFF6DAAE53E700BF0000004BF8B50546EB
:10ACF0000F46F5F75BFA064640F2A062C1F2000289
:10AD00004FF4117303FB05F01418115811B18A6840
:10AD10002846904784F820724FF00005C4F810527E
:10AD2000C4F81452C4F80451C4F808513046F5F779
:10AD300047FA04F5097029464FF00802F5F7F0F9D3
:10AD4000F8BD00BF70B588B0054640F2A064C1F2FE
:10AD500000044FF4117303FB004494F82002002810
:10AD600047D042F24C01C2F201010878FF2803D01B
:10AD70004FF00401FFF7BAFF28464FF00001FFF73C
:10AD8000B5FF42F24C06C2F2010635704AF6486041
:10AD9000C0F603004FF007014FF6E162C0F6020271
:10ADA000FBF71CFDC4F81C02246830784FF0010248
:10ADB00000924FF00002019248F6C173C0F6020300
:10ADC000029349F2B951C0F60201039149F2D94305
:10ADD000C0F60203049349F22131C0F60201059145
:10ADE000069264684FF416514FF00803A047FEF72F
:10ADF000C9F908B070BD00BF704700BF08B5B0F119
:10AE0000FF3F04D040B90246F6F764FE08BD4FF09C
:10AE100000000246F6F75EFE08BD00BF38B505F03B
:10AE2000F1FC42F24D03C2F201034FF001021A702D
:10AE30004FF000042546E0B229462A46FFF724FADF
:10AE400040B904F10104E0B229462A46FFF71CFA92
:10AE5000002867D04FF0FF304FF00001FFF7CEFF22
:10AE60004FF000004FF00001FFF77EFA42F2AC1104
:10AE7000C2F201010C6834B12368DA6802B190476C
:10AE80006468002CF8D142F24400C2F20100046868
:10AE90003CB121680B680BB1A06898476468002C2E
:10AEA000F7D1FAF7ADFBFEF75DFA40F2A062C1F20E
:10AEB000000292F82002042806D028B14FF00000CA
:10AEC0004FF00401FFF712FF40F2A061C1F2000150
:10AED00091F86434042B06D02BB14FF001004FF0F1
:10AEE0000401FFF703FF40F2A062C1F2000292F8F2
:10AEF000A806042806D028B14FF002004FF0040144
:10AF0000FFF7F4FE40F2A061C1F2000191F8EC38C5
:10AF1000042B06D02BB14FF003004FF00401FFF7D4
:10AF2000E5FE38BD04F10104B4F5807F83D191E7DB
:10AF300038B5054642F23004C2F201042068FBF73E
:10AF400037FD4FF0000323608DB14AF65860C0F61C
:10AF500003004FF007014BF26502C0F60202FBF757
:10AF60003DFC42F23802C2F20102106038BD42F2EA
:10AF70003804C2F201042068FBF71AFD4FF000000C
:10AF80002060FAF7F1FEFFF749FF0AF01BF942F2E1
:10AF90004C01C2F201010878FF2803D04FF00401F0
:10AFA000FFF7A4FE38BD00BF70B542F27800C2F2D0
:10AFB00001004AF66861C0F60301FBF73FF842F270
:10AFC0004C03C2F201034FF0FF021A7040F2A0647A
:10AFD000C1F200044FF0040684F820624FF000052F
:10AFE000C4F81C522846FBF713FA206084F8646406
:10AFF000C4F860544FF00100FBF70AFAC4F84402A9
:10B0000084F8A866C4F8A4564FF00200FBF700FAD3
:10B01000C4F8880484F8EC68C4F8E8584FF00300DA
:10B02000FBF7F6F9C4F8CC0641F6F070C2F2010065
:10B030004AF67461C0F60301FBF700F842F25000D3
:10B04000C2F201004AF2A471C0F603012A462B465F
:10B05000FEF7FEFFFDF7B0FE4FF00100FFF768FFBF
:10B0600070BD00BF2DE9F04F2DED0A8BABB01CAFCA
:10B0700026AC4AF21475C0F6030595E80F0084E883
:10B080000F00A76048F64553C0F60203E360204670
:10B090002AA9F8F791F922AE95E80F0086E80F008B
:10B0A000B76048F66150C0F60200F06030462146B5
:10B0B000F8F782F94FF000041B9441F6F070C2F2E9
:10B0C00001002146FAF7D2FF42F26401C2F2010107
:10B0D0000C72FFF7A3FE0AF075F84FF00200FFF7BD
:10B0E00031FE42F2A412C2F2010215680DBB0DF04E
:10B0F0004BFEF0B9F6F744F910F0C20F19D14FF03A
:10B100000300FEF749FC4FF47A754FF032063046E3
:10B11000FBF7A2FBF6F734FA05F1FF343046FBF7F4
:10B120009BFBF6F72DFA651EF1D14FF00000FEF7FC
:10B1300033FC42F2B013C2F201034FF000041C6072
:10B140004FF00100187040F2A066C1F2000606F54B
:10B1500015652846214642F654220CF059F841F66E
:10B16000F060C2F2010021464FF480720CF050F8FA
:10B1700006F5116021464FF040020CF049F842F20A
:10B18000A000C2F2010021464FF0FC020CF040F892
:10B1900021954FF00A01C6F8741920462946FDF79B
:10B1A0006DFD42F22802C2F20102146042F23C0339
:10B1B000C2F201031C6042F2A415C2F201054FF075
:10B1C00030042C6040F20004C0F6010494F82F0013
:10B1D00000F1010094F82E1000EB0122101942F248
:10B1E0009C13C2F201031860FBF7B0FF0B902B68B1
:10B1F000E15CFF2930D142F26400C2F201004FF05D
:10B20000010101720360219A106A18B100F1010076
:10B2100052F8203042F26401C2F201014B604FF05B
:10B22000FF024A7242F23800C2F201004FF00003FE
:10B23000036042F24C01C2F20101087840F2A062C0
:10B24000C1F200024FF4117303FB0021D1F81C027C
:10B25000FBF76CF904F00EBE05F0B2FA4FF00007F0
:10B260000A97BA463C46DFEDC38A9FEDC39ADFEDED
:10B27000C3AA9FEDC38ADFEDC39A9FEDC3AA01E085
:10B280004FF000042CB94FF00000FEF747FC4FF0E0
:10B29000640404F1FF3442F2B016C2F201063578BC
:10B2A00005F0F7026FF30412327042F2A410C2F2FA
:10B2B00001000368099342F2A416C2F2010640F2AB
:10B2C0000007C0F6010742F2B018C2F201084AF6C0
:10B2D000D809C0F6030931687D5C01F101013160D4
:10B2E00098F8002012F0010F0ED10AF1010A40F285
:10B2F000FF30824508D942F26403C2F201034FF0E5
:10B300003601197204F06EBD0DF1700C28464946E5
:10B31000FEF770F94BF27043C0F6030353F8252093
:10B320004BF2E02BC0F6030B42F0010108473268F4
:10B33000B85C0C9002F1010232600F2804F24A85D9
:10B340000DF1700C5946FEF755F94AF26473C0F6D8
:10B3500003030C9953F82120E6E73268B85C0C909F
:10B3600002F101023260102802D9054604F033BD13
:10B370000DF1700C0C984BF67001C0F60301FEF74E
:10B3800039F94BF29803C0F603030C9953F82120C6
:10B39000CAE73268B85C0C9002F1010232600F28F3
:10B3A00002D9054604F017BD0DF1700C0C984AF255
:10B3B0002471C0F60301FEF71DF94BF22033C0F6ED
:10B3C00003030C9953F82120AEE73268B85C0C9067
:10B3D00002F1010232602F2802D9054604F0FBBCBD
:10B3E0000DF1700C0C984AF6D871C0F60301FEF707
:10B3F00001F94AF61053C0F603030C9953F82120C3
:10B4000092E73268B85C0C9002F1010232603B288E
:10B4100002D9054604F0DFBC0DF1700C0C984BF21C
:10B42000DC01C0F60301FEF7E5F84BF6B403C0F605
:10B4300003030C9953F8212076E73268B85C0C902E
:10B4400002F1010232603F2802D9054604F0C3BC74
:10B450000DF1700C0C984BF2E011C0F60301FEF7F1
:10B46000C9F84AF2B073C0F603030C9953F82120CF
:10B470005AE73268B85C0C9002F10102326043284E
:10B4800002D9054604F0A7BC0DF1700C0C984BF2E4
:10B490006031C0F60301FEF7ADF84AF6C863C0F6A6
:10B4A00003030C9953F821203EE7219F97F846604B
:10B4B0000DF1700CFDF744FB219D301895F85030CC
:10B4C00003F0010142181C9285F84720FF2A94BF1F
:10B4D0000022012285F85020D4E6219F97F846608B
:10B4E0000DF1700CFDF72CFB35181C95219880F898
:10B4F0004750FF2D94BF0025012580F85050C1E62C
:10B500000DF1700CFDF71CFB30B1219991F847202B
:10B51000131C18BF012301E04FF00003219F87F89F
:10B520004730AFE60DF1700CFDF70AFB219E96F84F
:10B530004750284086F84700A4E61D98A0F1FB007C
:10B540001C9013E11D9BA3F1FB031C939BE11D9930
:10B55000A1F1FB011C91CCE11D9AA2F1FB021C920E
:10B5600068E21D9EA6F1FB061C964FF002001B90A0
:10B5700000E200BF00000034FFFF7F4BFFFF7FCBE6
:10B5800000000000FEFFFFCAFEFFFF4A1D9BA3F163
:10B59000FB031C931E991B911DE21D9AA2F1FB0255
:10B5A0001C9217E11D9EA6F1FB061C9699E21D98C0
:10B5B000A0F1FB001C90D5E21D9FA7F1FB071C9793
:10B5C0001E9B1B9312E31D99A1F1FB011C911E9A76
:10B5D0001B924FF000068DF86A60C0E31D98A0F141
:10B5E000FB001C901E9B1B934FF001018DF86A100D
:10B5F000B5E31D9AA2F1FB021C9200F04DBC1D9D0B
:10B60000A5F1FB051C9500F0A2BC9DF874004FF05D
:10B610000101FEF7F7FD8DF86B0000283FF432AE14
:10B6200042F26404C2F20104207204F0DBBB1D9EEE
:10B630001C964FF001038DF86A301E46219890F851
:10B6400047100B4205D09DF870003146FEF7DAFD39
:10B6500068B99DF86A304FEA43008DF86A001C9A79
:10B6600002F101021C9210F0FE03E7D10CE09DF8FC
:10B670006A60012E08D19DF86B4042F26401C2F26B
:10B6800001010C7204F0AEBB0DF1700CFDF758FA1D
:10B69000F8E59DF8740005F085F8F3E50DF1700C00
:10B6A000FDF74EFA1C9042F2A416C2F20106306871
:10B6B0001C9900EB41023260FDF758FA1C9001F032
:10B6C000DDBC1D98FA2808D942F26406C2F20106D0
:10B6D0004FF01304347204F085BB41F6F062C2F2FD
:10B6E0000102135C1C93DEE7219991F852001C9033
:10B6F000D9E7219A92F850301C93D4E74FF0000A12
:10B70000C0E50DF1700CFDF71BFA1C90219F97F816
:10B7100047101B91FDF7CAFA87F84700B2E5219D53
:10B7200095F8470095F84610FDF7C0FA85F85000E7
:10B73000A8E50DF1700CFDF72BFA1E9B41F6F066A3
:10B74000C2F20106F05C1D9920EA0102F25499E56B
:10B7500042F2A000C2F201004FF000014FF0FB02E4
:10B760000BF056FD8EE54FF000031C930DF1A80C75
:10B770001CF8386DFDF7E4F90146304607F078FE15
:10B780008DF86B0000283FF47DAD42F26404C2F2F4
:10B790000104207204F026BB06F0FCF972E506F005
:10B7A00001FA8DF86B0000283FF46CAD42F26401A1
:10B7B000C2F20101087204F015BB42F29C17C2F2FA
:10B7C00001073D681D98281806F0D8F95AE54FF092
:10B7D00000021C921C9B40F2A066C1F200064FF4CE
:10B7E000117101FB036090F82022032A3FD140F23F
:10B7F000A067C1F2000701FB03F303F58876B919CE
:10B80000FB1803F104034FF00000D1F80021FE2AD9
:10B8100094BF551C0025D1F80471BD4214BF00250A
:10B82000012565F30000BA4214BF0022012262F331
:10B830004100D3F80051FE2D94BF013500250DF1D4
:10B84000A80C4CF8385DD3F80461B54214BF00254C
:10B85000012565F38200D3F80811D1F1010338BF47
:10B86000002363F3C300C0B2FDF752F90AE542F2C8
:10B870006404C2F201044FF04803237204F0B2BA28
:10B880004FF000001C901C9E40F2A062C1F200022A
:10B890004FF4117101FB062393F8200203281CD1F9
:10B8A00040F2A067C1F2000701FB0675D5F810222F
:10B8B000D5F81412531AB3F5807F88BF03F580734F
:10B8C0001C931C98FF2884BFFF201C900DF1A80C2E
:10B8D0001CF8380DFDF71CF9D4E442F26404C2F2FE
:10B8E00001044FF04806267204F07CBA4FF00006BF
:10B8F0001C961C9B40F2A062C1F200024FF4117131
:10B9000001FB032090F82062032E24D140F2A067AF
:10B91000C1F2000701FB037505F58876D6F8002112
:10B92000D6F80411501AB0F5807F88BF00F58070FA
:10B930001C900DF1700CFDF703F98DF86A001C9B4B
:10B94000984238BF1C90D6F804711C9DEA19D1B2F8
:10B95000C6F8041196E442F26404C2F201044FF006
:10B960004803237204F03EBA4FF000061C964FF0D5
:10B9700002001B901C9B40F2A062C1F200024FF437
:10B98000117101FB032696F82002032815D140F21D
:10B99000A067C1F2000701FB03750DF1700C1B9845
:10B9A00048F6C141C0F6020148F6D542C0F602028F
:10B9B00005F58873FDF7FEF864E442F26404C2F210
:10B9C00001044FF04803237204F00CBA4FF0000258
:10B9D0001C921D991B911C9E40F2A060C1F20000B8
:10B9E0004FF4117303FB060292F82012032915D1BC
:10B9F00040F2A067C1F2000703FB06750DF1700C61
:10BA00001B9848F6C141C0F6020148F6D542C0F67F
:10BA1000020205F58873FEF715F933E442F2640477
:10BA2000C2F201044FF04806267204F0DBB94FF071
:10BA300000001C901C9B40F2A062C1F200024FF477
:10BA4000117101FB032696F8200203283DD140F234
:10BA5000A067C1F2000701FB037505F588750DF1BC
:10BA6000700CFDF76DF88DF86A00D5F804211C9272
:10BA70004FF000011B91D5F800711346974207D093
:10BA8000AE5C864219D04FF001024FF0000E0CE080
:10BA90004FF0FF001B9010E002F10106E95C8142CB
:10BAA00002D11C931B9208E03246FF2B14BF0133D6
:10BAB00073469F42F0D11C93EAE70DF1700C9DF89C
:10BAC0006C00FDF725F8FFF7DDBB42F26404C2F21B
:10BAD00001044FF04803237204F084B94FF00003CF
:10BAE0001C931C9E40F2A062C1F200024FF411713F
:10BAF00001FB062090F82032032B27D140F2A065ED
:10BB0000C1F2000501FB065707F58875D7F81462E6
:10BB1000D7F81022964212D00DF1700CFDF710F8F4
:10BB20008319DFB21C970DF1700CE85DFCF7F0FF94
:10BB30004FF00005219E86F85050FFF7A3BB4FF051
:10BB40000101219880F85010FFF79CBB42F2640479
:10BB5000C2F201044FF04806267204F043B94FF0D8
:10BB600000021C921C9840F2A063C1F200034FF443
:10BB7000117101FB003696F82022032A28D140F2E9
:10BB8000A067C1F2000701FB007505F58876D6F8BD
:10BB90000431D6F800118B4213D00DF1700CF05C1B
:10BBA000FCF7B6FFD6F80471FF2F14BF013700274A
:10BBB000C6F804714FF00005219E86F85050FFF73B
:10BBC00061BB4FF00102219880F85020FFF75ABB6B
:10BBD00042F26404C2F201044FF04800207204F003
:10BBE00001B94FF000031C931D991B9142F29C1266
:10BBF000C2F20102D2F800801B9F08EB070640F258
:10BC00000000C0F60200864208D942F26406C2F281
:10BC100001064FF01F02327204F0E4B81C9B032BA4
:10BC200008D942F26400C2F201004FF037030372F8
:10BC300004F0D8B8F1780D2908D942F26404C2F2B0
:10BC400001044FF03701217204F0CCB840F2A06536
:10BC5000C1F200054FF4117202FB035090F820323C
:10BC60003BB118F8071021B10FE04846FDF756FF29
:10BC700005E04CF24F354FF09609DDF82CB0FBF79C
:10BC800065FACBEB0002AA42EFD918F80770032F30
:10BC90003FF6F8AADFE807F002080F169DF87000DB
:10BCA000FFF750F8FFF7EEBA9DF87000314607F045
:10BCB00001FCFFF7E7BA9DF87000314605F0C6FEBB
:10BCC000FFF7E0BA9DF87050B77828464FF00301AF
:10BCD000FFF70CF84FF4117000FB05F340F2A06180
:10BCE000C1F20001C85800283FF4CCAA4BF2CC1393
:10BCF000C0F6030307EB470703EB0708F6784AF69D
:10BD0000D842C0F6030252F82610DA5D98F80130E6
:10BD100098F8027000974FF00006019649F29107DB
:10BD2000C0F60207029749F2D107C0F6020703974F
:10BD300049F20117C0F60207049749F22137C0F60D
:10BD400002070597069646682846B047FFF79ABA55
:10BD50004FF000011C911D981B908DF86A101C98E3
:10BD600040F2A063C1F200034FF4117101FB0036F1
:10BD700096F82022032A79D140F2A065C1F200058D
:10BD800001FB005707F5887942F29C13C2F20103C8
:10BD90001968219EB26B01EB020B8B5CFF2B5CD010
:10BDA000D8464FF001054FF0000B0994CDF830A0B4
:10BDB000AA4698F8014004EB032742F29C13C2F212
:10BDC00001031E68F219D9F804111C919DF86A004C
:10BDD00018B1F75D02F1010200E05F4602F1FF34A5
:10BDE0009DF86A502DB177B9099C5046DDF830A016
:10BDF00005E063783BB9099C5046DDF830A01C99FA
:10BE0000C9F804112BE01C99D9F800618E4218D0B2
:10BE100014F8016F19F801501B9A3AB930460AF02C
:10BE200065FDC6B228460AF061FDC5B2AE4208D132
:10BE30001C98FF2814BF013058461C9007F1FF37AB
:10BE4000CEE70AF1010A18F8023FFF2BB1D1099C95
:10BE5000DDF830A04FF0000001E04FF000000DF1E0
:10BE6000700CC0B2FCF754FEFFF70CBA42F2640447
:10BE7000C2F201044FF04800207203F0B3BF4FF04C
:10BE800000031C931E9E1B964FF001028DF86A2042
:10BE900065E74FF000021C921C9E40F2A060C1F2C8
:10BEA00000004FF4117303FB060191F82022032ACE
:10BEB00031D140F2A065C1F2000503FB065707F53A
:10BEC00088750DF1700CFCF73BFE8DF86A004FF0A1
:10BED00000031C93D5F80471D5F800118F4212D0DD
:10BEE000EA5D82420FD14FF00006FF2F14BF0137E9
:10BEF0003746B94202D1C5F8047104E0EB5D8342D4
:10BF0000F3D0C5F804710DF1700C4FF00000FCF790
:10BF1000FFFDFFF7B7B942F26404C2F201044FF02B
:10BF20004806267203F05EBFFBF710F90B9D401B1D
:10BF30000DF1700C4CF24F37B8428CBF002001203D
:10BF4000FCF7E6FDFFF79EB94FF000001C901C9E29
:10BF500040F2A062C1F200024FF4117101FB06230E
:10BF600093F82052032D7FF48DA940F2A067C1F20F
:10BF7000000701FB067000F10406D0F80811D6F89E
:10BF8000002102F10102914238BF01F580718B1A44
:10BF9000FF2B34BF1D46FF250DF1700CE8B2FCF7F6
:10BFA000B7FDFFF76FB91D9F41F6F060C2F20100C7
:10BFB000C65D06F1FF31C155FFF764B91D9BFA2B31
:10BFC00008D942F26404C2F201044FF01300207257
:10BFD00003F008BF41F6F060C2F20100C25C02F15A
:10BFE000FF36F1B2C15400293FF44CA91E9B1C93AB
:10BFF00001F044B81D9EFA2E08D942F26404C2F240
:10C0000001044FF01306267203F0ECBE41F6F06116
:10C01000C2F201018A5D02F1FF33D8B288550028CF
:10C0200042F03584FFF72EB91D9BFA2B08D942F256
:10C030006404C2F201044FF01303237203F0D2BE72
:10C0400041F6F061C2F20101CA5C02F1FF30C6B2F2
:10C05000CE54002E02F01B84FFF714B9219D95F8F1
:10C06000517007F1FF3185F85110FFF70BB9219896
:10C0700090F8472002F1FF3680F84760FFF702B9D9
:10C08000219BD86C0AF044FB219DE864FFF7FAB8C5
:10C09000219F97ED137AD7ED127A37EE270A87EDB5
:10C0A000130A2199C86C0AF0A7FA30B14FF00205C3
:10C0B000219981F85050FFF7E5B8219BD86C0AF020
:10C0C000ABFA30B14FF00102219880F85020FFF711
:10C0D000D9B84FF00006219F87F85060FFF7D2B81B
:10C0E0009DF87400219901F14C01FEF709F98DF8D2
:10C0F0006B0000283FF4C6A842F26404C2F20104B7
:10C10000207203F06FBE9DF874002199C96CFEF790
:10C110002BF98DF86B0000283FF4B4A842F26402BA
:10C12000C2F20102107203F05DBE2198C06C0AF0E9
:10C1300073FA20B9219EB06C0AF06EFA30B14FF05C
:10C140000300219E86F85000FFF79CB8219BD3ED99
:10C1500013BA93ED12BA7BEECB0A10EE900A0AF0F6
:10C16000D7FA0CEE100A1BEE900A1BEE101A0AF01A
:10C1700069FA01464FF07E500AF064FA01EE100AA7
:10C1800061EE281AB4EEE1CAF1EE10FA06D84FF0CB
:10C190000001219A82F85010FFF774B8219D95EDA7
:10C1A000132AD5ED122AB4EEE22AF1EE10FA05DDDB
:10C1B0004FF0010785F85070FFF764B8B4EEE22A3B
:10C1C000F1EE10FA4CBF0222032285F85020FFF74F
:10C1D00059B8219B93ED133AF7EE003A33EE634AD8
:10C1E00083ED134A2198C06C0AF016FA30B14FF073
:10C1F0000307219981F85070FFF744B8219A92ED16
:10C2000013BA7BEE49BA1BEE900A0AF081FA0BEEE4
:10C21000900A1BEE100A19EE101A0AF013FA0146E2
:10C220004FF07E500AF00EFA00EE100A60EE280A77
:10C23000F4EEE0BAF1EE10FA1ED9219E96ED13BA93
:10C240003BEE091A11EE100A0AF062FA0BEE900AA0
:10C250001BEE100A1AEE901A0AF0F4F901464FF09C
:10C260007E500AF0EFF901EE900A21EEA82AF4EED2
:10C27000C2BAF1EE10FA06D84FF00406219B83F8FB
:10C280005060FEF7FFBF219BDF6C38460AF040FA92
:10C290000BEE100A384618EE101A0AF0D3F90146D0
:10C2A0004FF07E500AF0CEF902EE900A22EEA83A44
:10C2B000B4EEC3BAF1EE10FA06D84FF00000219A9E
:10C2C00082F85000FEF7DEBF2199D1ED133AF4EE6B
:10C2D000C83AF1EE10FA05DD4FF0010581F8505033
:10C2E000FEF7D0BFF4EEC83AF1EE10FA4CBF0222CE
:10C2F000032281F85020FEF7C5BF219DD5ED124ADB
:10C3000095ED135AC4EE855AC5ED135AC9E6219925
:10C31000C86C0AF06DF9002840F0AE86FEF7B2BF97
:10C32000219AD66C30460AF0F3F90BEE100A30462B
:10C3300018EE101A0AF086F901464FF07E500AF006
:10C3400081F906EE100A66EE286AB4EEE6BAF1EE5E
:10C3500010FA00F39186FEF795BF2198C06C0AF0A1
:10C3600047F9002800F08886FEF78CBF219B93EDEB
:10C37000137AD3ED127AB4EEE77AF1EE10FA80F286
:10C380007B86FEF77FBF219991ED130AD1ED120A4A
:10C39000B4EEE00AF1EE10FA00F36E86FEF772BF1B
:10C3A000219A92ED131AD2ED121AB4EEE11AF1EEBF
:10C3B00010FA40F26186FEF765BF219E96ED132AC2
:10C3C000D6ED122AB4EEE22AF1EE10FA00F154860C
:10C3D000FEF758BF2198C66C30460AF099F90BEE6B
:10C3E000100A304618EE101A0AF02CF901464FF0E8
:10C3F0007E500AF027F903EE100A63EE283AB4EEF5
:10C40000E3BAF1EE10FA40F23786FEF73BBF219F08
:10C41000F86CFCF7CDF9F8640DF1700C4FF00000EA
:10C42000FCF762FCFEF72EBF1D9BF62B08D942F2EB
:10C430006404C2F201044FF01203237203F0D2BC71
:10C44000219DE86C0AF0D4F838B9219AD2ED134A4C
:10C45000B6EE005A34EE85BA06E0219991ED13BA92
:10C46000B6EE004A3BEE44BA1BEE100A0AF0C0F8E2
:10C4700088B9B4EECABAF1EE10FA04DC1BEE100A69
:10C480000AF0BAF838B14FF00100219E86F850004A
:10C490006FF000402CE01BEE100A0AF0A9F888B1FA
:10C4A000B4EEE9BAF1EE10FA04D41BEE100A0AF069
:10C4B000A3F838B14FF00101219A82F850104FF0E3
:10C4C000004015E01BEE100A0AF0A6F838B14FF054
:10C4D0000205219B83F850504FF0000008E0BDEEAC
:10C4E000CBBA1BEE100A4FF00006219F87F8506070
:10C4F0004FEA006747EA106500F47F4345EA0321ED
:10C5000000F47F0241EA122042F2A006C2F20106C4
:10C510001D9FF051FEF7B6BE1D99F62908D942F2CB
:10C520006404C2F201044FF01203237203F05ABCF8
:10C5300042F2A005C2F201056A584FEA026040EAE1
:10C54000126602F47F4746EA072302F47F0143EABA
:10C55000112505EE905AB8EEE56A219880ED136A30
:10C56000B4EECA6AF1EE10FA04DCB4EEE96AF1EE58
:10C5700010FA05D54FF0010680F85060FEF782BE34
:10C580004FF0000280F85020FEF77CBE0DF1700CD9
:10C590004FF00100FCF7A8FB219FF86CFCF732F983
:10C5A0002199C864FEF76EBE219DD5ED136AB7EEE2
:10C5B000007A76EE877AC5ED137A13E6219DE86C52
:10C5C0000AF02AF850B1219F4FF0000187F8471078
:10C5D0004FF0040587F85050FEF754BE219890EDB7
:10C5E000134AB4EEC84AF1EE10FA23DB9FEDD66A87
:10C5F000B4EEC64AF1EE10FA0FD5FCEEC46A16EEA0
:10C60000902A0DF1700CD0B2FCF782FA4FF00006C0
:10C61000219B83F85060FEF735BE0DF1700C4FF092
:10C62000FF00FCF775FA4FF00205219880F8505092
:10C63000FEF728BEB4EEC84AF1EE10FA7EF522AE3F
:10C64000DFEDC24AB4EEE44AF1EE10FA11DDB1EECC
:10C65000445AFCEEC55A15EE903A0DF1700CD8B262
:10C66000FCF756FA4FF00107219981F85070FEF758
:10C6700009BE0DF1700C4FF0FF00FCF749FA4FF0C6
:10C680000302219E86F85020FEF7FCBD1D98F92874
:10C6900008D942F26404C2F201044FF01300207280
:10C6A00003F0A0BB219A92ED137AFDEEC77A17EE44
:10C6B000906A33B21C939FB2C6F3072141EA072563
:10C6C00041F6F062C2F201021552FEF7DBBD1D9E7B
:10C6D000F92E08D942F26404C2F201044FF01306A5
:10C6E000267203F07FBB219B93ED130AFCEEC00A78
:10C6F00010EE907ABDB21C954FEA152141EA052251
:10C7000041F6F060C2F201008253FEF7BBBD1D9FEF
:10C71000219B9F64FEF7B6BD1D9D2199CD64FEF758
:10C72000B1BD0DF1700CFCF70BFA01EE100AF8EE3A
:10C73000411A219AC2ED131AFEF7A4BD1D98F928DB
:10C7400008D942F26404C2F201044FF013002072CF
:10C7500003F048BB41F6F066C2F20106375A4FEAD1
:10C76000172343EA0725A9B202EE101AF8EE422A6F
:10C77000219AC2ED132A9FED763AF4EEC32AF1EE28
:10C7800010FAFEF67FADDFED733A32EEE34A82ED4A
:10C79000134AFEF777BD1D9EF92E08D942F26404B4
:10C7A000C2F201044FF01306267203F01BBB41F6E0
:10C7B000F067C2F20107BB5B4FEA132545EA03218C
:10C7C0008AB204EE902AB8EE645A219880ED135A8A
:10C7D000FEF758BD1D98072808D942F26403C2F23B
:10C7E00001034FF00801197203F0FCBAFCF7FCFDDD
:10C7F00005EE900AB8EE656A219F87ED136AFEF791
:10C8000041BD219DD5ED136A95ED127A66EE877ACA
:10C81000C5ED137A45E4219A92ED130AF1EE400A30
:10C82000C2ED130AFEF72EBD4FF000004FF00101DC
:10C830000A46FDF729FD219890ED131AF1EE041A2E
:10C8400021EE212A4FF000060096019642F2B41024
:10C85000C2F20100FCEEC22A12EE901A4FF0FF0263
:10C860004AF2ED23C0F60203FAF73AFCFEF70ABDDE
:10C870001D9BF72B08D942F26404C2F201044FF069
:10C880001302227203F0AEBA41F6F067C2F201075A
:10C89000F858FBF7B7FF21998864FEF7F3BC1D98A1
:10C8A000F72808D942F26403C2F201034FF01301E2
:10C8B000197203F097BA41F6F065C2F201052858E3
:10C8C000FBF7A0FF219EF064FEF7DCBC1D9A072A4F
:10C8D00008D942F26404C2F201044FF0080626723D
:10C8E00003F080BA219F97ED133AB4EEC83AF1EE07
:10C8F00010FA0DDBB4EEC93AF1EE10FA08D8FCEEEE
:10C90000C33ACDED1C3A4FF0000587F8505028E0AF
:10C91000B4EEC93AF1EE10FA07DD6FF07F421C92D7
:10C920004FF0010087F850001BE04FF000001C9012
:10C9300013EE100A09F05CFE70B14FF00201219B6A
:10C9400083F850100DE000BF00008043000080C35A
:10C9500000000047800080474FF00305219E86F8C5
:10C9600050501D981C99FCF711FDFEF78BBC219FC0
:10C97000F86C09F051FE00287EF484AC219991ED09
:10C98000134AB4EEC84AF1EE10FA04DD4FF07E52BD
:10C99000CA64FEF777BCB4EEC84AF1EE10FA7EF531
:10C9A00071AC4FF00003CBF68073CB64FEF76ABC2A
:10C9B0002198856ACDB1FAF7C9FB219FB96AC1F107
:10C9C000040318184CF6CD42CCF6CC42A2FB00155D
:10C9D0004FEA9506796AB6FBF1F304EE903AB8EEA9
:10C9E000645A87ED135AFEF74DBC4FF6FF76C7F633
:10C9F0007F76C664FEF746BC1D9EF72E08D942F22C
:10CA00006404C2F201044FF01300207203F0EAB98B
:10CA1000219FF86CFBF7CCFE41F6F062C2F20102F6
:10CA20009051FEF72FBC219DD5ED125A95ED136A5A
:10CA300075EEC66AC5ED136AFFF733BB219BDE6C4A
:10CA40001C969F6CDF649E64FEF71CBC219AD06C20
:10CA500009F0E2FD30B14FF00306219981F85060F2
:10CA6000FEF710BC2198C06C09F0C6FD30B14FF044
:10CA70000400219D85F85000FEF704BC219DEE6C5A
:10CA8000304609F045FE0BEE100A304618EE101A3B
:10CA900009F0D8FD01464FF07E5009F0D3FD07EEB6
:10CAA000100A67EE287AB4EEE7BAF1EE10FA06D86B
:10CAB0004FF00007219A82F85070FEF7E3BB2199EE
:10CAC00091ED130AB4EEC80AF1EE10FA05DD4FF04D
:10CAD000010381F85030FEF7D5BBB4EEC80AF1EE81
:10CAE00010FA4CBF0222032281F85020FEF7CABB85
:10CAF000219BD3ED13BA93ED12BA3BEECBCA1CEED9
:10CB0000100A09F005FE0CEE100A1BEE900A1BEE4F
:10CB1000101A09F097FD01464FF07E5009F092FD82
:10CB200000EE900A20EEA81AB4EEC1CAF1EE10FA97
:10CB30000DF1700C8CBF00200120FBF7E9FFFEF720
:10CB4000A1BB219FFD6C284609F0E2FD0BEE100A07
:10CB5000284618EE101A09F075FD01464FF07E5078
:10CB600009F070FD01EE900A21EEA82AB4EEC2BAD7
:10CB7000F1EE10FA0DF1700C8CBF00200120FBF7D4
:10CB8000C7FFFEF77FBB219AD2ED132A92ED123A2E
:10CB9000F4EEC32AF1EE10FA0DF1700CB4BF0020D0
:10CBA0000120FBF7B5FFFEF76DBB2198D0ED133ADE
:10CBB000F5EEC03AF1EE10FA0DF1700CB4BF0020A2
:10CBC0000120FBF7A5FFFEF75DBB219E96ED134A02
:10CBD000D6ED124AB4EEE44AF1EE10FA0DF1700C03
:10CBE000D4BF00200120FBF793FFFEF74BBB219938
:10CBF00091ED135AD1ED125AB4EEE55AF1EE10FA56
:10CC00000DF1700C8CBF00200120FBF781FFFEF7B7
:10CC100039BB219B93ED136AD3ED126AB4EEE66A39
:10CC2000F1EE10FA0DF1700C54BF00200120FBF75B
:10CC30006FFFFEF727BB219F97ED137AB5EEC07A01
:10CC4000F1EE10FA0DF1700C54BF00200120FBF73B
:10CC50005FFFFEF717BB219DD5ED13BA95ED12BA14
:10CC60007BEECB7A17EE900A09F052FD0CEE100A1B
:10CC70001BEE900A1BEE101A09F0E4FC01464FF07F
:10CC80007E5009F0DFFC00EE100A60EE280AB4EED8
:10CC9000E0CAF1EE10FA0DF1700CD4BF00200120B3
:10CCA000FBF736FFFEF7EEBA219AD66C304609F054
:10CCB0002FFD0BEE100A304618EE101A09F0C2FCD8
:10CCC00001464FF07E5009F0BDFC01EE100A61EE06
:10CCD000281AB4EEE1BAF1EE10FA0DF1700CD4BFDF
:10CCE00000200120FBF714FFFEF7CCBA1D98F828AE
:10CCF00008D942F26404C2F201044FF01303237214
:10CD000003F070B8FAF722FA219B00F104004CF608
:10CD1000CD41CCF6CC41A1FB00174FEA97055A6AEA
:10CD2000B5FBF2F71D9D41F6F060C2F2010041191A
:10CD30004E78425D4FEA024545EA0620897840EA8E
:10CD400001061B96BF1B27F07F421C9202EE102AA1
:10CD5000F8EE422AC3ED132AFEF794BA219DE86C3F
:10CD6000A864FEF78FBA219991F85160002E40F027
:10CD70008381FEF787BA219A92F85130002B00F098
:10CD80007B81FEF77FBA1D98FA2808D942F2640425
:10CD9000C2F201044FF01303237203F023B841F6EB
:10CDA000F061C2F201010E5C002E7EF46BAA1E9AA5
:10CDB0001C9263E11D98FA2808D942F26404C2F279
:10CDC00001044FF01303237203F00CB841F6F06135
:10CDD000C2F201010E5C002E3EF454AA1E9A1C926F
:10CDE0004CE142F26400C2F201004FF00101017215
:10CDF00002F0F8BF1D9EF92E08D942F26404C2F277
:10CE000001044FF01206267202F0ECBF42F2A002BB
:10CE1000C2F20102905D1E9B18427EF433AA1F9954
:10CE20001C912BE11D98F92808D942F26404C2F242
:10CE300001044FF01200207202F0D4BF42F2A002AF
:10CE4000C2F20102115C1E9B19423EF41BAA1F9EF6
:10CE50001C9613E11D99FA2908D942F26404C2F222
:10CE600001044FF01300207202F0BCBF41F6F062E3
:10CE7000C2F20102535C002B7EF404AA1E9E1C9693
:10CE80002DE11D99FA2908D942F26404C2F2010485
:10CE90004FF01300207202F0A5BF41F6F062C2F21B
:10CEA0000102535C002B3EF4EDA91E9E1C9616E178
:10CEB0001D99FA2908D942F26404C2F201044FF024
:10CEC0001301217202F08EBF41F6F062C2F201023C
:10CED000565C1E9B9E427EF6D5A91F981C90CDE005
:10CEE0001D9EFA2E08D942F26404C2F201044FF0EA
:10CEF0001306267202F076BF41F6F062C2F201021A
:10CF0000905D1E9B9842FEF4BDA91F991C91B5E04F
:10CF10001D98FA2808D942F26404C2F201044FF0C5
:10CF20001300207202F05EBF41F6F062C2F201020D
:10CF3000115C1E9B99427EF4A5A91F9E1C969DE044
:10CF40001D99FA2908D942F26404C2F201044FF093
:10CF50001301217202F046BF41F6F062C2F20102F3
:10CF6000565C1E9B9E423EF48DA91F981C9085E046
:10CF70001D9EFA2E08D942F26404C2F201044FF059
:10CF80001306267202F02EBF41F6F062C2F20102D1
:10CF9000905D1E9B98423EF675A91F991C916DE00D
:10CFA0001D98FA2808D942F26404C2F201044FF035
:10CFB0001300207202F016BF41F6F062C2F20102C5
:10CFC000115C1E9B9942BEF45DA91F9E1C9655E004
:10CFD000219A92F847101D9B99427EF453A91E9EF8
:10CFE0001C967CE0219890F847201D998A423EF4D7
:10CFF00049A91E9B1C9372E0219E96F847001D9A3A
:10D0000090427EF63FA91E991C9168E0219B93F8FF
:10D0100047601D988642FEF435A91E9A1C925EE078
:10D02000219991F847601D9B9E42BEF42BA91E9842
:10D030001C9054E0219A92F847101D9EB1423EF692
:10D0400021A91E9B1C934AE09DF874000DF16B0111
:10D05000FDF73AF88DF86A009DF86B1031B142F295
:10D060006404C2F20104217202F0BCBE00283EF446
:10D0700009A91E981C9001E01D9A1C921C9A40F26E
:10D080000000C0F6010090F82E1090F82F3043EA0F
:10D090000126964208D242F26404C2F201044FF023
:10D0A0000902227202F09EBE42F2A417C2F20107E8
:10D0B0003A60FEF7E7B80DF1700CFBF741FD1C90EC
:10D0C0000028D9D0FEF7DEB80DF1700CFBF738FD63
:10D0D0001C900028D0D1FEF7D5B81D9E1C96219E2D
:10D0E000336A052B08D942F26404C2F201044FF0FE
:10D0F0000A03237202F076BE03F1020242F2A41088
:10D10000C2F20100016846F8221003F10103219EDA
:10D110003362B3E70DF1700CFBF712FD1C90002891
:10D12000DBD0FEF7AFB80DF1700CFBF709FD1C90DA
:10D130000028D2D1FEF7A6B80DF1700CFBF700FD68
:10D140001C901D9B98427EF49DA81E991C9195E70A
:10D150000DF1700CFBF7F4FC1C901D9A90423EF40C
:10D1600091A81E981C9089E70DF1700CFBF7E8FC64
:10D170001C901D9EB0427EF685A81E9B1C937DE7E9
:10D180000DF1700CFBF7DCFC1C901D998842FEF43D
:10D1900079A81E9A1C9271E70DF1700CFBF7D0FC78
:10D1A0001C901D9EB042BEF46DA81E981C9065E7B1
:10D1B0000DF1700CFBF7C4FC1C901D9B98423EF6D1
:10D1C00061A81E991C9159E79DF874000DF16B013F
:10D1D000FCF74AFF8DF86A009DF86B6036B142F2A9
:10D1E0006404C2F20104267202F0FCBD00283EF481
:10D1F00049A81E9A1C9241E79DF874000DF16B013D
:10D20000FCF732FF8DF86A009DF86B3033B142F2C3
:10D210006401C2F201010B7202F0E4BD00287EF449
:10D2200031A81E981C9029E70DF1700CFBF7B0FC9B
:10D2300041F6F066C2F201061E9AB05C1D9B1842D0
:10D240003EF420A81F991C9118E70DF1700CFBF714
:10D250009FFC41F6F066C2F201061E9AB05C1D9B6F
:10D2600018427EF40FA81F991C9107E70DF1700C6E
:10D27000FBF78EFC41F6F066C2F201061E9AB05C26
:10D280001D9B18427DF4FEAF1F991C9127E70DF1FD
:10D29000700CFBF77DFC41F6F066C2F201061E9AA7
:10D2A000B05C1D9B18423DF4EDAF1F991C9116E731
:10D2B00098F8005045F0080288F80020FEF70BB8F7
:10D2C0000DF1700CFBF73CFC8DF86A00219991F888
:10D2D00051601D9BF1181C911E9AC2F1FB06B142D0
:10D2E00008D942F26404C2F201044FF0130323721E
:10D2F00002F078BD4FF000071B971E99D9B11C9D15
:10D3000041F6F063C2F201035A5D824234D001F16A
:10D31000FF3241F6F066C2F20106731941F6F0677A
:10D32000C2F20107C7F10101C5EB010E12F0010FB6
:10D330001AD002F0C2BD4FF0FF001B901CE013F8A2
:10D34000019F02F1FF36484504D11C95CDF86CC011
:10D350001E9211E03246CD180EEB030C13F8017F3C
:10D36000B84242F0B785F0E7CD180EEB030C002A67
:10D37000E5D11C951E92DEE70DF1700C9DF86C0056
:10D38000FBF7C6FBFDF77EBF0DF1700CFBF7D8FB7A
:10D3900042F2180BC2F2010B8BF800004FF00101B2
:10D3A0001C91CDF834B095E0219E96F851201D983F
:10D3B00013181C93F92B08D942F26404C2F2010439
:10D3C0004FF01301217202F00DBD1E981B900DF15C
:10D3D000700C26AD45F0010122AF47F001024FF07D
:10D3E0000003FBF7E7FBFDF74DBF219E96F85120A8
:10D3F0001D9813181C93FA2B08D942F26404C2F248
:10D4000001044FF01301217202F0ECBC1F9D1E9825
:10D41000A84228BF28461B900DF1700C26AF47F09C
:10D42000010122AE46F001024FF00003FCF70AFCB6
:10D43000FDF728BF0DF1700CFBF782FB034642F2AB
:10D44000180BC2F2010B58464FF010014AF67C62ED
:10D45000C0F6030209F0A6FA1C90CDF834B039E00A
:10D460001E9A1C921F981B904FF000030D9331E001
:10D470004FF0FF361C960D962CE02199C86C9DF854
:10D4800078109DF87C2042F21806C2F20106009640
:10D490004FF0100301934FF00103FDF785FA4FF0B1
:10D4A000FF321C920D9615E02198C06C9DF8781003
:10D4B0009DF87C2042F21806C2F2010600964FF059
:10D4C000100301934FF00003FDF76EFA4FF0FF31A8
:10D4D0001C910D961D9800F10506F2B20C92A0F178
:10D4E000FB01032923D840F2A060C1F200004FF4F1
:10D4F00011760C9A06FB020191F82032032B08D01A
:10D5000042F26400C2F201004FF04806067202F0D7
:10D5100069BC40F2A060C1F200004FF411770C9E8C
:10D5200007FB060707F104074FF0000605E0219FFF
:10D5300097F851301E184FF00007DDF870B0BBF1BE
:10D54000FF3F0CD14FF0FF0B4FF00009C84641F6EA
:10D55000F062C2F201020E920F950D9D05E0BBF143
:10D56000000FF1D14FF0000961E01D99A1F1FB011D
:10D57000032910D8D7F80061FF2E14BF01364646A4
:10D58000D7F804319E4206D14046FCF7C7FAD7F8D7
:10D5900004018642F8D0B5F1FF3F15D1219850F82B
:10D5A000343F1A68D2F800C0494610AA4FF0010370
:10D5B000E0478DF86B0080B10F9D42F26404C2F227
:10D5C0000104207202F00EBC25B115F809108DF887
:10D5D000401002E01B9A8DF840201C98B0F1FF3FEC
:10D5E00002D19DF8401011B31D9BA3F1FB03032B47
:10D5F00007D8D7F800119DF840307B54C7F8006178
:10D6000011E0FA2E09D90F9D42F26404C2F201041E
:10D610004FF01306267202F0E5BB9DF840200E98ED
:10D62000825506F1010609F10109D9459DD31D9FD7
:10D63000A7F1FB07032F04D80C98FBF711FDFDF7AA
:10D6400021BE219D95F8512009EB020E85F851E08D
:10D65000FDF718BE1D9AA2F1FB0003285AD802F16B
:10D660000502D7B240F2A060C1F200004FF4117180
:10D6700001FB070292F82032032B08D042F2640427
:10D68000C2F201044FF04803237202F0ABBB40F238
:10D69000A066C1F200064FF4117505FB076505F1A0
:10D6A00004051E9800F1FF311E9170B34FF0000881
:10D6B00042F2A419C2F2010940F200029346C0F6F8
:10D6C000010BD5F80061FF2E14BF01364646D5F890
:10D6D00004319E4206D14046FCF720FAD5F80401F9
:10D6E0008642F8D0D9F80030D5F800211BF8031095
:10D6F000A95403F10103C9F80030C5F800611E9E6A
:10D7000006F1FF301E90002EDBD13846FBF7A8FC57
:10D71000FDF7B8BD1E9B1C93219991F8510082180A
:10D720001B92C3F1FB06B24208D942F26404C2F272
:10D7300001044FF01306267202F054BBC51881F89D
:10D7400051501C9A02F1FF351C95002A3DF49AAD08
:10D7500042F2A417C2F201073E681B9F41F6F06334
:10D76000C2F20103D91940F20000C0F601003018DE
:10D770004FF0000305F0010E10F803C001F803C0DC
:10D7800003F10103934242F089830DE010F8038016
:10D7900001F8038003F1010310F803E001F803E04E
:10D7A00003F101039342F1D1E819A91901F1010133
:10D7B00042F2A412C2F2010211604FF0FF331C9337
:10D7C00000F101001B90FDF75DBD4FF000028DF8E8
:10D7D0006A20219E96F851001D9BC1181C911E9A2B
:10D7E0001B92C2F1FB00814208D942F26404C2F2EA
:10D7F00001044FF01303237202F0F4BA41F6F0670C
:10D80000C2F2010707EB01099DF87CB042F29C15BA
:10D81000C2F201052A68B66B9119975DFF2F52D0AD
:10D8200088464FF0010009900C9498F8014004EBF1
:10D83000072742F29C15C2F201052A68D6194FF05B
:10D8400000011C919DF86A30002B02F0FD82D75D2B
:10D8500006F1010602F0FABA9DF86A5015B15FB9F7
:10D860000C9C02E062783AB90C9C219E96F85120FB
:10D87000851886F8515029E014F8015F19F800B0B6
:10D8800046B9284609F032F8C5B2584609F02EF8D4
:10D890005FFA80FB5D4508D11C9800F101001C90E7
:10D8A00007F1FF371B998142D6D2B346099B03F19A
:10D8B0000103099318F8027FFF2FB6D10C9C4FF09B
:10D8C0000000099002E04FF0000309930DF1700C85
:10D8D0000999C8B2FBF71CF9FDF7D4BC4FF0010160
:10D8E0008DF86A1075E70DF1700CFBF729F9034606
:10D8F00042F2180BC2F2010B58464FF010014AF6E3
:10D900008462C0F6030209F04DF81C90CDF834B0E3
:10D91000E0E50DF1700CFBF713F9034642F2180B2A
:10D92000C2F2010B58464FF010014AF68C62C0F665
:10D93000030209F037F81C90CDF834B0CAE50DF1B8
:10D94000700CFBF7FDF8034642F2180BC2F2010B14
:10D9500058464FF010014AF69062C0F6030209F0F3
:10D9600021F81C90CDF834B0B4E50DF1700CFBF744
:10D97000E7F8034642F2180BC2F2010B58464FF08B
:10D9800010014AF69862C0F6030209F00BF81C90E9
:10D99000CDF834B09EE5219991F8513003F101039F
:10D9A00081F85130FDF76EBC1D9F41F6F065C2F263
:10D9B0000105EA5D02F10102EA55FDF763BC219819
:10D9C00090F8476006F1010680F84760FDF75ABC01
:10D9D0009DF874000DF16B01FCF746FB0DF1700C26
:10D9E000FBF796F89DF86B1000293DF44BAC42F222
:10D9F0006404C2F20104217202F0F4B99DF87400CB
:10DA00000DF16B01FCF798FB0DF1700CFBF780F842
:10DA10009DF86B30002B3DF435AC42F26402C2F24B
:10DA20000102137202F0DEB91D981C904FF000063F
:10DA30001B964FF001018DF86A109DF870000DF1F2
:10DA40006B01FCF711FB9DF86B309BB920B19DF881
:10DA50006A201B9810431B909DF86A604FEA4601AC
:10DA60008DF86A101C9B03F101031C9311F0FE0F4B
:10DA7000E3D10AE09DF86A20012A06D142F264044B
:10DA8000C2F20104237202F0ADB90DF1700C9DF8E1
:10DA90006C00FBF73DF8FDF7F5BB1D981C904FF0AF
:10DAA00000061B964FF001018DF86A109DF870007A
:10DAB0000DF16B01FCF740FB9DF86B309BB920B179
:10DAC0009DF86A201B9810431B909DF86A604FEAEE
:10DAD00046018DF86A101C9B03F101031C9311F0A1
:10DAE000FE0FE3D10AE09DF86A20012A06D142F236
:10DAF0006404C2F20104237202F074B90DF1700CD7
:10DB00009DF86C00FBF704F8FDF7BCBB9DF87400B2
:10DB10000DF16B01FCF7D8FA8DF86A009DF86B6087
:10DB200036B142F26400C2F20100067202F05AB944
:10DB30000DF1700CFAF7ECFFFDF7A4BB1D991C91D9
:10DB40004FF000031B934FF001008DF86A00219AFB
:10DB500092F8476030420ED09DF870000DF16B01D5
:10DB6000FCF7B2FA9DF86B1099B920B19DF86A00E4
:10DB70001B9B03431B939DF86A204FEA42068DF8D6
:10DB80006A601C9901F101011C9116F0FE00DED1C2
:10DB90000AE09DF86A30012B06D142F26404C2F219
:10DBA0000104217202F01EB91B9F219D85F8477068
:10DBB000FDF768BB9DF874000DF16B01FCF7ECFA02
:10DBC0000DF1700CFAF7A4FF9DF86B60002E3DF488
:10DBD00059AB42F26402C2F20102167202F002B9BB
:10DBE0001D991C91C8B20DF16B01FCF7D5FA1B9081
:10DBF0009DF86B0030B142F26404C2F2010420725D
:10DC000002F0F0B84FF001038DF86A301C9FFA184B
:10DC10001C92D0B20DF16B01FCF7BEFA9DF86A5070
:10DC200000FA05F01B9E06431B9605F101058DF8D1
:10DC30006A501C9A02F101021C92E9B20729E8D944
:10DC40000DF1700C9DF86C00FAF762FFFDF71ABB3E
:10DC50000DF1700C219890F85100FAF759FFFDF77B
:10DC600011BBFDF70FBB42F24D03C2F201034FF0AF
:10DC700001071F70FDF706BB42F24D05C2F2010518
:10DC80004FF000062E70FDF7FDBA21984FF000010D
:10DC90004FF0540209F0BCFA4FF00002219242F218
:10DCA0002801C2F201010C6804F1FF30086002F0A3
:10DCB00005B842F22802C2F2010211687F2908D990
:10DCC00042F26404C2F201044FF03000207202F00C
:10DCD00089B84FF001071C9740F2A065C1F200051A
:10DCE000D5F8A809002842F0BC8005E0D6F8AC10B1
:10DCF00000294ED11C9301E04FF001031D9840F222
:10DD0000A066C1F200064FF0540505FB03F3F218BC
:10DD1000C2F85009C2F854091E9982F8A2194FF0AE
:10DD20000A07C2F8747906F51567F81800F134008F
:10DD3000219901F134014FF0100209F045FA1C9BC2
:10DD400005FB037000F14400219901F144014FF0FB
:10DD5000040209F039FA1C9805FB007000F1480034
:10DD6000219901F148014FF0080209F02DFA219A9A
:10DD700092F851101C9F05FB076686F8A11942F224
:10DD80002805C2F201052B6803F101032B60FDF7A2
:10DD900079BA03F101073B4606F15406D6F8AC50B8
:10DDA000002D42F07280A5E71C93FDF76BBA219B12
:10DDB00093F852601E967CE70DF1700CFAF7C0FEE6
:10DDC0001E9076E71D9A219981F85120FDF75ABAE5
:10DDD0000DF1700C9DF87400FAF79AFEFDF752BA37
:10DDE000219EB36A002B3DF44DAAF9F7AFF92199B2
:10DDF0008A6A801A4E6A1D9B06FB03F303EB8301BC
:10DE00008842BDF43FAA1E9A1C92FFF737B9F9F772
:10DE10009DF9219FB862FDF735BA42F2A000C2F227
:10DE2000010090F8FB201E9E9319FB2B08D942F2AB
:10DE30006400C2F201004FF01206067201F0D2BF78
:10DE40001D9BC2F1FB018B4208DD42F26404C2F269
:10DE500001044FF01302227201F0C4BF42F2A00588
:10DE6000C2F20105A81941F6F067C2F20107F918DC
:10DE700009F0AAF9FDF706BA98F8003043F010014E
:10DE800088F80010FDF727BA219D95F84770002FFC
:10DE90000CBFFF22002285F84720FDF7F3B9219837
:10DEA00090F847606FEA060380F84730FDF7EAB95B
:10DEB0000DF1700CFAF76CFE1E9D41F6F067C2F290
:10DEC00001077A5D1D9951407955FDF7DBB921981D
:10DED000866B1D9B9A191C92A1E12199C86B8E6BD0
:10DEE00083191C939BE121990A6C42B942F26404A4
:10DEF000C2F201044FF02000207201F073BF02F162
:10DF0000FF350D64FDF7BEB9219E336C03F10103AB
:10DF10003364002B7DF4B6A942F26401C2F2010120
:10DF20004FF020020A7201F05DBF2198466B336802
:10DF3000596841B942F26400C2F201004FF01E0379
:10DF4000037201F04FBF0DF1700CFAF7F9FD1C9050
:10DF5000219850F8342F166876681D991CAA4FF046
:10DF60000103B0478DF86B0000283DF48BA942F205
:10DF70006404C2F20104207201F034BF0DF1700C90
:10DF8000FAF7DEFD1C9038E10DF1700CFAF7D8FDC0
:10DF9000219FF863FDF776B90DF1700CFAF7D0FD0B
:10DFA000219D2864FDF76EB9219850F8341F0A6846
:10DFB00016681D991CAA4FF00103B0478DF86B003D
:10DFC00030B142F26404C2F20104207201F00ABFCF
:10DFD0000DF1A80C1CF8380DFAF79AFDFDF752B9AF
:10DFE0002198436B0DF1700C187AFAF791FDFDF74B
:10DFF00049B90DF1700C219F97F83C00FAF788FDA4
:10E00000FDF740B921990A6CFF2A08D942F264064B
:10E01000C2F201064FF02004347201F0E3BE0DF1AC
:10E02000700CD0B2FAF774FDFDF72CB9219850F8B6
:10E03000345F2B689F68B84703EE100AF8EE433A46
:10E040002198C0ED133AFDF71DB9219991ED0E4AC3
:10E05000F8EE444AC1ED134AFDF714B9219A92ED46
:10E06000105AF8EE455AC2ED135AFDF70BB9219E2E
:10E0700096ED136AFCEEC66ACDED1C6ACFE0219BDB
:10E08000D3ED137A9FEDC17AF4EEC77AF1EE10FA70
:10E0900008DB42F26404C2F201044FF02000207257
:10E0A00001F0A0BEBCEEE70A83ED100AFDF7EAB866
:10E0B000219850F8341F0A6816681D991CAA4FF061
:10E0C0000403B0478DF86B0030B142F26403C2F232
:10E0D0000103187201F086BE1C98FAF793FB219D8C
:10E0E000A864FDF7CFB8219850F8341F0A68166865
:10E0F0001D991CAA4FF00403B0478DF86B0030B196
:10E1000042F26404C2F20104207201F06BBE1C985A
:10E11000FAF778FB219FF864FDF7B4B82198436BB8
:10E1200019684A6842B942F26400C2F201004FF035
:10E130001E01017201F056BEC06CFAF739FB1C904B
:10E14000219850F8346F33685E681D991CAA4FF00F
:10E150000403B0478DF86B0000283DF493A842F209
:10E160006404C2F20104207201F03CBE1D9A2198A1
:10E17000C36BC3F1FB06B24208D942F26404C2F297
:10E1800001044FF01300207201F02CBE50F8347FD0
:10E1900039680E684FF0000141F6F067C2F20107DE
:10E1A000BA18B0478DF86B0000283DF46BA842F216
:10E1B0006403C2F20103187201F014BE219850F8F2
:10E1C000342F11680E681D991BAA4FF00403B04745
:10E1D0008DF86B0030B142F26404C2F20104207287
:10E1E00001F000BE1B9B98B2C3F3072242EA002154
:10E1F0008EB21C9613E01D9B1C931C982199FAF774
:10E200003DFD8DF86B0000283DF43CA842F264020D
:10E21000C2F20102107201F0E5BD1D981C901C9E17
:10E22000B6F5803F08D342F26404C2F201044FF015
:10E230001F03237201F0D6BD219DAE63FDF722B806
:10E240001D9D219FFD63FDF71DB81D99219E316421
:10E25000FDF718B8219B9A6B1D98111A1C91DEE7E7
:10E260001E9A219BD96B8818FB2808D942F26403B7
:10E27000C2F201034FF012021A7201F0B3BD42F272
:10E28000A007C2F2010787F8FB10184650F8346F58
:10E2900031680E681D99BA18DB6BB0478DF86B00BA
:10E2A00000283CF4EFAF42F26404C2F20104207291
:10E2B00001F098BD2198416B0E68766846B942F22C
:10E2C0006406C2F201064FF01E02327201F08ABDEE
:10E2D0001D9AC36BC3F1FB018A4208D942F2640064
:10E2E000C2F201004FF01303037201F07BBD00F195
:10E2F00034004FF0000141F6F067C2F20107BA188E
:10E30000B0478DF86B0000283CF4BCAF42F26404C7
:10E31000C2F20104207201F065BDF7F77FFA002810
:10E320007CF4B0AF1D991C91FEF7A8BEF7F776FA02
:10E3300000283CF4A7AF1D981C90FEF79FBE1D9BC4
:10E340000B2B08D942F26404C2F201044FF0050617
:10E35000267201F047BDD8B24FF00001F7F71CFA62
:10E3600000EE900AB8EE601A219F87ED131AFCF7B1
:10E3700089BF1D9A0B2A0BD942F26401C2F2010136
:10E380004FF00500087201F02DBD00BF000080476E
:10E39000D0B24FF00101F7F7FFF901EE900AB8EEA5
:10E3A000612A219D85ED132AFCF76CBF1D9B0B2B69
:10E3B00008D942F26404C2F201044FF00506267245
:10E3C00001F010BDD8B24FF00001F7F755F9FCF796
:10E3D00059BF1D9A0B2A08D942F26401C2F2010109
:10E3E0004FF00500087201F0FDBCD0B24FF0010102
:10E3F000F7F742F9FCF746BF1D9B0B2B08D942F2F9
:10E400006404C2F201044FF00506267201F0EABC72
:10E41000D8B24FF00001F7F77FF9FCF733BF1D9A30
:10E420000B2A08D942F26401C2F201014FF0050043
:10E43000087201F0D7BCD0B24FF00101F7F76CF9C8
:10E44000FCF720BF9DF87400F2F7B4FE00287CF4BE
:10E4500019AF42F26403C2F201034FF028041C72A8
:10E4600001F0C0BC9DF87400219901F14C01F2F754
:10E47000C1FE00287CF406AF42F26406C2F2010637
:10E480004FF02802327201F0ADBC2199D1ED132A70
:10E490009DF87400BCEEE23A13EE101AF2F7DCFEBF
:10E4A00000287CF4EFAE42F26400C2F201004FF0AB
:10E4B0002803037201F096BCFCF7E4BE0DF1700C6A
:10E4C000FAF73EFB30B9219F97F847502E1C18BF32
:10E4D000012601E04FF00106219A82F84760FCF71F
:10E4E000D1BE9DF874600DF1700CFAF729FB01465E
:10E4F00030464FF00102FBF7C7FE8DF86B00002895
:10E500003CF4C0AE42F26404C2F20104207201F095
:10E5100069BC0DF1700CFAF713FB01468DF86A0027
:10E520009DF87400FBF76EFE8DF86B0000283CF43C
:10E53000A9AE42F26401C2F20101087201F052BCBC
:10E540001D981C904FF001038DF86A301E46219AE9
:10E5500092F847100B420AD092F846109DF87000CE
:10E5600019403246FBF790FE8DF86B0068B99DF8B4
:10E570006A304FEA43008DF86A001C9A02F10102EA
:10E580001C9210F0FE03E2D10AE09DF86A60012EB1
:10E5900006D142F26404C2F20104207201F022BCEE
:10E5A0004FF000078DF86B700DF1700CFAF7C8FA98
:10E5B0000DF1700CFAF7C4FAFCF764BE9DF8740014
:10E5C0004FF001010A46FBF75FFE8DF86B00002853
:10E5D0003CF458AE42F26401C2F20101087201F04B
:10E5E00001BC9DF874004FF000014FF00102FBF7F1
:10E5F0004BFE8DF86B0000283CF444AE42F26402FE
:10E60000C2F20102107201F0EDBB0DF1700CFAF7CD
:10E6100097FA219D95F84730184385F84700FCF795
:10E6200031BE1D980DF1A80C4CF8380DFAF736FFE5
:10E6300000287CF427AE42F2A410C2F20100099E29
:10E64000066001F052BB10A8FAF7BAFD014640B1CE
:10E650009DF84070022F04D0D1484FF00D0208F011
:10E66000B3FD0DF1700C9DF84000FAF751FAFCF77C
:10E6700009BEFBF767FAFCF705BE0DF1700CFAF75F
:10E680005FFAFCF7FFBD1D9EFA2E08D942F2640422
:10E69000C2F201044FF01202227201F0A3BB0DF18D
:10E6A000700CFAF74DFA42F2A001C2F2010188554E
:10E6B000FCF7E8BD0DF1700CFAF742FA42F2A00542
:10E6C000C2F2010585F8FB00FCF7DCBD0DF1700C12
:10E6D000219B93F84700FAF71BFAFCF7D3BD1D986E
:10E6E000FA2808D942F26406C2F201064FF012017C
:10E6F000317201F077BB0DF1700C42F2A007C2F24B
:10E700000107385CFAF704FAFCF7BCBD0DF1700C98
:10E7100042F2A002C2F2010292F8FB00FAF7F8F905
:10E72000FCF7B0BD1D9EF62E08D942F26404C2F279
:10E7300001044FF01200207201F054BB219DA86C1F
:10E74000FAF736F842F2A003C2F201039851FCF73F
:10E7500099BD1D99FA2908D942F26406C2F2010650
:10E760004FF01302327201F03DBB0DF1700C41F617
:10E77000F067C2F20107785CFAF7CAF9FCF782BDCC
:10E780000DF1700CFAF704FA41F6F065C2F20105DA
:10E790001E9BE85C1D9908420DF1700C0CBF002017
:10E7A000FF20FAF7B5F9FCF76DBD1D9EF92E08D9CB
:10E7B00042F26400C2F201004FF01301017201F055
:10E7C00011BB41F6F062C2F20102905D93195978D3
:10E7D00041EA00261C96002E3CF454ADFEF74EBCD8
:10E7E0001D9BFA2B08D942F26404C2F201044FF0D7
:10E7F0001300207201F0F6BA41F6F066C2F201068B
:10E80000F25C002A43D1FCF73DBD1D99FA2908D9D5
:10E8100042F26404C2F201044FF01302227201F0CA
:10E82000E1BA41F6F063C2F201035E5C7EB3FCF72D
:10E8300029BD0DF1700CFAF783F91C9038BBFCF779
:10E8400021BD0DF1700CFAF7A3F941F6F060C2F2A8
:10E8500001001E99465C1D9B1E4218D0FCF712BD9C
:10E860000DF1700CFAF794F941F6F062C2F2010270
:10E870001E98115C1D9E314209D1FCF703BD0DF1BC
:10E88000700CFAF75DF91C9000287CF4FBAC219B1E
:10E890001A6A42B942F26404C2F201044FF0030062
:10E8A000207201F09FBA02F1FF351D6202F10102F0
:10E8B00053F8227042F2A411C2F201010F60FCF77A
:10E8C000E1BC219D95F847704FEAD71343EA470210
:10E8D00085F84720FCF7D6BC219890F847604FEAAE
:10E8E000560141EAC61580F84750FCF7CBBCFAF751
:10E8F00039FDFCF7C7BC42F27007C2F20107FB7892
:10E900004FF0010000FA03F03A7922EA00023A716E
:10E91000FCF7B8BC42F26404C2F201044FF00106F5
:10E92000267201F05FBA42F27001C2F20101CD78A5
:10E9300045B942F27000C2F201004FF00602C27007
:10E94000FCF7A0BC05F1FF3742F27003C2F20103ED
:10E95000DF70FCF797BC42F27006C2F20106317814
:10E9600001F1FF35EFB237703379FF2B0BD1632FF5
:10E970007CF688AC42F27006C2F201064FF06301E9
:10E980003170FCF77FBC172F7CF67CAC42F2700034
:10E99000C2F201004FF017020270FCF773BC00BF17
:10E9A000F61E012042F27005C2F201056F7807F1F0
:10E9B000FF33D8B268702A79FF2A0BD100287CF483
:10E9C00061AC42F27005C2F201054FF00C076F70A6
:10E9D000FCF758BC3B287CF655AC42F27006C2F2FC
:10E9E00001064FF03B017170FCF74CBC42F264042D
:10E9F000C2F201044FF00103237201F0F3B942F2B5
:10EA00006400C2F201004FF00102027201F0EAB9A3
:10EA100042F26406C2F201064FF00101317201F0C8
:10EA2000E1B942F26404C2F201044FF0010323721F
:10EA300001F0D8B942F27005C2F20105EF78052F56
:10EA400008D942F27006C2F201064FF00002F270DD
:10EA5000FCF718BC07F1010742F27000C2F2010096
:10EA6000C770FCF70FBC42F27001C2F201010B78D3
:10EA700003F10103DDB20D700F79FF2F0BD1632D70
:10EA80007CF600AC42F27001C2F201014FF00002CC
:10EA90000A70FCF7F7BB172D7CF6F4AB42F270005E
:10EAA000C2F201004FF000060670FCF7EBBB42F229
:10EAB0007005C2F201056B7803F10103DFB26F70DC
:10EAC0002879FF280BD10C2F7CF6DCAB42F27005C5
:10EAD000C2F201054FF001026A70FCF7D3BB3B2F75
:10EAE0007CF6D0AB42F27006C2F201064FF0000194
:10EAF0007170FCF7C7BB42F26404C2F201044FF02C
:10EB00000103237201F06EB942F27007C2F20107ED
:10EB1000F8784FF0010606FA00F6397986EA010521
:10EB20003D71FCF7AFBB0DF1700CFAF709F842F23A
:10EB30007002C2F201021071FCF7A4BB0DF1700C5F
:10EB4000F9F7FEFF062842F27003C2F2010392BFFA
:10EB5000D8700027DF70FCF795BB0DF1700CF9F74A
:10EB6000EFFF42F27006C2F201063070FCF78ABB7A
:10EB70000DF1700CF9F7E4FF42F27001C2F20101ED
:10EB80004870FCF77FBB0DF1700CF9F7D9FF42F22A
:10EB90007005C2F20105A870FCF774BB0DF1700C92
:10EBA00042F27000C2F201000079F9F7B1FFFCF700
:10EBB00069BB0DF1700C42F27002C2F20102D07812
:10EBC000F9F7A6FFFCF75EBB0DF1700C42F2700383
:10EBD000C2F201031878F9F79BFFFCF753BB0DF164
:10EBE000700C42F27007C2F201077878F9F790FFD3
:10EBF000FCF748BB0DF1700C42F27006C2F2010640
:10EC0000B078F9F785FFFCF73DBB42F26404C2F22D
:10EC100001044FF00101217201F0E4B81D9A0F2A9E
:10EC200008D942F26404C2F201044FF027002072B6
:10EC300001F0D8B8C24D05EB820042F27003C2F277
:10EC4000010315F822701F7046785E704FF00001C6
:10EC50009970D97082781A71FCF714BB42F2640380
:10EC6000C2F201034FF001061E7201F0BBB842F27E
:10EC70007005C2F20105EF784FF0010101FA07F1CA
:10EC80002A7941EA02002871FCF7FCBA42F26404D6
:10EC9000C2F201044FF00103237201F0A3B842F263
:10ECA0006406C2F201064FF00101317201F09AB818
:10ECB0004FF00005139512951195199542F27007C2
:10ECC000C2F201073A7802F164021692787800F1F4
:10ECD000FF331593BE78149611A808F09BF8179986
:10ECE00019B101F1FF37FDB201E04FF0060542F224
:10ECF0007002C2F20102D570FCF7C4BA1D9E0F2E3D
:10ED000008D942F26404C2F201044FF027062672C9
:10ED100001F068B88A4800EB860142F27003C2F243
:10ED200001031D7800F826505F784F701A798A70B9
:10ED3000FCF7A8BA42F26400C2F201004FF00101F0
:10ED4000017201F04FB80DF1700C219B93F8500047
:10ED5000F9F7DEFEFCF796BA42F2B012C2F20102F7
:10ED6000147814F0010F08D142F26404C2F20104D5
:10ED70004FF03002227201F035B842F22806C2F29A
:10ED80000106306840B942F26401C2F201014FF05D
:10ED900031030B7201F026B842F2B011C2F2010148
:10EDA0000B7803F0FE0242F004040C7042F23C06C1
:10EDB000C2F201064FF00000306000F07FBF42F267
:10EDC000B016C2F20106307810F0010F08D142F2FD
:10EDD0006406C2F201064FF03000307201F002B852
:10EDE00042F22801C2F201010B6843B942F2640405
:10EDF000C2F201044FF03402227200F0F3BF42F27B
:10EE0000B014C2F20104227802F0FE0646F00200BD
:10EE1000207042F23C01C2F201014FF000030B608E
:10EE200000F04CBF219D95F846700DF1700CF9F77C
:10EE300087FE21993B1A91F8502002F00106981B99
:10EE40001C9081F84700FF2894BF0020012081F822
:10EE50005000FCF717BA1D9BFA2B08D942F2640444
:10EE6000C2F201044FF01301217200F0BBBF41F662
:10EE7000F065C2F201051E9FEF54FCF703BA4FF094
:10EE800000021C921AE04FF001061C9616E04FF0AB
:10EE900002001C9012E04FF003031C930EE04FF0B1
:10EEA00004051C950AE04FF005071C9706E04FF09B
:10EEB00006011C9102E04FF007021C921D991B9164
:10EEC0001C98FAF763FAFCF7DDB90DF1700CF9F74D
:10EED0005FFE1E9E41F6F063C2F20103985D1D9D28
:10EEE00005439D55FCF7CEB91D9EF92E08D942F277
:10EEF0006404C2F201044FF01202227200F072BFE9
:10EF000042F2A007C2F201071E99B955FCF7BAB93F
:10EF100042F2A000C2F201001D9B80F8FB30FCF71A
:10EF2000B1B942F2CC26C2F20106316851B942F2BF
:10EF30006400C2F201004FF00106067200F052BFF9
:10EF4000443A00104E681D981E994FF001020DF1D1
:10EF50006A03B0478DF86B009DF86A20D2F1010179
:10EF600038BF0021219B83F8501000283CF48AA967
:10EF700042F26404C2F20104207200F033BF42F294
:10EF8000CC22C2F20102116841B942F26400C2F21D
:10EF900001004FF00106067200F024BF0B681D98B7
:10EFA0001E9998478DF86B0000283CF46BA942F23B
:10EFB0006404C2F20104207200F014BF42F2CC22B9
:10EFC000C2F20102116841B942F26400C2F20100CA
:10EFD0004FF00106067200F005BF4E681D981E999D
:10EFE0004FF000020DF16A03B0478DF86B009DF8F9
:10EFF0006A30D3F1010238BF0022219981F85020F4
:10F0000000283CF43FA942F26404C2F201042072D9
:10F0100000F0E8BE0A981E99F9F7B2FF0A9040B9CD
:10F0200042F26406C2F201064FF01702327200F09B
:10F03000D9BE0A9B1A68966A46B942F26400C2F2C7
:10F0400001004FF01503037200F0CCBE0A998868E6
:10F050009DF8741042F2A002C2F20102B0478DF88E
:10F060006B0000283CF40EA942F26404C2F20104D1
:10F07000207200F0B7BE0A981E99F9F781FF0A9036
:10F0800040B942F26400C2F201004FF0170303726C
:10F0900000F0A8BE0A990868436943B942F26401C6
:10F0A000C2F201014FF015020A7200F09BBE0A9EE7
:10F0B000B0689DF8741042F2A002C2F201029847B3
:10F0C0008DF86B0000283CF4DDA842F26404C2F223
:10F0D0000104207200F086BE0A981E99F9F750FFCD
:10F0E0000A9040B942F26406C2F201064FF01701DD
:10F0F000317200F077BE0A9F3E68B76947B942F2A5
:10F100006400C2F201004FF01503037200F06ABE02
:10F1100042F2A006C2F201060A9988689DF87410AE
:10F1200032460DF16A03B8478DF86B009DF86A20EE
:10F13000327000283CF4A6A842F26404C2F2010432
:10F14000207200F04FBE0A981E99F9F719FF0A9035
:10F150001D9E7F2E09D1051C18BF012542F2A00774
:10F16000C2F201073D70FCF78DB80A9A42B942F22B
:10F170006400C2F201004FF01703037200F032BEC8
:10F180000A9803685B6843B942F26406C2F201065A
:10F190004FF01502327200F025BE0A998868F1B26C
:10F1A00042F2A002C2F2010298478DF86B000028DB
:10F1B0003CF468A842F26404C2F20104207200F038
:10F1C00011BE0A981E99F9F7DBFE0A9040B942F287
:10F1D0006406C2F201064FF01702327200F002BE5E
:10F1E0000A990E68B76847B942F26400C2F201009A
:10F1F0004FF01501017200F0F5BD42F2A006C2F217
:10F2000001060A9A90689DF8741032780DF16A032D
:10F21000B8478DF86B009DF86A30337000283CF4D5
:10F2200031A842F26404C2F20104207200F0DABD97
:10F230000A981E99F9F7A4FE0A9040B942F26406B2
:10F24000C2F201064FF01700307200F0CBBD0A9FEA
:10F250003B68DF6847B942F26403C2F201034FF032
:10F2600015021A7200F0BEBD42F2A006C2F20106FB
:10F270000A9880689DF8741032460DF16A03B84709
:10F280008DF86B009DF86A10317000283BF4FAAFDE
:10F2900042F26404C2F20104207200F0A3BD0A9895
:10F2A0001E99F9F76DFE0A9040B942F26403C2F26A
:10F2B00001034FF017061E7200F094BD0A9F3968D3
:10F2C0000F6947B942F26400C2F201004FF0150124
:10F2D000017200F087BD0A9BD3F808809DF87490F6
:10F2E00042F2A006C2F201063068F9F78BFA024634
:10F2F000404649460DF16A03B8478DF86B009DF80A
:10F300006A20327000283BF4BDAF42F26404C2F2BE
:10F310000104207200F066BD0A984FF00001F9F771
:10F320002FFE0A9040B942F26400C2F201004FF091
:10F330001703037200F056BD0A9A1068C36A43B9F6
:10F3400042F26406C2F201064FF01502327200F07A
:10F3500049BD0A9988689DF8741098478DF86B002C
:10F3600000283BF48FAF42F26404C2F20104207221
:10F3700000F038BD0A981E99F9F702FE0A9040B9CC
:10F3800042F26406C2F201064FF01703337200F036
:10F3900029BD0A990E68F36943B942F26400C2F2CA
:10F3A00001004FF01501017200F01CBD0A9A90682F
:10F3B0009DF8741042F2A002C2F2010298478DF843
:10F3C0006B0000283BF45EAF42F26404C2F2010419
:10F3D000207200F007BD0A981E99F9F7D1FD0A9036
:10F3E00040B942F26400C2F201004FF01706067203
:10F3F00000F0F8BC0A9A1068066A46B942F2640343
:10F40000C2F201034FF015021A7200F0EBBC0A9928
:10F4100088689DF8741042F2A002C2F20102B0475F
:10F420008DF86B0000283BF42DAF42F26404C2F269
:10F430000104207200F0D6BC0A981E99F9F7A0FDCD
:10F440000A9040B942F26401C2F201014FF0170282
:10F450000A7200F0C7BC0A990B685E6A46B942F2AC
:10F460006403C2F201034FF015061E7200F0BABC2D
:10F470000A9A90689DF8741010AAB0478DF86B0036
:10F480001098F9F795F942F2A001C2F20101086063
:10F490009DF86B0000283BF4F5AE42F26404C2F222
:10F4A0000104207200F09EBC0A984FF00001F9F7A9
:10F4B00067FD0A9040B942F26403C2F201034FF0C3
:10F4C00017061E7200F08EBC0A9803681E6B46B9C0
:10F4D00042F26400C2F201004FF01502027200F025
:10F4E00081BC0A9988689DF8741042F2A002C2F2A9
:10F4F0000102B0478DF86B0000283BF4C3AE42F226
:10F500006404C2F20104207200F06CBC1D9907294A
:10F5100008D942F26404C2F201044FF008012172DA
:10F5200000F060BC40F2A065C1F2000505EBC10728
:10F53000D7F8100900287BF4A5AEF7F707FE0028DE
:10F5400008BF012040F2A062C1F200021D9B02EB45
:10F55000C306C6F81009FBF795BE1D98072808D901
:10F5600042F26404C2F201044FF00801217200F07B
:10F5700039BC40F2A065C1F2000505EBC007D7F821
:10F580001029002A3BF47EAEF7F7E0FD1D9B40F208
:10F59000A066C1F2000606EBC305D5F81019401AA3
:10F5A0001C90D5F81479B8428CBF0027C0EB070730
:10F5B0001B9740F2A062C1F2000202EBC3031B9E44
:10F5C000C3F814694FF00005C3F81059FBF75ABE91
:10F5D0001D9EFA2E07D942F26400C2F201004FF0DC
:10F5E00013020272FEE30DF1700CF9F7A9FA41F66D
:10F5F000F067C2F20107B855FBF744BE0DF1700C7D
:10F60000F9F7C6FA0DF1700CF9F79AFA1C9050B19F
:10F610001E9B41F6F062C2F20102D05C1D9D0543C3
:10F62000D554FBF72FBE1E9B41F6F065C2F20105D3
:10F63000EE5C1D9926EA0107EF54FBF723BE1D9EE1
:10F640001E9A9119CBB242F2A000C2F2010080F8DA
:10F65000FB30FA2B07D942F26404C2F201044FF0E6
:10F6600012012172BEE342F2A417C2F201073D6803
:10F6700042F2A001C2F20101881940F20006C0F670
:10F680000106A91907F0A0FD3A681E9BD018386042
:10F69000FBF7F8BD1D9EF82E07D942F26404C2F2B2
:10F6A00001044FF0130323729CE3F7F74FFD00F1C1
:10F6B00004004CF6CD47CCF6CC47A7FB00154FEA2B
:10F6C0009500219A536AB0FBF3F61C961D9F41F6F4
:10F6D000F061C2F201014FEA1645CD55C8194FEA53
:10F6E000162242708670FBF7CDBD1D9EF82E07D9FD
:10F6F00042F26404C2F201044FF01302227271E379
:10F70000F7F724FD00F104004CF6CD47CCF6CC47CA
:10F71000A7FB00214FEA91052198426AB5FBF2F65A
:10F720001D9B41F6F067C2F20107F8184178FD5CB5
:10F730004FEA054242EA0127837847EA03001B901B
:10F74000361A26F07F411C910DF1700C1E988142F3
:10F750002CBF00200120F9F7DBF9FBF793BD219DB9
:10F7600095F846700DF1700CF9F7EAF9381A1C900B
:10F77000219B83F84700FF2894BF0020012083F8D5
:10F780005000FBF77FBD1D9EF92E07D942F264069B
:10F79000C2F201064FF01303337223E342F2A411C5
:10F7A000C2F201010A6841F6F063C2F201034FEAB6
:10F7B000122098559E197270FFF769B8219D95F82F
:10F7C00047201C9295F8467085F8477085F84620CA
:10F7D000FBF758BD1D98072807D942F26401C2F211
:10F7E00001014FF008040C72FCE2F9F7FDFD0DF188
:10F7F000A80C4CF8380D003018BF0120F9F788F933
:10F80000FBF740BD219E96F8470096F846300DF173
:10F81000700C984214BF00200120F9F779F9FBF72A
:10F8200031BD219D95F8470095F846200DF1700CEB
:10F83000801A18BF0120F9F76BF9FBF723BD219F50
:10F8400097F8470097F846100DF1700C88422CBFCE
:10F8500000200120F9F75CF9FBF714BD219E96F812
:10F86000470096F846300DF1700C984294BF002086
:10F870000120F9F74DF9FBF705BD219D95F84700EB
:10F8800095F846200DF1700C90428CBF00200120AD
:10F89000F9F73EF9FBF7F6BC219F97F8470097F878
:10F8A00046100DF1700C884234BF00200120F9F79A
:10F8B0002FF9FBF7E7BC1D98F62807D942F264043C
:10F8C000C2F201044FF0120222728BE242F2A00651
:10F8D000C2F201063058F8F795FF219BD864FBF778
:10F8E000D1BC1D99F62907D942F26400C2F2010089
:10F8F0004FF01206067275E242F2A005C2F201054F
:10F900006858F8F77FFF219FB864FBF7BBBC42F251
:10F91000A003C2F2010393F8FB201D9E9119FB295D
:10F9200007D942F26406C2F201064FF012013172A9
:10F9300058E21E9BC2F1FB00834207DD42F26404E1
:10F94000C2F201044FF0130222724BE241F6F0655D
:10F95000C2F20105E81842F2A007C2F20107B91984
:10F9600007F032FCFBF78EBC2198436B1A6856688F
:10F970003EB942F26406C2F201064FF01E02327234
:10F9800030E21E9A42F2A001C2F2010191F8FB306E
:10F990009918FB2907D942F26400C2F201004FF026
:10F9A000120303721EE200F134001D9942F2A00717
:10F9B000C2F20107BA18B0478DF86B0000283BF47B
:10F9C00061AC42F26404C2F2010420720AE242F223
:10F9D0006401C2F201014FF001040C7202E20DF168
:10F9E000700CF9F7D5F841F6F065C2F201051E9FDB
:10F9F000E85D1D9B18423BF445AC42F2A416C2F2EE
:10FA00000106099A326070E10DF1700CF9F7C0F847
:10FA100041F6F061C2F201011E9D4F5D1D98074243
:10FA20007BF430AC42F2A414C2F20104099B2360BF
:10FA30005BE19DF874000DF16B01FAF715FB8DF891
:10FA40006A009DF86B602EB142F26400C2F20100C0
:10FA50000672C7E100283BF415AC42F2A412C2F2D0
:10FA600001020999116040E19DF874000DF16B01EC
:10FA7000FAF7FAFAD0F1010338BF00238DF86A30A3
:10FA80009DF86B0028B142F26402C2F201021072CA
:10FA9000A8E1219DEF6A17B98DF86A7002E09DF820
:10FAA0006A2062B90DF1700C1E98F9F7F7FC30B9B5
:10FAB00042F2A414C2F201040999216015E10DF18A
:10FAC000700C9DF86A00F9F723F84FF00006219BAF
:10FAD000DE62FBF7D7BB9DF874000DF16B01FAF7FE
:10FAE000C3FA8DF86A009DF86B602EB142F264048F
:10FAF000C2F20104267275E100287BF4C3AB42F226
:10FB0000A415C2F20105099F2F60EEE09DF8740074
:10FB10000DF16B01FAF7D8FA8DF86A009DF86B10B9
:10FB200029B142F26403C2F2010319725AE10028BA
:10FB30007BF4A8AB42F2A410C2F20100099A026061
:10FB4000D3E09DF874000DF16B01FAF7BDFA061CC5
:10FB500018BF01268DF86A6092E79DF874000DF1D8
:10FB60006B01FAF781FA011C18BF01218DF86A10A8
:10FB700086E71D9EF62E07D942F26403C2F2010306
:10FB80004FF012041C722DE12198C06CF8F710FEA2
:10FB900042F2A005C2F20105A851FBF773BB0DF1BB
:10FBA000700CF8F7CDFF219F97F84710D1F10102B3
:10FBB00038BF0022002814BF164682F0010687F8DD
:10FBC0004760FBF75FBB0DF1700CF8F7B9FF219DA3
:10FBD00095F84730584085F84700FBF753BB0DF1C7
:10FBE000700CF8F7ADFF219F87F85100FBF74ABB77
:10FBF00005F06CFF0DF1A80C4CF8380DFF2828BF5C
:10FC0000FF20C0B2F8F784FFFBF73CBB05F054FFC0
:10FC10000DF1A80C4CF8380DFF2828BFFF20C0B20A
:10FC2000F8F776FFFBF72EBB05F05AFF0DF1A80C95
:10FC30004CF8380DFF2828BFFF20C0B2F8F768FF46
:10FC4000FBF720BB05F02EFF0DF1700C00280CBF58
:10FC5000FF200020F8F75CFFFBF714BB42F29C107A
:10FC6000C2F2010001681D9A881805F07DFA8DF82E
:10FC70006B0000283BF406AB42F26404C2F20104BC
:10FC80002072AFE01D9805F02DFAFBF7FBBA0DF1DD
:10FC9000700CF8F755FF05F01FFAFBF7F3BA42F2C4
:10FCA0009C16C2F2010635681D9BE81805F036FA6D
:10FCB000FBF7E8BA05F01AFAFBF7E4BA42F22800BB
:10FCC000C2F20100016881B942F2B012C2F201022F
:10FCD000147804F00206F3B23BB142F26404C2F2BB
:10FCE00001044FF0350323727CE042F2B017C2F2F8
:10FCF00001073D7815F0010F7BF4C2AA219828B1C5
:10FD000042F2A411C2F201010A68426042F23C04CC
:10FD1000C2F2010426687F2E00F29F8006F10106E0
:10FD20001B961C9616B94FF001071B976B4E4FF0B0
:10FD3000540542F2B014C2F2010442F22807C2F2A2
:10FD400001071C9B05FB036021909BB9217801F002
:10FD50000402D1B209B93A6842B9217841F00102EE
:10FD60006FF382022270426842B115E04FF0010049
:10FD70001C90E6E742687AB9802B02D003F10103B8
:10FD800001E04FF000031C931B988342D9D14FF040
:10FD90000000F9F7C3FED4E742F23C06C2F20106C6
:10FDA000336042F2A415C2F201052A604FF0000A46
:10FDB0005446FBF767BA219F396A41F000423A6323
:10FDC000FBF760BA4FF00006219D2E63FBF75ABA8D
:10FDD000FBF758BA0C9D42F26400C2F201004FF0EA
:10FDE0000104047242F26402C2F20102099E16602A
:10FDF0002198046A24B104F1010450F824300993D5
:10FE000042F26401C2F20101099A4A604D72F1F7AF
:10FE1000B7FBF1F7B5FB219D2E6A7EB14FF00000D4
:10FE20001C90219C236A4BB1F1F7AAFB1C9901F1AC
:10FE300001011C91219A156A8D42F5D84FF00000FE
:10FE4000F9F76CFEFBF745B94FF0000706F1FF34F8
:10FE50004FF000005E46FDF7FFBC4FF000031C931F
:10FE600061E74FF002031C931C4ED6F8AC2032B968
:10FE7000FDF740BF2BB0BDEC0A8BBDE8F08F03F15E
:10FE8000010306F15406FDF731BF07F1010306F146
:10FE90005406812B7DF42AAFFDF786BFBEF1000F1B
:10FEA0003DF474AC10F8039001F8039003F10103E2
:10FEB00093427DF46BACFDF777BCCD180EEB030CD1
:10FEC00013F8017F02F1FF36B8423DF43EAA3246F4
:10FED000FDF74ABA06F1FF32FDF746BAF00F0010FF
:10FEE0002DE9F04F2DED028B8FB04FF0000842F25C
:10FEF0003807C2F2010742F23003C2F20103039352
:10FF000042F24C0BC2F2010B40F2A066C1F20006B5
:10FF10009FEDB98B39684FF0FF3041B9F1F730FBF5
:10FF2000386800280CBFFA204FF0FF30FFE7F6F7E3
:10FF300093FC28B1B8F1320F09D808F1010806E0A6
:10FF4000B8F1330F0CBF4FF034084FF000083A6897
:10FF5000D2B9F1F715FBB8F1320F0ED1039C20682E
:10FF6000F6F726FD4FF00005039B1D60F5F7FCFE3C
:10FF70004FF00200F9F710FD06E0B8F1340F03D19D
:10FF80004FF00100F9F708FD9BF800104FF41170D5
:10FF900000FB0162D2F81842002CBBD04FF411755F
:10FFA00005FB01F303F5887406EB0409315DE029D4
:10FFB0000CD199F801000E2808D14FF6FF70494680
:10FFC000D9F80021F8F78EFB10B36BE2325D02F036
:10FFD0001F0509EB05035A78294605F0010019F8B9
:10FFE0000550521B01F1FF33002940F078820BE0ED
:10FFF00019F80300151A03F1FF3119F80120AA1AA4
:020000040803EF
:1000000001F1FF330029F3D112F0FF0F40F04A82D3
:10001000335D4FEA5310072800F23C82DFE810F00E
:1000200008003A023A023500A6003A028A00260188
:10003000335D09F1010513F01F0000F0338209F16F
:10004000020905F1020500F1FF3255FA82F402942B
:100050004FF000054FF0010A15E019F8011CE8B255
:1000600021405246FAF710F9002840F01B8205F1B2
:1000700001054FEA4404FF2CEFD909F10109029967
:10008000894500F00F825446E7E799F80140386847
:1000900070B1F6F78DFC4FF000003860F5F764FEA4
:1000A000FAF7BCFE4FF00100F9F776FCF1F768FAB9
:1000B00003990B686BB94AF69C60C0F603004FF0D9
:1000C00007014AF29962C0F60202F6F787FB039D28
:1000D000286005A84FF00001F9F78CFE7CB9F7F70E
:1000E00035F8C1B201F1FF33DDB2FD2D42F2A810A7
:1000F000C2F2010092BF01700122027009E042F2D7
:10010000A810C2F20100027802FB04F404EB1424EC
:10011000047042F2A814C2F2010421780EAB03F875
:10012000241D4FF003004FF000014FF01802F9F7C3
:1001300057FCEFE60DF11300F9F742F801469DF880
:1001400013508DF81450012D06D828B10DF115006B
:100150004FF00D0207F038F84FF006004FF00001A5
:100160004FF00E0205ABF9F73BFCD3E69BF800100D
:100170004FF4117303FB01F499F80100032872D8BE
:10018000DFE800F002263E504FF00100FAF7D0FE03
:100190004FF000050EAB03F8255D4FF00400294633
:1001A0004FF00102F9F71CFC4FF0C800F8F782FA93
:1001B00032599BF800004FF0010400940195D2F8E9
:1001C0000CC04FF416512A464FF00803E04766E191
:1001D0004FF0000142F26403C2F2010319724FF0C2
:1001E00001040EAB03F8254D4FF004002246F9F749
:1001F000F7FB54E1AFF300800000000000E06F4027
:10020000F9F7A0FC0EAB4FF0020103F8251D4FF0EB
:1002100004004FF000014FF00102F9F7E1FB4FF04D
:1002200001043CE10EAB4FF0120203F8252D4FF014
:1002300004004FF000014FF00102F9F7D1FB4FF03D
:10024000C800F8F737FA35599BF800004FF0010461
:1002500000944FF000020192ED684FF416414FF008
:100260000803A8471BE14FF0000418E199F801507A
:10027000A5F102050C2D00F21081DFE815F00D004C
:1002800067007E000E010E010E010E010E010E012F
:100290000E010E010E019D00315DC1F30403DAB2BF
:1002A000012A00F0FF8009F1050509F1080403EBBC
:1002B000C30003EB400101EBC10303F15403DAB2C5
:1002C00002EB42002418C5EB040CACF1030E0EF057
:1002D000010A99F8029015F8010C05F01BFD53EC8A
:1002E000182B06F029F805F0EFFD01464846FAF70D
:1002F0003BF805F10305A54240F0D780D2E015F8A0
:10030000039C15F8010C05F005FD53EC182B06F0C5
:1003100013F805F0D9FD01464846FAF725F805F12E
:10032000030515F803AC15F8010C05F0F3FC53ECCC
:10033000182B06F001F805F0C7FD01465046FAF704
:1003400013F805F10305A542D9D1ABE099F80230C5
:10035000305DC0F30405A5F10305EAB209F103011C
:100360009C18FF2CC4BF5A42D2B241F6F060C2F2D0
:100370000100C01806F028FF94E099F8023099F8BF
:1003800003500EAC04F8243D0DF1150041F6F06168
:10039000C2F20101C918202D34BF2A46202206F0DE
:1003A00013FF05F101024FF007004FF00301D2B235
:1003B0002346F9F715FBADE599F80240C4B999F861
:1003C0000310A9B904F0FEFE039A1068F6F7F0FADC
:1003D0004FF0000303980360F5F7C6FC4AF6AC60E3
:1003E000C0F6030008F0E0FCF9F78CFC002848D0C8
:1003F00099F8025099F803404AF6BC60C0F6030031
:1004000044EA052108F0D0FC99F803A0494611F808
:10041000022F40F20003C0F6010303EB022541F670
:10042000F064C2F2010404EB0A0001F102014FF092
:10043000800206F0C9FE4FF68071CFF6FF71CAEB5D
:100440000100C2B2A018A9184FF0800206F0BCFE4D
:10045000204629464FF48072F2F7BEF9A0B9204633
:1004600029464FF4807206F059FA80B94FF0010026
:100470004FF000010A460B46F9F7B2FA4FF00104BB
:100480000DE04FF000040AE04FF0000407E04FF0E9
:10049000000404E04FF0000401E04FF00004002CE1
:1004A0007FF438ADF8F76EFE34E5BAF1000F3FF493
:1004B00026AF15F803AC15F8010C05F02BFC53EC36
:1004C000182B05F039FF05F0FFFC01465046F9F7FF
:1004D0004BFF05F10305A5427FF411AFE2E70028C9
:1004E0003FF486AD19F80310521A03F1FF33B3F14C
:1004F000FF3F7FF47DAD87E542F24003C2F2010386
:100500001B684B634BB19A68824209D0DB684B632E
:100510001BB19A688242F9D102E04FF01E00704789
:100520004FF00000704700BF42F2D913C2F201033E
:100530001A78027042F2D810C2F2010003780B70F0
:10054000704700BF42F2D913C2F201031B78834205
:1005500025D842F2D812C2F2010212789A189042BB
:1005600020DAC01A4FEA50034FF0010202FA03F3F7
:1005700010F0010F09D042F2E410C2F2010002684B
:1005800013400B704FF00100704742F2DC10C2F2D2
:100590000100026813400B704FF0010070474FF0EC
:1005A000000070474FF00000704700BF10B542F2E6
:1005B000D913C2F201031B7883427AD842F2D812CF
:1005C000C2F2010212789A18904275DAC31A03F047
:1005D000FE0442F2E810C2F201000278A418E4B26C
:1005E0004FEA53024FF0010000FA02F213F0010F3C
:1005F00012D041B142F2E410C2F20100016842EAB5
:10060000010303601AE042F2E410C2F20100036841
:1006100023EA0203036011E041B142F2DC10C2F2AE
:100620000100036842EA0301016007E042F2DC13C3
:10063000C2F20103196821EA0201196042F2DC10DA
:10064000C2F2010001680A4224D042F2E413C2F26D
:100650000103186802420ED020464FF00001F0F767
:100660000BFC04F10102D0B24FF00101F0F704FCE1
:100670004FF0010010BD20464FF00101F0F7FCFBE8
:1006800004F10101C8B24FF00001F0F7F5FB4FF0A3
:10069000010010BD20464FF00001F0F7EDFB04F122
:1006A0000102D0B24FF00001F0F7E6FB4FF001007D
:1006B00010BD4FF0000010BD4FF0000010BD00BF96
:1006C00008B542F2E813C2F20103187042F2E013D7
:1006D000C2F20103197042F2D913C2F201031A7077
:1006E000091A01F10101C8B242F2D812C2F20102A4
:1006F0001070412801D9EFF703FD40F2CC10C2F28F
:1007000000004FF00101F9F71FFC08BD2DE9F84387
:1007100042F2E913C2F2010318784FEA400111F0E6
:10072000FF0405D042F2E912C2F20102147006E0A1
:1007300042F2E915C2F201054FF001062E7042F2B5
:100740000C27C2F20107387842F2E913C2F2010322
:10075000197808420CBF4FF000094FF001094FF023
:1007600000052C464FF0010742F2EC16C2F20106DA
:10077000A84604F01F0207FA02F0AB59184204D051
:10078000204649464246F9F77FFD04F10104E4B2F0
:1007900014F01F0FEDD105F10405202DE9D1BDE8BE
:1007A000F88300BF42F20C23C2F20103187042F238
:1007B000E910C2F201004FF001020270704700BF61
:1007C00000B583B042F2EC10C2F201004FF000011C
:1007D0004FF00802EFF7A4FC4FF0000300934FF036
:1007E0000100019042F21020C2F201004FF47A7130
:1007F0004FF0060240F20D73C0F60303F6F770FCEB
:1008000003B000BD08B542F21020C2F20100F6F7B5
:10081000C1FB4FF0CC00FFF7C5FF08BD89B14FEA1F
:10082000501242F2EC13C2F2010300F01F004FF02D
:10083000010101FA00F053F82210084343F82200A6
:1008400011E04FEA501242F2EC13C2F2010300F041
:100850001F004FF0010101FA00F053F8221021EAC5
:10086000000143F822104FF00000704708B54FF424
:1008700040404BF6B811C0F6030142F23422C2F2F6
:100880000102F9F71FFB08BD10B584B0144649BB3F
:100890000DF10D0300930DF10E0001904FF00000DB
:1008A00001460DF10A020DF10B03F5F709F94FF0BE
:1008B00000018DF80C109DF80B201AB14FF00103C8
:1008C0008DF80C309DF80A0028B19DF80C1041F00D
:1008D00002028DF80C204FF000008DF80F00039BF2
:1008E000236001E04FF0140004B010BD70B5144651
:1008F0008AB199B94FF0000001460246F5F758F960
:1009000006462578F5F738FA85420AD2735D2370DA
:100910004FF0000070BD4FF0160070BD4FF0140096
:1009200070BD4FF0160070BDF8B515461F464FF06C
:1009300000033B70A9B992F8FB0060B14FF00004CE
:100940002646285D3146F5F72DF804F1010495F8A7
:10095000FB20A242F5D84FF0010139704FF00000A2
:10096000F8BD4FF01400F8BD10B586B04FF001048B
:100970001C70F1B942F24023C2F20103197842F22D
:100980004120C2F20100037802AC00944FF0100045
:10099000019010461A464FF00103FAF705F84BF69E
:1009A000B410C0F60300214608F0FEF94FF0000035
:1009B00004E04FF000021A704FF0140006B010BDB2
:1009C0002DE9F04115461C464FF001032370042920
:1009D0007CD8DFE801F0030B7B1B64006878297882
:1009E000F5F7D6F84FF00000BDE8F081287842F224
:1009F0004021C2F2010108706A7842F24123C2F23A
:100A000001031A704FF00000BDE8F0812C786D787A
:100A100005F1040546F26761C6F2666181FB0523B4
:100A20004FEA630202EB820010F0FF0555D04FF051
:100A30000007A5F1050808F00108042C94BF26461C
:100A4000052630463946F4F7ADFFA41BE4B2A5F104
:100A5000050515F0FF0544D11DE0042C94BF264682
:100A6000052630463946F4F79DFFA31BA5F1050581
:100A700005F0FF0503F0FF04042C94BF264605266D
:100A800030463946F4F78EFFA21BD4B2A5F1050516
:100A900015F0FF05E1D14FF00000BDE8F0812E78A0
:100AA000F5F76AF9864206D34FF0000020704FF048
:100AB0001600BDE8F081304605F101014FF001025A
:100AC000F5F792F84FF00000BDE8F0814FF000001C
:100AD00020704FF01400BDE8F0814FF00000BDE839
:100AE000F0814FFA88F6002EB7D0042C94BF26462A
:100AF000052630463946F4F755FFA11BCCB2A5F1C7
:100B0000050515F0FF05A8D1C5E700BF10B51C46C7
:100B10004FF001032370052941D8DFE801F0030EEF
:100B200018222C361046F4F7FBFF00283DD14FF079
:100B3000000020704FF0160010BD4AF69860C0F615
:100B40000300114608F030F94FF0000010BD4AF6DE
:100B50009060C0F60300114608F026F94FF000003F
:100B600010BD4AF68C60C0F60300114608F01CF96F
:100B70004FF0000010BD4AF68460C0F60300114635
:100B800008F012F94FF0000010BD4AF67C60C0F684
:100B90000300114608F008F94FF0000010BD4FF0B7
:100BA000000121704FF0140010BD4FF0000010BD87
:100BB00008B5012805D0022814BF002201221146E1
:100BC00003E04FF000024FF001014FF00100F5F794
:100BD000B1F808BD08B54FF00103137001F1FF3102
:100BE000032921D8DFE801F0020B12194AF6D05090
:100BF000C0F6030008F0D8F84FF0000008BD4FF031
:100C00000000FFF7D5FF4FF0000008BD4FF00100D6
:100C1000FFF7CEFF4FF0000008BD4FF00200FFF7D6
:100C2000C7FF4FF0000008BD4FF0000010704FF0FC
:100C3000140008BD08B5F5F797F84FF001004FF024
:100C400000010A46F5F776F8F5F79AF84FF00C0030
:100C50004FF00001F4F7A6FEF5F786F808BD00BFD7
:100C6000037B13B9437B13B90EE0994208D301F11A
:100C7000FF318A18437B9A428CBF0020012001E09B
:100C80004FF00000C0B270474FF00100704700BF46
:100C900010B540F2D413C2F20003187800F1FF310E
:100CA000CAB2FD2A31D940F6F071C1F200014C6B95
:100CB000A4684FF00200FFF71FFC38B940F2D413CC
:100CC000C2F200034FF00200187017E04FF003006B
:100CD00040F6F071C1F20001FFF70EFC38B940F2A6
:100CE000D411C2F200014FF003020A7006E040F294
:100CF000D413C2F200034FF000001870204640F6F3
:100D0000F071C1F20001FFF7F7FB40F2D411C2F21B
:100D10000001087810BD00BF70B4447A24B14FF0D0
:100D2000320606FB04F610E0C5784AF6D844C0F651
:100D3000030454F82550B5F5964F9DBF49F26466FB
:100D4000B6FBF5F606EB86060826847A24B14FF04A
:100D5000320505FB04F501E041F28835C07A18B18F
:100D6000FF2808BF012001E04FF0010001B10E6033
:100D700002B1156003B1186070BC704740F2A06307
:100D8000C1F200034FF4117202FB00304FF000017A
:100D9000C0F810124FF6FF73C0F82C32C0F81812CA
:100DA000704700BFF8B505460E4640F2A064C1F298
:100DB00000044FF4117303FB0044D4F8240200EB49
:100DC0005007F6F7C3F9D4F82812421A974202D90D
:100DD000B81AF5F741FD23689A6928464FF00101DA
:100DE000904740F2A060C1F200004FF4117101FB86
:100DF00005014FF6FF7001F104013246F7F772FC6E
:100E0000A31918714FEA10225A7106F10206C4F8AC
:100E100004614FF00000C4F8080121680B6A2846FD
:100E20009847F5F751FB2846FFF7A8FFF8BD00BF2C
:100E300030B583B040F2A064C1F200044FF41175E4
:100E400005FB0040D0F83002B1F57A7F1BD3A1F545
:100E50007A7163B1837B13B9C37B13B907E09942FD
:100E600023D38A1802F1FF32C07B824220D8C8B255
:100E70000DF10701F9F790F99DF80710D1F1010084
:100E800038BF002019E04FEAD10402F107024FEA0F
:100E9000D20523B121462A46FFF7E2FE58B12819B0
:100EA000FA288CBF0020012007E04FF0000004E08A
:100EB0004FF0000001E04FF0000003B030BD00BF74
:100EC00008B5B0F57A7F21D279B14FEAD00341F667
:100ED000F062C2F2010200F007004FF0010101FAD6
:100EE00000F0D15C0843D05408BD4FEAD00341F66E
:100EF000F062C2F2010200F007004FF0010101FAB6
:100F000000F0D15C21EA0000D05408BD00F11800C7
:100F1000C0B24FF00102F9F7B7F908BD10B540F2C1
:100F2000A064C1F200044FF4117303FB0044D4F831
:100F30001C02F5F73DFD4FF00000C4F81C0210BD87
:100F400038B54FF4117101FB00F140F2A062C1F21B
:100F500000028C18D4F80831D4F80451AB420BD0FD
:100F60008958E3188A6A1979904728B1D4F808019A
:100F700000F10100C4F8080138BD00BF08B540F217
:100F8000A063C1F200034FF4117202FB0031D1F8EB
:100F9000082101F10401D1F800319A420BD140F24D
:100FA000A061C1F200014FF4117202FB0010D0F8F1
:100FB0001C02F5F7BBFA08BD70B582B005468DF886
:100FC000071040F2A064C1F200044FF4117303FB58
:100FD0000044D4F81802002850D11AB12846FFF76F
:100FE000CDFE4BE0F6F7B2F8D4F82812431AC4F855
:100FF0002802D4F81002D4F82422934204D800F135
:101000000103B3F5807F04D12846FFF7B7FE4FF008
:101010000103D4F81012621802A911F8010D82F828
:101020001001C4F81032B4F82C024FF00102F7F7A7
:1010300059FBC4F82C0208BB04F5887694F82032DA
:10104000012B03D1304602F0A5FA38B994F82012EA
:10105000022913D1304600F0C1FD78B14FF00102F2
:10106000C4F8182240F2A060C1F200004FF41173DE
:1010700003FB0505D5F81C02F5F758FA02B070BD60
:10108000836B42F24822C2F201021360016C42F209
:101090004423C2F201031960C16B40F2D812C2F2BC
:1010A000000211604FF0000383630364C363704761
:1010B00042F24823C2F201031968816342F24422DA
:1010C000C2F201021368036440F2D811C2F20001B7
:1010D0000A68C263704700BF2DE9F0418046174699
:1010E0001E4640F6F074C1F20004656BAD68084618
:1010F0002146FFF701FA002840D1606B0468002CFC
:1011000031D0616800292ED040F6F074C1F200049D
:101110002046FFF7B5FF204650F8342F13685C686F
:1011200041463A463346A04770B140F6F074C1F2EA
:1011300000042046FFF7BCFF28462146FFF7DCF9F4
:101140004FF00000BDE8F08140F6F074C1F20004F9
:101150002046FFF7ADFF28462146FFF7CDF94FF0B7
:101160000100BDE8F081284640F6F071C1F20001AF
:10117000FFF7C2F94FF00000BDE8F0814FF000002A
:10118000BDE8F0812DE9F8430446894690461F46A4
:10119000FFF77EFD0146D0B140F6F075C1F20005C3
:1011A0004FF00006AE632E64EE632068C9EB0002C8
:1011B0009DF8203002FB03F042463B46FFF78CFFD0
:1011C00021689DF824208B182360BDE8F8834FF038
:1011D0000000BDE8F88300BFF0B585B00D461E469F
:1011E000ADF80E2040F2A062C1F200024FF411717E
:1011F00001FB0020D0F83002037BFF2B03D1427BA0
:10120000FF2A00F0D0802C68B4F57A7F28D2F92C20
:1012100018D821464FF00202FFF722FD002800F007
:10122000C580002E40F0C58041F6F063C2F2010394
:10123000BDF80E20E252296801F1020129604FF049
:101240000100C7E04FF0010000904FF0020301934E
:1012500028464FF000010DF10E02FFF793FFB9E0B1
:10126000A4F57A77B7F57A7F2AD240F2E1418C4231
:101270001AD839464FF00102FFF7F2FC002800F0BF
:101280009B80002E40F09B80BDF80E004FEA10229C
:1012900041F6F063C2F20103DA55296801F1010158
:1012A00029604FF0010095E04FF001030093019396
:1012B00028464FF47A710DF10E02FFF763FF89E0C3
:1012C000A4F6B831B1F57A7F2ED240F634439C4271
:1012D0001CD804F10044A4F6B8344FEA44014FF09E
:1012E0000202FFF7BDFC00286CD0002E6DD141F644
:1012F000F061C2F20101BDF80E2021F814202B6824
:1013000003F101032B604FF0010063E04FF0020393
:1013100000934FF001000190284640F6B8310DF1DE
:101320000E02FFF72FFF55E0A4F5BB50A0F110000F
:10133000B0F57A7F0FD24EF69002C7F6FF72A11871
:101340004FEA41004FF001010DF10E024FF0020390
:10135000FFF7C2FE3EE0A4F5DA53A3F11803B3F59C
:101360007A7F0ED24EF2A840C7F6FF7023184FEADC
:1013700043004FF002010DF10E020B46FFF7ACFEE9
:1013800028E0A4F5FA52B2F57A7F21D24FEA44015F
:10139000A1F57A504FF003010DF10E024FF0020358
:1013A000FFF79AFE16E04FF0000013E04FF0000048
:1013B00010E04FF001000DE04FF000000AE04FF0A8
:1013C000010007E04FF0000004E04FF0010001E0F1
:1013D0004FF0000005B0F0BD2DE9F04182B080462D
:1013E00017461D464FF00003ADF8063040F6F07486
:1013F000C1F20004606B866808462146FFF77CF85E
:1014000038B1002D42D04FF001032B704FF0000097
:101410003EE040F6F071C1F200014A6B13683BB345
:10142000186828B340F6F074C1F200042046FFF7B4
:1014300027FE204650F8342F13681C6841460DF1F2
:1014400006024FF00203A04718B115B14FF001009A
:101450002870012F05D19DF806104FEA0122ADF842
:10146000062040F6F070C1F20000FFF721FE03E015
:1014700015B14FF001012970304640F6F071C1F20C
:101480000001FFF739F8BDF8060001E04FF0000059
:1014900002B0BDE8F08100BFF8B505460C4617461E
:1014A0001E46FFF7F5FB014678B12868C71B9DF87B
:1014B000180007FB00F032462346FFF78DFF29682E
:1014C0009DF81C208B182B60F8BD2CB14FF0010348
:1014D00023704FF00000F8BD4FF00000F8BD00BFD2
:1014E00030B583B004460D4611B14FF000030B70C8
:1014F0002268B2F57A7F17D2F92A08D841F6F0634C
:10150000C2F20103D05A02F102022260D0E04FF091
:10151000010200924FF002030193204629464FF04A
:101520000002FFF7B9FFC3E0A2F57A70B0F57A7F49
:1015300019D240F2E1439A420AD841F6F061C2F270
:101540000101085C4FEA002002F101022260AFE0D5
